:100000000C94E83A0C94103B0C94103B0C94103B6D
:100010000C94103B0C94103B0C94103B0C94103B34
:100020000C94103B0C943D700C9448700C94103B55
:100030000C94103B0C94345F0C94103B0C94103BCC
:100040000C949B700C94103B0C94103B0C94103B44
:100050000C9405580C94103B0C94103B0C94103BE2
:100060000C9481B40C94103B0C94103B0C94103BFA
:100070000C94CD560C9404570C94103B0C94103BEC
:100080000C94103B0C94103B0C94103B4E7D7C7EEA
:10009000537D5D7D677D767D877D947D7C7EA77DAC
:1000A000B47D047E327E4A7E5C7E6C7E6C99709953
:1000B0007A9976997E99829986998A999099949954
:1000C0009A999E99A299A699AA99B399B799BD9917
:1000D000C199C799CD99D399DDC3EDC3F2C3FCC3D0
:1000E0000AC411C417C429C42CC4D4C8D7C8DAC8D8
:1000F000DDC8E0C819C9F2C8F5C8F8C800C903C905
:100100009DC8B3C8B6C8B9C8BCC8BFC8C2C8C5C8EE
:10011000C8C8CBC8CEC8D1C8B0C80BC916C905A8B5
:100120004CCDB2D44EB93836A9020C50B99186885C
:10013000083CA6AAAA2ABE000000803F4552523AB7
:100140002000414F4B0D0A005769466C79007665D7
:10015000720D005265706C6163653D005478506F9C
:100160007765723D00526174653D004A6F696E3D6E
:10017000005265626F6F743D0050726F62653D00A2
:10018000426561636F6E3D00676574206164686FEE
:10019000630D0050524F544F3D00464C4147533D74
:1001A000307800525353493D282D0073686F7720F3
:1001B000727373690D00466C75736853697A653D97
:1001C000004D61746368436861723D00466C7573ED
:1001D0006854696D65723D0067657420636F6D6D6D
:1001E0000D004D6F64653D005254433D0073686FD0
:1001F00077207420740D00416464726573733D0050
:1002000067657420646E730D0054696D653D00551B
:100210007054696D653D0073686F772074696D6512
:100220000D005A6F6E653D006765742074696D65D9
:100230000D0042617564726174653D0067657420EC
:10024000750D0044657669636549643D00676574B2
:10025000206F70740D004368616E3D005353494434
:100260003D0067657420776C616E0D004D61632001
:10027000416464723D00676574206D61630D0044E4
:100280004843503D00484F53543D0047573D004EB2
:100290004D3D0049503D006765742069700D002494
:1002A000242400434D440D0A0024242400434D44DB
:1002B0000D0A005769466C79206E6F7420666F7561
:1002C0006E64004572726F7220536574426175648A
:1002D00072617465007365742075206D203100466D
:1002E000207475726E206F6666206563686F007398
:1002F000657420636F6D6D2072656D6F746520305D
:1003000000462073657420636F6D6D2072656D000B
:10031000496E6974204164686F63204E6574776F1D
:10032000726B004661696C20496E69742041646893
:100330006F632000736176650D0053746F72696E90
:1003400067004552523A2000414F4B0D0A003C7461
:10035000696D656F75743E00657869740D00455868
:1003600049540D0A007365742069702064686370D5
:100370000073657420776C616E2073736964007319
:10038000657420776C616E206368616E00736574BC
:1003900020776C616E206B65790073657420776CD3
:1003A000616E207068726173650073657420776C8C
:1003B000616E206869646520310073657420776C14
:1003C000616E206A6F696E007365742069702061C8
:1003D000646472657373007265626F6F740D002AD6
:1003E0005265626F6F742A007365742069702068AB
:1003F0006F737400736574206970206E65746D612D
:10040000736B007365742069702067617465776130
:100410007900323430300034383030003936303002
:10042000003139323030003338343030003537362F
:1004300030300031313532303000736574207561F1
:1004400072742062617564007365742075617274E2
:1004500020696E7374616E740073656172636820E5
:100460005769466C7900736561726368203936306C
:1004700030204261756400736561726368203131B8
:100480003532303020426175640073656172636893
:1004900020333834303020426175640073656172F6
:1004A00063682031393230302042617564007365F1
:1004B00061726368203438303020426175640073A3
:1004C00065617263682032343030204261756400A7
:1004D0005769466C792046696E644572726F720086
:1004E00055736520636F6E6669672077697468204D
:1004F000504300574C414E20205365747570004D99
:100500006F64756C2065696E6765626175743F0024
:100510006D6F64756C65206275696C7420696E3FDF
:10052000004D6F64756C65206765696E7374616CEE
:100530002E3F0053534944004B616E616C00636869
:10054000616E6E656C0070617373776F72640049E1
:100550006E697469616C6973696572656E00696E54
:10056000697469616C697A6500496E697469616C66
:1005700069736572656E004B6F6E6669672E206DDC
:10058000697420504300636F6E6669672E20776937
:10059000746820504300436F6E6669672E206D6556
:1005A0007420504300202020202020576C616E20B2
:1005B0005353494420202020202000576C616E2096
:1005C000496E69742000576C616E20496E69742011
:1005D0006F6B00576C616E20496E697420457272B2
:1005E0006F7200207769746820202020202020204E
:1005F00042617564002020323430300020203936CA
:10060000303000203139323030002033383430304F
:10061000002035373630300031313532303000731C
:1006200065617263682057692E323332204D6F64E2
:10063000756C006E6F2057692E32333220666F75ED
:100640006E640057692E32333220537974617865B5
:1006500072726F722020200057692E32333220666A
:100660006F756E64200057692E3233322077726FB7
:100670006E67204261756472617465004572726FC5
:100680007220736574204E562D52414D0045727292
:100690006F72207365742052414D2020202020006D
:1006A00056657273696F6E3A00496E6974205769B6
:1006B00032333220776169742E2E2E2E002E002EBA
:1006C000002E002E002E002E002E002E002E002EBA
:1006D000002E002E002E002E002E002E002E002EAA
:1006E000002E00576932333220496E6974457272A8
:1006F0006F72202000576932333220496E697420AE
:100700006F6B2E2E2E2E00576932333220496E69C0
:10071000744572726F7220200057692E3233322076
:100720004E414B00204552524F525F4E4F4D454E69
:1007300055202000204552524F525F4D41584D45A3
:100740004E552000204552524F525F4D415849545A
:10075000454D2000204552524F525F4E4F4954455F
:100760004D20200020202020206E6F7420706F7399
:100770007369626C652020202000202025313953C8
:1007800000202025313973002025323053002025E8
:10079000323073002534530025355300256325631B
:1007A00025313653256320002563256325313753D2
:1007B00020002563256325313673256320002563DA
:1007C000256325313773200020202020206E6F7490
:1007D00020706F737369626C6520202020002000F8
:1007E0001D00120013004572726F723A205363723B
:1007F0006F6C6C426F78004E6F206D6F7265205287
:10080000414D0020202020005556F732EE1AAB0D46
:10081000DC066F03B801DC006E0037001B000E0021
:100820000700030002000100536572766F3A00531F
:100830006572766F203200536572766F20310053F7
:100840006572766F2041646A7573740052657665CF
:100850007273650072657665727365004C696E6BC4
:1008600073006C656674006C696E6B73005265632F
:100870006874730072696768740072656368747382
:10088000004D69747465006D6964646C65006D6920
:100890006464656E00536572766F7465737420438B
:1008A0006F6E742E005374617274205465737400FB
:1008B000737461727420746573740045696E7A652F
:1008C0006C736368726974740073696E676C652019
:1008D0007374657000416E7A61686C20546573743E
:1008E000006E756D626572206F66207465737400AA
:1008F00061616E74616C207465737473005061750E
:10090000736520456E64706F736974696F6E0070F3
:100910006175736520656E6420706F73007061751A
:1009200073652065696E6420706F732E0050617569
:1009300073652070726F20496E632E00706175734D
:10094000652070726F6320696E632E005365727646
:100950006F7465737400546573742050756C736C98
:10096000EFBFBD6E676500746573742070756C733E
:10097000207769647468005465737420666F7274BC
:100980006C66642E007465737420636F6E742E0041
:10099000536572766F00736572766F005065726989
:1009A0006F6465006672616D6500547261636B69A6
:1009B0006E6720536572766F7300536572766F733E
:1009C0006368726974746500736572766F207374FE
:1009D00065707300536572766F20310073657276AF
:1009E0006F203200536572766F2032007365727625
:1009F0006F203200536572766F746573740073658F
:100A000072766F7465737400010000000A000000C4
:100A100064000000E803000010270000A086010029
:100A200040420F008096980000E1F50500CA9A3B0D
:100A3000426561723A001E00446973743A006D00A9
:100A400050616E203A0054696C743A00203F3F2098
:100A500000204F4B20004641494C0053204C61740C
:100A6000697475646520204C6F6E67697475646580
:100A70000048004D005361743A004669783A0048D6
:100A8000444F503A006C6F73742042542064617478
:100A90006100475053207472656E6E656E0045723A
:100AA000726F7220617420636F6E6E656374696E1D
:100AB0006700737769746368206F6E204254204D1D
:100AC0006F7573652121004665686C6572206265EB
:100AD000696D205472656E6E656E0053204C6174B2
:100AE000697475646520204C6F6E67697475646500
:100AF00000576861697420666F7220475053204622
:100B000069782000576861697420666F72204750C9
:100B100053204669782000202020202020202020FB
:100B200020202020202020202000475053206F6BC1
:100B30002C207374617274206F6B2020006C6F73B3
:100B4000742057692E32333220646174610054720C
:100B500061636B696E6720426C7565746F6F746852
:100B60002020200020547261636B696E67204D69FC
:100B70006B726F6B6F7074657200456E64650020F8
:100B8000204C49504F202021215761726E756E67AD
:100B900021212020002073657269656C6C652050EE
:100BA0006F74697320312D352000194F18002020F3
:100BB000204A6F79737469636B2053657475702074
:100BC0002020200053204D696E204D6178205479FB
:100BD00070202044697220204E00506F74690054C8
:100BE000617374004E6F726D00526576004E00594D
:100BF00000504B54204C69706F6D657373756E6750
:100C0000202020004F4B004A6F79737469636B009A
:100C10004D696E696D616C2057657274006D696E07
:100C2000696D616C2076616C7565006D696E696DCA
:100C30002E20776161726465004D6178696D616C29
:100C40002057657274006D6178696D616C20766102
:100C50006C7565006D6178696D2E207761617264D5
:100C60006500547970650074797065005269636835
:100C700074756E6700646972656374696F6E007283
:100C800069636874696E67004E65757472616C693A
:100C9000736965726564006E65757472616C697AFA
:100CA000696E67006E65757472616C6973657265F3
:100CB0006E64004A6F79737469636B732053657453
:100CC000757000DC62657273696368740073756DBA
:100CD0006D61727900537469636B203100737469BC
:100CE000636B203100537469636B20320073746945
:100CF000636B203200537469636B20330073746933
:100D0000636B203300537469636B20340073746920
:100D1000636B203400537469636B2035007374690E
:100D2000636B203500504B54204C69706F6D6573B8
:100D300073756E6700504B54204C69706F206D6561
:100D400061737572652E00504B54204C69506F20B2
:100D50006D6574696E67004F4B006B65696E20426C
:100D6000544D3232320065696E6765626175742177
:100D7000004465766963653A004D41433A00426933
:100D800074746520657273742042542D44657669CD
:100D90006365730073756368656E21004254207348
:100DA000656C6563742044657669636500616B7486
:100DB00075656C6C65732042542044657669636583
:100DC0003A20004254204465766963657320737548
:100DD0006368656E3F007375636865204254204404
:100DE0006576696365006B65696E652047505320C1
:100DF0004D617573006B6F6E6669677572696572B8
:100E000074210074727920746F20636F6E6E656355
:100E100074004572726F7220636F6E6E65637469E1
:100E20006E6721004F4B005361743A2000584572A1
:100E3000723A20004669783A200048444F503A20E0
:100E400000204C617469747564652020204C6F6EBD
:100E500067697475646500416C743A200020202D28
:100E60002D2D006D006C6F737420425420646174EA
:100E70006100475053207472656E6E656E00626942
:100E80007474652077617274656E2E2E2E00425444
:100E90002D4D6F75736531004D696B726F6B6F709F
:100EA00074003234303020200039363030202000B9
:100EB000313932303020003338343030200035378B
:100EC0003630302000313135323030003438303077
:100ED0002020004164686F63005750412020004C7F
:100EE00069706F20004C69496F6E00576932333268
:100EF00000576932333200250020002020202020B6
:100F000020202020202020204300201720202020E7
:100F10002016202020202019202020204F4B0020A8
:100F20004645484C45522120312E205A6569636858
:100F3000656E212000566F6C74004F53442053653A
:100F4000747570004F53442053637265656E73006F
:100F5000475053204D6F757365205365747570004D
:100F6000537563686520475053204D617573007356
:100F7000656172636820475053206D6F757365001B
:100F80005A6F656B204750532D6D756973005A6514
:100F900069676520476572E474656C697374650000
:100FA00073686F77206465766963656C6973740034
:100FB00053686F772061707061726161746C6973DE
:100FC00074005A6569676520475053204465766907
:100FD00063650073686F77204750532064657669B6
:100FE00063650053686F77204750532061707061CC
:100FF0007261617400475053204D617573205479BC
:101000007000475053206D6F7573652074797000C0
:1010100054797065204750532D6D756973004750A2
:1010200053204D61757320616B7469763F004750A2
:1010300053206D6F7573652061637469763F004757
:1010400050532D6D75697320616B746965663F003F
:1010500047505320446174656E00475053206461CB
:10106000746100426C7565746F6F746820536574A9
:101070007570004D6F64756C2065696E676562619F
:1010800075743F006D6F64756C65206275696C7472
:1010900020696E3F004D6F64756C65206765696EF1
:1010A0007374616C2E3F004E616D65006E616D65FD
:1010B000004E61616D0050696E0070696E00496E8E
:1010C000697469616C6973696572656E00696E69DE
:1010D0007469616C697A6500496E697469616C69EB
:1010E000736572656E00426C7565746F6F7468200D
:1010F0004D41430052452D4944004B6F6E66696770
:101100002E206D697420504300636F6E6669672EF0
:10111000207769746820504300436F6E6669672EBC
:10112000206D65742050430020426C7565746F6FAC
:101130007468204E616D6520202020202000204210
:101140006C7565746F6F74682050696E2020202064
:1011500020202000425420496E6974206F6B0042A9
:101160005420496E6974204572726F720020425497
:101170004D2D323232204D41432D416472657373DF
:101180006520004D41433A003A002052452D494424
:10119000204E6F74697A20202020202020202000FB
:1011A00057692E3233322053657475700054582FAE
:1011B0005258204B616E616C0054582F5258204396
:1011C00068616E6E656C004E6574572E20477275AF
:1011D000707065004E6574572E2047726F757000F1
:1011E0004E6574572E204D6F646500545820546925
:1011F0006D656F7574005458204D545500426175EB
:1012000064726174652057693233322F4254005042
:101210004B5420616C6C67656D65696E005370722C
:1012200061636865006C616E677561676500546134
:10123000616C005A6569747A6F6E650074696D65DA
:10124000207A6F6E6500536F6D6D65727A65697493
:101250000073756D6D65722074696D65004C434453
:1012600020617573206E6163682E2E2E004C4344FE
:10127000206F6666206166746572004C4344207579
:101280006974206E612E2E2E004C43442048656CFC
:101290006C69676B656974004C43442062726967CE
:1012A00068746E657373004C43442048656C6465D4
:1012B0007268656964004C4344204B6F6E747261C0
:1012C0007374004C434420636F6E747261737400D6
:1012D0004C434420436F6E7472617374004C4344FA
:1012E000204E6F726D616C2F496E76657273004C83
:1012F0004344206E6F726D616C2F696E76657274F7
:10130000004C4344204E6F726D61616C2F676569BC
:101310006E7600486172647761726520426565701F
:1013200065720048617264776172652070696570EA
:10133000657200416B6B75747970004163637574FD
:1013400079700061636375207479706500416B6B1F
:1013500075204D657373756E6700416363754D65E8
:1013600061737572650061636375206D6574696E84
:101370006700504B54205365747570005665726257
:10138000696E64756E67204D4B00636F6E6E6563AA
:1013900074696F6E204D4B0041616E736C7569749A
:1013A000696E67204D4B00504B5420616C6C676533
:1013B0006D65696E00504B5420676C6F62616C0004
:1013C000504B5420616C67656D65656E0057692EE2
:1013D00032333200426C7565746F6F746800576CFD
:1013E000616E004F534420416E7A65696765004F16
:1013F00053442073637265656E004F5344207363DA
:101400006865726D004F53442053637265656E7357
:1014100000475053204D61757300475053206D6F46
:1014200075736500547261636B696E6720536572F2
:10143000766F7300747261636B696E672073657297
:10144000766F73004A6F79737469636B00504B5405
:101450002055706461746500454550726F6D20526F
:101460006573657400504B542D546F6F6C20464368
:101470002000322E303161002020202020205570A5
:10148000646174653F20202020202020200020500F
:101490004B5420557064617465202020202020204A
:1014A0002020200066FC7220322053656B756E642C
:1014B000656E0020504B542076253853202573004C
:1014C000332E372E32000028432920474E5520471F
:1014D000504C204C6963656E736500202020204EBF
:1014E0004F2057415252414E54590000204D6F64D5
:1014F000756C657320696E7374616C6C656400252E
:1015000031355320253453004F53442D44617461C9
:10151000004D4B20506172616D65746572004D4BDA
:101520002044656275672044617461004D4B20441E
:101530006973706C617900536F756E6400547261E9
:10154000636B696E6700466F6C6C6F77204D65004A
:10155000574C414E205779466C79004A6F79737425
:1015600069636B00493243204D6F746F7274657309
:1015700074004F5344204F6C642053637265656E52
:1015800073004F5344204E617669676174696F6ED2
:10159000004F534420456C656374726963004F5378
:1015A00044204D4B537461747573004F5344205560
:1015B000736572475053004F53442033442D4C61A0
:1015C0006765004F53442053746174697374696391
:1015D00000466F6E742042696700002043726564A4
:1015E0006974730032303133204F6C697665722034
:1015F00047656D6573690032303132204368722E61
:10160000204272616E64746E65720020202020207A
:10161000486172616C6420426F6E676172747A0017
:1016200032303132204D617274696E2052756E6BAA
:10163000656C00323031322067656261640032309F
:1016400031302053656261737469616E20426F6549
:10165000686D00323030392D3230313020506574B1
:101660006572204D61636B00323030382054686FF2
:101670006D6173204B616973657200361839183CCF
:10168000183F184218451848184B180E0F0E4E0EEA
:101690000F0E4F0E0F0E530E0F0E570E0F0E4E0E57
:1016A0000F0E4F0E0F0E530E0F0E570E0F0E4E0E47
:1016B0000F0E4F0E0F0E530E0F0E574E1857186980
:1016C000187D189118A518BA18CC18DB18EB18FF5C
:1016D000180C191919251931193D19461956195D92
:1016E000196819741983198C199919A719B519C48E
:1016F00019CF19E219F019FD19081A1C1A1D1A1E22
:101700001A1F1A201A211A221A231A241A414800D1
:101710005048004346004348006F31006F3200429A
:1017200041004341005354004D5200465900454C7E
:1017300000465300475000532100545500544400C4
:10174000465200524C00534C005452004D43004846
:10175000F66865006D005300560056006D41680044
:1017600041006D004B6D6800486F6D65006D202D68
:101770000020200050430020536174005A69656CBA
:10178000006D202D006D7300575000206D41004109
:101790006C743A004469723A002020493A00206B88
:1017A0006D6800416C743A00486F6D653A006D00D9
:1017B00055475053006D006D4168006D4168004110
:1017C0000073006B6D680020202030006D416800C0
:1017D0006D617820424C2020437572723A006D6131
:1017E0007820424C202054656D703A000B43005025
:1017F0004B54204F5344004D4B2053657474696E15
:1018000067002D206572726F72202D002A2A204DEC
:101810004B2D4572726F72202020202A2A003A0038
:101820006C6F6E672070726573733A005547707302
:1018300000496E666F004E45004520005345005339
:1018400020005357005720004E57004E20004E6F87
:10185000204572726F72004643206E6F7420636F72
:101860006D70617469626C65004D4B334D6167202A
:101870006E6F7420636F6D706174692E006E6F20DF
:10188000464320636F6D6D756E69636174696F6E39
:10189000006E6F204D4B334D616720636F6D6D752A
:1018A0006E69632E006E6F2047505320636F6D6D1D
:1018B000756E69636174696F6E0062616420636F45
:1018C0006D706173732076616C75650052432053AF
:1018D00069676E616C206C6F73740046432073708F
:1018E00069207278206572726F72006E6F204E43AD
:1018F00020636F6D6D756E69636174696F6E00460C
:1019000043204E69636B204779726F004643205233
:101910006F6C6C204779726F0046432059617720C5
:101920004779726F004643204E69636B2041434301
:1019300000464320526F6C6C2041434300464320D5
:101940005A2D41434300507265737375726520735D
:10195000656E736F720046432049324300426C202B
:101960004D697373696E67004D69786572204572C1
:10197000726F7200436172656672656520457272AE
:101980006F7200475053206C6F7374004D61676E27
:101990006574204572726F72004D6F746F722072A1
:1019A00065737461727400424C204C696D69746196
:1019B00074696F6E00576179706F696E742072611F
:1019C0006E6765004E6F2053442D4361726400536F
:1019D00044204C6F6767696E672061626F7274653F
:1019E0006400466C79696E672072616E67652100DC
:1019F0004D617820416C746974756465004E6F2088
:101A00004750532046697800636F6D70617373208F
:101A10006E6F742063616C6962722E0000000000BA
:101A200000000000504B54205258206C6F7374001B
:101A3000202020200020202020206E6F2064617450
:101A4000612E2E2E00426567696E3A202530327570
:101A50003A253032752020253032752E25303275EA
:101A60002E00456E643A202020253032753A25300C
:101A700032752020253032752E253032752E00200B
:101A80004F53442053746174697374696300204C2C
:101A900061737420466C792020253032753A2530E8
:101AA0003275206D696E002563416C7469747564CC
:101AB00065253764206D00256344697374616E6326
:101AC00065253775206D00256347726E642E53704F
:101AD00065656425332E3164206B6D68002563567F
:101AE0006572742E537065656425332E3164206BE6
:101AF0006D680020436170616369747925376420E3
:101B00006D416800256343757272656E7425362ECB
:101B10003164204100256343757272656E74253609
:101B20002E31642041002563424C253164204375E9
:101B300072722E25342E31752041002563424C25CA
:101B400031642054656D702E202535752025634342
:101B5000002563566F6C7461676525362E316420ED
:101B60005600256352432D5175616C697479253592
:101B70006400256352432D5175616C697479253574
:101B8000640025634E69636B253131642025630051
:101B900025634E69636B253131642025630025631D
:101BA000526F6C6C25313164202563002563526FC0
:101BB0006C6C253131642025630020424C20537425
:101BC0006174697374696300256343757272656E2D
:101BD0007425362E31642041002563437572726589
:101BE0006E7425362E31642041002563424C253128
:101BF000642043757272656E7425322E31752041F2
:101C0000002563424C2531642054656D702E2025DB
:101C10003575202563430020424C204461746100E7
:101C20002531643A256343757272656E7425342ECE
:101C300031752041002020256343757272656E74F2
:101C400025342E31752041002020256354656D70A8
:101C50002E25387520256343002055736572204773
:101C6000505300253032752E253032752E253034F4
:101C7000752020253032753A253032753A253032BC
:101C80007500253764206D4725352E3164206D425F
:101C90000025332E366C6425332E366C6400204DBF
:101CA0004B204572726F727300253032753A2530C1
:101CB00032753A253032752020253032752E253088
:101CC00032752E253034750020436F646520253031
:101CD000327500253230530044656C004F53442068
:101CE000446174656E004F534420446174656E0016
:101CF0004F5344206461746100424C20204461745D
:101D0000656E00424C202064617461004D4B2020C0
:101D10004665686C65726C69737465004D4B202074
:101D20006572726F72736C6973740047505320420E
:101D3000656E75747A65726C69737465004750538B
:101D400020757365726C69737400475053206C651D
:101D5000747A746520506F732E00475053206C6165
:101D6000737420506F732E004CD653434845206146
:101D70006C6C6520446174656E0044454C45544567
:101D800020616C6C20646174610020424C2D4374AE
:101D9000726C2054657374202020202020202000A5
:101DA0004D6F746F723A202020310056616C75655A
:101DB0003A20202030001A201B001D00416C6C00CE
:101DC0001D00200020001D0000000000000078150C
:101DD000141578002055545578003845444538008E
:101DE0003049484930003C4140413C0038414021A5
:101DF00078007E1515150A0022170F17220000849F
:101E000082FF82841C141C000000000705070000EC
:101E100010385410101E180C18000000101010106C
:101E200010101010107C101008100800000008148A
:101E300000001408100804040810081020201008DE
:101E400000081422410000412214080004027F020D
:101E5000040010207F2010001038541010101010B3
:101E60001054381010181C1C18100818383818088E
:101E700000081C3E7F00007F3E1C0800060909097F
:101E800006001020100804020000000000000000FE
:101E90002F000000000700070000147F147F1400CB
:101EA000242A6B2A12002313086462003649552243
:101EB0005000000503000000001C2241000000410A
:101EC000221C000014083E08140008083E08080000
:101ED000005030000000080808080800006060009A
:101EE00000002010080402003E5149453E00004217
:101EF0007F4000004261514946002141454B31007D
:101F00001814127F10002745454539003C4A4949BD
:101F10003000030171090700364949493600064976
:101F200049291E0000363600000000563600000029
:101F30000814224100001414141414000041221447
:101F40000800020151090600324979413E007E1124
:101F500011117E007F49494936003E41414122002E
:101F60007F4141221C007F49494941007F090909FD
:101F700001003E4149497A007F0808087F0000417E
:101F80007F4100002040413F01007F0814224100B2
:101F90007F40404040007F020C027F007F04081019
:101FA0007F003E4141413E007F09090906003E4154
:101FB00051215E007F0919294600464949493100EF
:101FC00001017F0101003F4040403F001F204020B1
:101FD0001F003F4038403F006314081463000708A7
:101FE000700807006151494543007F4141000000EE
:101FF0000204081020000041417F00000402010299
:102000000400404040404000000102040000205411
:10201000545478007F4844443800384444442000F5
:10202000384444487F00385454541800087E09014D
:1020300002000C5252523E007F0804047800004413
:102040007D4000002040443D00007F1028440000F7
:1020500000417F4000007C04180478007C080404E0
:1020600078003844444438007C14141408000814E0
:1020700014187C007C0804040800485454542000C0
:10208000043F444020003C4040207C001C20402075
:102090001C003C4038403C004428102844000C50B0
:1020A00050503C004464544C440000083641000049
:1020B00000007F00000000413608000008082A1CCC
:1020C0000800081C2A08080020203031323334353B
:1020D000363738394142434445460D0A00201A201C
:1020E0002020201B202020202045786974002020FB
:1020F0002E20202E20202020003234303000343892
:102100003030003936303000313932303000333839
:102110003430300035373630300031313532303000
:10212000002A2A204F5554204F462052414D202A44
:102130002A00746869732066756E6374696F6E2017
:102140006973006E6F7420617661696C61626C65A1
:1021500021004E7572206D6974204E432021004687
:1021600069782054797065203A20005361742020EA
:10217000202020203A20004163637572616379203A
:102180003A200050444F5020202020203A20005375
:1021900070656564202020203A20004C6F6E672017
:1021A000202020203A20004C617420202020202074
:1021B0003A2000416C742020202020203A20004F3B
:1021C00000580078002D0020003344003244006E97
:1021D0006F00440020006F6B00202000636D002E14
:1021E000006B6D2F68002E002E006D00504B5400C8
:1021F00031323334003136392E3235342E303031ED
:102200002E303031003235352E3235352E303030EB
:102210002E303030003136392E3235342E303031D8
:102220002E30303100454550726F6D5570646174C9
:102230006520746F206E65770020202020202056B6
:10224000657273696F6E202020202020006368650E
:10225000636B207468652073657474696E6773219D
:10226000004F4B002020205772697465204545506F
:10227000524F4D202020200020454550524F4D20E8
:10228000506172616D657465722020202000776551
:102290007264656E20617566005374616E6461726C
:1022A0006477657274652067657365747A7400304D
:1022B00030303000504B5400303030302D30302D25
:1022C000303030303030003030303000504B54003F
:1022D0003132333435363738003136392E323534F1
:1022E0002E3030312E303031003235352E3235350A
:1022F0002E3030302E303030003136392E323534F9
:102300002E3030312E303031002121436865636B2F
:1023100020506172616D65746572212120004F4B00
:1023200000504B5400425420736574206E65772032
:1023300042617564726174652E2E004572726F720F
:1023400031207365742042617564726174652E2E4C
:1023500000736574204261756472617465206F6BEF
:102360000073657420426175647261746520457202
:10237000726F72004154503D0041545A3000415434
:102380004C2A0041544C300041544C310041544CD3
:10239000320041544C330041544C340041544C35CC
:1023A00000415451310041544530004154513000F6
:1023B00041544531004154004154410041544800CA
:1023C00041544430004154443D004154463F004193
:1023D000544F310041544F30004154523000415469
:1023E00052310041544E3D0041545331004154425A
:1023F0003F000D004F4B0D0A004552524F520D0A3F
:1024000000736574204563686F206F6666004572CF
:10241000726F7220736574204563686F0073656125
:1024200072636820776974683A0032343030202053
:102430000034383030202000393630302020003150
:1024400039323030200033383430302000353736E0
:1024500030302000313135323030002E002E2E0049
:102460002E2E2E002E2E2E2E00666F756E6400739B
:102470006561726368206572726F720042542069F0
:102480006E697469616C6973696572656E2E2E0080
:1024900042544D323232206E6F7420666F756E6416
:1024A000210042544D32323220496E6974204F4B24
:1024B00000444953434F4E4E45435400434F4E4E04
:1024C0004543540054696D65206F75742C466169ED
:1024D0006C20746F20636F6E6E65637421000D0A4B
:1024E000002E00496E717569727920526573756CA2
:1024F00074733A0D0A000D0A00496E71756972799C
:1025000020456E6400720A000D0A004F4B004861BE
:1025100072647761726520504B5420332E396D0000
:1025200030392E32303131005769466C7950617440
:10253000636800486172647761726520504B542073
:10254000332E39780031312E32303132005769461E
:102550006C79506174636800536F6674776172655B
:102560003A00332E372E3200426175647261746511
:102570003A20002042542052616E67656578746588
:102580006E64657200426C7565746F6F7468202D9F
:102590003E2057692E32333200414354495645217B
:1025A0000052452D49443A2000574C414E2052617B
:1025B0006E6765657874656E642E00576C616E2079
:1025C0002D3E2057692E323332004143544956453F
:1025D000210042544D2D323232204B6F6E666967B6
:1025E0007572696572656E004643203E204D4B2D25
:1025F000555342203E2042544D2D323232004D4B35
:102600002D55534220616E20504320616E736368E4
:102610006C2E20005A7769736368656E204D4B2DD0
:1026200055534220756E64202000504B542065693C
:102630006E2067656B7265757A7465732020200063
:102640004B6162656C20616E7363686C696573735E
:10265000656E2E2020005769466C79204B6F6E66A0
:1026600069677572696572656E005043206D6974A3
:10267000204164686F63205769666900504B54209D
:1026800076657262696E64656E0050757474793A2D
:102690002074656C6E6574004950203136392E32D5
:1026A00035342E312E3100506F727420323030307C
:1026B0000020555342204272696467652020202023
:1026C000202000555342202D3E2057692E323332B0
:1026D000004143544956452100526164696F747248
:1026E0006F6E69782057692E323332445453004557
:1026F00076616C756174696F6E20283836384D4884
:102700007A2920200052656164696E673A00416E43
:10271000616C6F67204E616D65733A200020200068
:102720004552524F523A206E6F20646174610046E8
:1027300043004E43004552524F523A206E6F206480
:1027400061746100204E6176692D4374726C20447F
:102750006973706C61792020200046430020446931
:1027600073706C61792020202020202020202020E0
:1027700020200020200020466C696768742D437477
:10278000726C20446973706C617920004E430020A4
:102790004E6176692D4374726C20446973706C616C
:1027A000792020200046430020446973706C6179D1
:1027B0002020202020202020202020202000202039
:1027C0000020466C696768742D4374726C204469FC
:1027D00073706C617920004E4300204E6176692D44
:1027E0004374726C20446973706C617920202000FE
:1027F0004643004665686C65723A204B65696E65B4
:1028000020446174656E0020504B54207600332EB6
:10281000372E32003A2046432D5265762000322E64
:1028200030316100504B542D546F6F6C7300425423
:10283000202052616E6765657874656E646572000C
:10284000574C414E2052616E6765657874656E64C1
:102850002E00555342204272696467653A205769D9
:1028600032333200555342204272696467653A2020
:1028700053563200425420204272696467653A2000
:1028800053563200424C2F4D6F746F7274657374DF
:10289000004F5344004F534420446174656E004F11
:1028A00053442044617461004D4B20446973706C43
:1028B0006179004D4B20506172616D6574657200E5
:1028C0004D4B2044656275672044617461004D4B37
:1028D0002047505320496E666F00547261636B69E4
:1028E0006E67004A6F79737469636B00504B5420B4
:1028F000546F6F6C7300504B5420536574757000A7
:10290000504B5420496E666F005375636865204DC7
:10291000696B726F6B6F707465720073656172635F
:1029200068204D696B726F6B6F707400A82EA82EB3
:10293000A82EBD2ED32EE92EFF2E152F2B2F412F83
:10294000532F652F772F812F8B2F952F9F2F652F3B
:10295000A92FB92FC92FD92FEA2FFF2F14302230DA
:1029600030303F3055306B3081309730AD30C33030
:10297000D930EF3005311B311B31313147315D31F9
:10298000733188319C31AF31B431B831BE31C1318E
:10299000BE31C431CB31D131D631DC31E231E93114
:1029A000FC310A321C3225322E3237324032463266
:1029B0004F326232623276327A327A327F32863205
:1029C00086328C32923298329E32A432AA32B0329F
:1029D000B032B032B432C732D832ED32F7320133CE
:1029E0000B3315331F3329333833453353336933AE
:1029F0007F339533AB33C033D433EA3300341634EA
:102A00002C34423458346D3481348F349C34A9349E
:102A1000B634CC34D834EE34013514352635373558
:102A20004135533569357C359135A735B935CD35C7
:102A3000E335ED35FF3512361E362C363F364B3634
:102A40005F36733687369A36AA36B936CB36DD36D8
:102A5000EF36013717372D374337533766377B3714
:102A60008B379B37AD37AD37AD37C337D937EF37F6
:102A700005381B38313847385D387338893889381C
:102A800089389F38AF38AF38BD38D338E938FF3888
:102A900011392039313947395D3972397239723912
:102AA00088399E39B439CA39E039F6390C3A223AB4
:102AB000383A4E3A643A6C3A783A7E3A843A8A3AEC
:102AC0008A3A8A3A933A933A933A9B3AA33AAB3A80
:102AD000B33ABD3AC73AD13AE23AF03A023B0C3B3C
:102AE000153B1E3B2A3B363B423B4E3B5A3B663B2B
:102AF000723B7E3B8A3BA03BB63BCC3BDD3BEE3B97
:102B0000FF3B0A3C153C1C3C2C3C3D3C4D3C5B3C9B
:102B1000693C773C853C853C933C933C933CA23C90
:102B2000B23CB23CC23CC23CC23CCC3CCC3CCC3CB7
:102B3000DB3CDB3CDB3CEA3CEA3CEA3CF93CF93C74
:102B4000F93C083D083D083D183D2A3D3C3D4E3DC1
:102B5000643D733D833D8E3D983DAA3DAF3DB43D00
:102B6000B93DBE3DC33DC83DDE3DDE3DF43D0A3EC0
:102B70001B3E2D3E383E423E543E663E783E8A3EE7
:102B8000A03EA03EB63EC43ED23EE03EE03EE03E29
:102B9000F03E063F1A3F2F3F423F4F3F653F653FA4
:102BA000743F833F853F853F873F893F8B3F8D3F04
:102BB0008D3F8D3F8F3F8F3F8F3F913F913F913FA3
:102BC000943F943F943F973F9A3F9A3F9D3FB33F36
:102BD000C43FDA3FEA3FF63F05400F40194022402C
:102BE00038404E4064406B4072407D408840914088
:102BF0009B40A540AF40BB40D140E140F440044180
:102C00000F411D412D413B414C415D416A4176419F
:102C10008C41A241B841CB41D841E841FE41144228
:102C200029423F4255426B4281429742AD42C342E4
:102C3000D942EF42044319432E43444344435A4389
:102C40007043704386439743A843B843C643C64383
:102C5000D443E243F043FE430C441A442844364430
:102C600036444444524460446E447C448A4498440C
:102C7000A644B444C144C144C144C944C944C9443C
:102C8000D144E044EF44FE441245254535454045D6
:102C90004B455645614561456C45774582458D45B7
:102CA00098459845A345A345A345AD45AD45AD45DC
:102CB000B745B745B745BC45BC45BC45C145C14511
:102CC000C145C645D245DE45EA45F645F6450246CC
:102CD000024602460E460E460E46184622462C4630
:102CE00036463646364640464A464A4654465E468C
:102CF000684672467C467C46864690469A46A4467E
:102D0000BA46BA46D046E146E146F2460147014797
:102D10001047214732474347544754476547764752
:102D200087479847A847B847C847D847D847E8478C
:102D3000F847F8470A480A480A48194819481948FC
:102D40002C482C482C483C484D485E486F486F48FA
:102D500080489148A248B348C348D448E548F6485B
:102D60000749074918492E492E49434951495149B4
:102D70005F49754975498B499C499C49AD49AD49A5
:102D8000AD49C349C349C349D949D949D949E24998
:102D9000E949F049F749FF49064A0E4A154A1D4AD2
:102DA000254A384A384A4B4A5E4A714A844A974A09
:102DB000974AAA4ABD4AD04AE34AF64AF64A094B1C
:102DC0001C4B2F4B424B554B684B7B4B7B4B7B4BF0
:102DD0008E4B994BA44BAF4BC24BD54BE84BFB4BA7
:102DE0000E4C214C344C474C5A4C6D4C804C934CFF
:102DF000A04CAD4CBA4CC74CC74CD44CE54CF34C32
:102E0000034D164D294D3C4D434D434D4A4D514DBB
:102E1000514D584D6E4D6E4D844D974D974DAA4D69
:102E2000B74DB74DC44DD64DD64DE74DF74DF74D87
:102E3000054E154E154E244E354E354E444E524ECF
:102E4000524E5E4E674E6F4E774E894E894E9A4E69
:102E5000AA4EBA4ECA4EDA4EEA4EFA4E0A4F1A4FF0
:102E60002A4F3A4F4A4F5A4F5A4F5A4F624F624F6A
:102E7000624F6D4F6D4F6D4F764F764F764F804F4F
:102E8000804F804F894F894F894F914F914F914F7C
:102E90009C4F9C4F9C4FA14FA14FA14FA64FA64FB7
:102EA000A64FAB4FAB4FAB4F202020666F726D61CA
:102EB00074206861726469736B20433F00201A209C
:102EC000202020201B20202020456E64652020200B
:102ED0004F4B00201A20202020201B20202020657E
:102EE0006E64202020204F4B00201A20202020201C
:102EF0001B2020202045696E646520204F4B002058
:102F00001820202020201920202020456E646520D4
:102F100020204F4B00201820202020201920202086
:102F200020656E64202020204F4B00201820202098
:102F30002020192020202045696E646520204F4BF9
:102F400000201820202020201920202020456E64F9
:102F50006520002018202020202019202020206516
:102F60006E642020002018202020202019202020FE
:102F70002045696E646500456E64652020204F4BD6
:102F800000656E64202020204F4B0045696E64650B
:102F900020204F4B00456E646520496E666F0065CA
:102FA0006E642020696E666F005461737465203111
:102FB0002053656B756E6465004B656570207468A1
:102FC0006520627574746F6E00486F756420646567
:102FD000206B6E6F70202020006C616E672066652C
:102FE000737468616C74656E2E00707265737365BE
:102FF0006420666F722031207365636F6E640031E8
:10300000207365636F6E646520696E6765647275B1
:103010006B742E002066FC7220464320322E303125
:10302000610020666F7220464320322E30316100ED
:1030300020566F6F7220464320322E3031610020BF
:1030400020204C65747A746520506F736974696FC1
:103050006E202020002020206C61737420202070BE
:103060006F736974696F6E202020002020204C61EE
:10307000617473746520706F7369746965202020B2
:1030800000204272656974656E677220204CE46EA0
:1030900067656E67722000206C6174697475646581
:1030A00020206C6F6E6769747564652000627265BC
:1030B0006564746567722E206C656E6774656772EF
:1030C0002E20006CF6736368656E2020202020207F
:1030D00020207765697465720064656C657465208D
:1030E000202020202020202020657869742000776F
:1030F000697373656E2020202020202020207665B3
:10310000726465720020202020476F6F676C652015
:1031100045696E67616265202020002020202047DD
:103120006F6F676C6520496E7075742020202020B9
:103130000020202020202067656CF67363687420CF
:103140002020202020200020202020202064656CCA
:10315000657465642020202020202020002020206D
:10316000202020676577697374202020202020208C
:103170002020007375636865204D696B726F6B6FFB
:10318000707465722E2E2E00736561726368696EAD
:1031900067204B6F707465722E2E2E007A6F656BF0
:1031A00020696B726F6B6F707465722E2E2E0045E6
:1031B0006E646500656E640045696E6465004F6B02
:1031C000006F6B004665686C6572006572726F72A5
:1031D00000666F757400616B746976006163746971
:1031E0007600616374696566004643206E696368B2
:1031F0007420676566756E64656E21004643206EB7
:103200006F7420666F756E6421004643206E696599
:1032100074206765766F6E64656E210065727761F4
:1032200072746574006578706563746564007665B2
:1032300072776163687400676566756E64656E00B9
:10324000666F756E64006765766F6E64656E0050BC
:103250004B54206E7572206B6F6D7061746962657E
:103260006C00504B54206F6E6C7920636F6D7061F1
:103270007469626C65006D697400776974680046F2
:1032800045484C4552004552524F520045696E2008
:1032900020004F6E2020200041616E2020004175EB
:1032A000732020004F66662020005569742020009E
:1032B000455343002020504B54206175737363685D
:1032C000616C74656E3F00202073687574646F775D
:1032D0006E20504B54203F002020504B54207569E5
:1032E00074736368616B656C656E203F004A612092
:1032F00020204E65696E00796573202020206E6F56
:10330000004A61202020204E6565004E65696E20D0
:1033100020204A61006E6F20202020796573004EC6
:103320006565202020204A6100446174656E206C30
:10333000F6736368656E3F0064656C657465206450
:103340006174613F00446174656E207769737365D1
:103350006E3F0056657262696E6465205043206D51
:10336000697420504B54202000436F6E6E65637467
:1033700020504320746F20504B542D55534200561B
:10338000657262696E64205043206D657420504BF5
:1033900054202020004472FC636B65202753746125
:1033A00072742720616D20504B5400507265737306
:1033B0002027537461727427206F6E20504B540085
:1033C0004472756B2027537461727427206F7020CC
:1033D000504B540020202020202020202020204559
:1033E0006E646520537461727400202020202020B8
:1033F0002020202020456E642020537461727400C8
:103400002020202020202020202045696E64652077
:103410005374617274002050432D517569636B2D94
:1034200056657262696E64756E6720002050432D88
:10343000517569636B2D436F6E6E656374696F6E52
:10344000200020536E656C6C652050432D766572AC
:1034500062696E64696E670056657262696E646562
:103460002064617320504B54206D697400436F6E6B
:103470006E65637420504B542077697468204D4BFF
:103480000056657262696E6420504B5420200064BF
:10349000656D204D4B20FC6265723A002020206F44
:1034A000766572202020203A002020206D6574204F
:1034B000202020203A0064656D204D4B20FC626581
:1034C000723A20204B6162656C2C20006F76657229
:1034D0003A204B6162656C004D4B207669613A2061
:1034E0006B6162656C202020202020202000657305
:1034F00020697374206B65696E2057692E323332F0
:10350000007468657265206973206E6F2057692E9C
:10351000323332006572206973206765656E20570B
:103520006932333220004D6F64756C2065696E67B7
:1035300065626175742E006275696C7420696E2E07
:10354000006D6F64756C6520696E6765626F757775
:10355000642E0057656E6E20646F63682C20646172
:103560006E6E206269747465006966207965732CDB
:10357000207468656E206669727374007A6F206AC1
:10358000612C2064616E20617562206565727374C0
:1035900000646173204D6F64756C207A7565727379
:1035A0007420696D20200061637469766174652000
:1035B0006D6F64756C20696E006465206D6F647555
:1035C0006C6520616B7469766572656E0053657415
:1035D00075706D656EFC20616B74697669657265E6
:1035E0006E2E0053657475706D656E7500696E2082
:1035F0006865742053657475704D656E752E005343
:103600006965206DFC7373656E2064617320504B97
:103610005400596F75206861766520746F005520DD
:103620006D6F657420646520504B54006A65747A30
:1036300074206E6575207374617274656E210072FA
:1036400065737461727420504B54006E75206F70F6
:103650006E69657577207374617274656E210045BB
:103660007320697374206B65696E2042544D2D324E
:103670003232005468657265206973206E6F204293
:10368000544D2D32323200457220697320676565D2
:103690006E2042544D2D323232004D6F64756C20D5
:1036A00065696E676562617574004D6F64756C2045
:1036B0006275696C7420696E006D6F64756C65204D
:1036C000696E6765626F7577642E00204D4B2D55CE
:1036D00053422046756E6B74696F6E2000204D4B0F
:1036E0002D5553422046756E6374696F6E2000201D
:1036F0004D4B2D5553422046756E637469652020ED
:1037000000204254202D2D3E204B6162656C2061CB
:103710006E204643202000204254202D2D3E204B79
:103720006162656C20746F20464320200020425463
:10373000202D2D3E206B6162656C206E61617220D0
:103740004643005043206D697420425420766572D0
:10375000622E00636F6E6E6563742050432077693C
:1037600074682042540050432076696120425420FE
:10377000766572626F6E64656E2E00504B542D4BF1
:103780006162656C20616E20464300504B542D4BA6
:103790006162656C20746F20464300504B542D6B62
:1037A0006162656C206E6161722046430020425464
:1037B000202D2D3E2057692E32333220202020200C
:1037C00020200057692E32333220616E204643207C
:1037D00020202020202020200057692E3233322044
:1037E000746F2046432020202020202020200057D6
:1037F00069323332206E61617220464320202020DE
:10380000202020200020555342202D2D3E204B61AA
:1038100062656C20616E2046432000205553422093
:103820002D2D3E206361626C6520746F204643201D
:1038300000555342202D2D3E206B6162656C206E39
:10384000616172204643005043206D6974205553D6
:10385000422076657262696E64656E2000636F6EE9
:103860006E65637420504320776974682055534215
:1038700020200056657262696E64205043206D6599
:1038800074205553422020200020555342202D2DD6
:103890003E2057692E323332202020202020004D38
:1038A0004B2D546F6F6C207374617274656E00736E
:1038B00074617274204D4B2D546F6F6C00205769EA
:1038C0002E323332204B6F6E66696775726965728E
:1038D000656E002057692E32333220436F6E666961
:1038E0006775726174696F6E0020576932333220D8
:1038F000436F6E6669677572617469652020005058
:10390000726F6772616D6D207374617274656E2E73
:103910000073746172742070726F6772616D200041
:1039200073746172742070726F6772616D6D612E55
:103930000042544D2D323232204B6F6E66696775EE
:1039400072696572656E0042544D2D3232322063C9
:103950006F6E66696775726174696F6E0042544D6F
:103960002D32323220636F6E6669677572617469D9
:1039700065004643203E204D4B2D555342203E20AE
:1039800042544D2D323232004D4B2D555342206161
:103990006E20504320616E7363686C2E2000636F4D
:1039A0006E6E65637420504320746F204D4B2D550F
:1039B0005342200056657262696E64205043206D48
:1039C0006574204D4B2D555342005A7769736368D7
:1039D000656E204D4B2D55534220756E642020009E
:1039E000636F6E6E6563742063726F7373656420BA
:1039F0006361626C650074757373656E204D4B2D49
:103A000055534220656E20504B542000504B54209B
:103A100065696E2067656B7265757A7465732020C1
:103A200020006265747765656E204D4B2D555342BD
:103A300020616E642020200065656E2067656B72D2
:103A40007569737465206B6162656C2020004B6141
:103A500062656C20616E7363686C69657373656E13
:103A60002E202000504B54205356320061616E735B
:103A70006C756974656E2E004B6162656C006361E4
:103A8000626C65004B6162656C00536C6176652009
:103A90002020004E6F726D616C2000526576657259
:103AA000736500696E7665727365006765696E7629
:103AB000657200456E64652020204F4B00456E64A2
:103AC000202020204F4B0045696E642020204F4B62
:103AD0000020454550726F6D207769726B6C696389
:103AE0006800205265616C792064656C65746500BE
:103AF00020456570726F6D207765726B656C696AC1
:103B00006B00206CF6736368656E3F00204545705E
:103B1000726F6D3F002077697373656E3F00646557
:103B2000757473636820202020006765726D616E74
:103B3000202020202000647569747320202020201C
:103B40002000656E676C6973636820202000656ED5
:103B5000676C6973682020202000656E67656C7350
:103B6000202020202000686F6C6CE46E6469736311
:103B700068006475746368202020202020006E6532
:103B80006465726C616E64732000416E7A6569676A
:103B9000652045696E7374656C6C756E67656E0043
:103BA00020446973706C61792053657475702020AE
:103BB000202020202000446973706C617920696E98
:103BC0007374656C6C696E67656E2000496E666F14
:103BD00073206265692053746172743A00496E669D
:103BE0006F20617420737461727475702000496E67
:103BF000666F2062696A206F70737461727400531B
:103C0000707261636865203A20004C616E6775616F
:103C100067653A20005461616C3A20004C69636822
:103C20007420617573206E6163683A004C6967683F
:103C300074206F66662061667465723A004C696331
:103C4000687420756974206E613A2020004C4344EA
:103C50002048656C6C69676B2E3A00204272696778
:103C600068746E657373203A0020496E74656E73D4
:103C700069746569743A004C4344204B6F6E7472EA
:103C80006173743A004C434420636F6E74726173C5
:103C9000743A004C4344204E6F726D2F496E763A51
:103CA00020005243204665686C657270696570201B
:103CB0003A005243204572726F726265657020202F
:103CC0003A00446562756720504B54005769205490
:103CD000582F5258204368616E3A005769204E654C
:103CE00074572E204772702E3A005769204E657423
:103CF000572E204D6F64653A005769205458205460
:103D0000696D656F75743A005769205541525420AA
:103D10004D54552020203A0057692E323332206509
:103D2000696E6765626175743A0057692E32333285
:103D3000206275696C7420696E203A0057693233CD
:103D40003220696E6765626F7577643A2000497347
:103D5000742065696E2057692E3233322D4D6F64A1
:103D6000756C20004973205769323332206D6F64BF
:103D7000756C0049732065722065656E2057693245
:103D800033320065696E6765626175743F00627504
:103D9000696C7420696E3F006D6F64756C65206995
:103DA0006E6765626F7577643F004A612020007915
:103DB000657320004A612020004E65696E006E6FB9
:103DC0002020004E656520002042544D32323220C2
:103DD00045696E7374656C6C756E67656E00202046
:103DE00042544D2D3232322073657474696E67739C
:103DF000202020004973742065696E2042544D2DA7
:103E00003232322D4D6F64756C0049732042544D2F
:103E10002D323232204D6F64756C0049732065720B
:103E20002065656E2042544D2D3232320065696E38
:103E30006765626175743F006275696C7420696EB4
:103E40003F006D6F64756C6520696E6765626F75A4
:103E500077643F0042544D3232322065696E6765A7
:103E6000626175743A0042544D3232322062756993
:103E70006C7420696E203A0042544D32323220690F
:103E80006E6765626F7577643A0020504B5420412D
:103E90006B6B752045696E7374656C6C756E67002D
:103EA00020504B5420416363752053657475702016
:103EB000202020202000504B5420416B6B757479DA
:103EC000703A2000504B5420416363757479703A06
:103ED0002000504B542041636375747970653A003B
:103EE000416B6B752055204F66667365743A2000F0
:103EF0004F6666736574207665727374656C6C6565
:103F00006E206269730061646A757374206F6666FF
:103F100073657420756E74696C004F6666736574A2
:103F2000206166726567656C656E20746F740064ED
:103F30006965205370616E6E756E67207061737372
:103F40007400766F6C7461676520666974730064D1
:103F500065207370616E6E696E67206A756973742F
:103F60002069732E004C6F77426174205761726E26
:103F700020563A004C6F7742617420616C61726D1B
:103F8000203A00560046004800420041004C0052D2
:103F9000004E6900526F004B6F00436F004645486A
:103FA0004C45523A20446174656E7665726C757347
:103FB0007420004552524F523A2044617461206C83
:103FC0006F73740056657262696E64696E672076FD
:103FD000657262726F6B656E21004C65747A7465F0
:103FE0002062656B616E6E7465004C617374206B4A
:103FF0006E6F776E20004C61617473742062656B24
:10400000656E646500506F736974696F6E2000702F
:104010006F736974696F6E2000706F73697469657E
:1040200020002045696E7374656C6C756E67656EF3
:1040300020202020202020002053657474696E67A2
:104040002020202020202020202020202000204967
:104050006E7374656C6C696E67656E20202020201D
:1040600020202000E46E6465726E006368616E67F4
:104070006500766572616E646572656E00616B7471
:104080006976696572656E006163746976617465ED
:104090000061637469766572656E00616B74697640
:1040A0006965727400616374697661746564006740
:1040B0006561637469766565726400205365747424
:1040C000696E6720782073706569636865726E3FFA
:1040D000002073746F72652073657474696E673F36
:1040E000002073657474696E6773206F70736C6100
:1040F000616E3F004765737065696368657274201F
:10410000756E640073746F72656420616E64006F15
:10411000706765736C6167656E20656E004B6F70CC
:10412000696572652053657474696E6700636F70AA
:10413000792073657474696E6773006B6F7069655D
:1041400065722073657474696E67730020766F6E94
:1041500020207820206E616368202079002066721C
:104160006F6D207820746F2079002076616E207842
:10417000206E61207900766F6E2020206E6163686A
:104180002020456E64652020204F4B0066726F6DC5
:104190002020746F20202020656E64202020204F76
:1041A0004B0076616E2020206E6120202020656902
:1041B0006E646520204F4B005769726B6C696368B1
:1041C000206B6F70696572656E3F007265616C6C23
:1041D0007920636F70793F0065636874206B6F703E
:1041E00069656572656E3F004B6F7069657274201A
:1041F000756E6420616B7469766965727400636FB3
:104200007069656420616E642061637469766174AD
:104210006564200047656B6F706965EB72642065AB
:104220006E2061637469656600E46E646572652082
:1042300045696E7374656C6C756E67656E200020E1
:1042400020206368616E67652073657474696E67AA
:104250007320202000696E7374656C6C696E6765ED
:104260006E2077696A7A6967656E002057E4686C2A
:104270006520506172616D65746572202020202078
:10428000002073656C65637420706172616D657484
:104290006572732020200053656C656374656572D8
:1042A00020706172616D657465727320002057E43F
:1042B000686C6520536569746520202020202020CB
:1042C000202000202020202073656C6563742070FE
:1042D000616765202020202000202053656C6563E5
:1042E0007465657220706167696E6120202000200E
:1042F00057E4686C652053657474696E673A2020D2
:10430000202020002073656C6563742073657474CD
:10431000696E672020202020002053656C6563743F
:104320006565722073657474696E672020002020B3
:104330004750532045696E7374656C6C756E676584
:104340006E20200020202020475053207365747475
:10435000696E6773202020202000676577E4686C11
:104360007465732047505320476572E47420200021
:1043700073656C656374656420475053206465768B
:1043800069636520200047505320456D70662E619B
:104390006B7469763F3A007265636569766520479C
:1043A0005053206F6E3F3A00475053206F6E747623
:1043B0002E2061616E3F3A006D61782048F6686595
:1043C000202020203A006D617820616C746974753A
:1043D00064653A006D6178204765736368772E20C5
:1043E0003A006D61782073706565642020203A0082
:1043F0006D617820736E656C686569643A006D6103
:104400007820456E746665726E2E3A006D61782074
:1044100064697374616E63653A006D6178206166EA
:104420007374616E643A20006D696E205370616E22
:104430006E756E673A006D696E20766F6C74616799
:1044400065203A006D6178205A656974202020202B
:104450003A006D61782074696D65202020203A0053
:104460006D61782074696A64202020203A006D61B3
:1044700078205374726F6D2020203A006D6178208F
:1044800063757272656E74203A006D617820737482
:10449000726F6F6D20203A00456E742E4B61706113
:1044A0007A69742E3A00557365644361706163697B
:1044B00074793A00476562722E6361706163693A8C
:1044C000004C6F6E672E203A004C61742E20203A0B
:1044D000004E7572206D6974204E4320212020000B
:1044E0004F6E6C792077697468204E43202100411B
:1044F0006C6C65656E206D6574204E4321004B65C4
:10450000696E652053657474696E6773202121207C
:1045100020004E6F2073657474696E677320726536
:1045200061642121004765656E2073657474696E4E
:10453000677321200048F6686520206175732000AC
:10454000416C74692E206F66662000416C74692E80
:1045500020756974200048F6686520626567722ED0
:1045600000416C74692E4C696D6974005661726902
:104570006F206175732000566172696F206F6666E7
:104580002000566172696F2075697420005661724F
:10459000696F2048F6686500566172696F20416C4A
:1045A000742E002020202020202020200043617233
:1045B0006520467265650020202020004C4544316E
:1045C000004C454432004E617669202061757320AD
:1045D00020004E61766920206F66662020004E61C3
:1045E00076692020756974202000506F732E206832
:1045F000616C74656E00506F732E20486F6C642080
:104600002000436F6D696E6720486F6D6500202044
:1046100020202020202020004A757374696572656F
:104620006E0043616C6962726174650043616C691C
:10463000627265722E005374617274202020200013
:104640004265747269656220200052756E202020D8
:1046500020202000466C696567656E202000466C4E
:104660007920202020202000566C696567202020BA
:1046700020004C616E64756E672020004C616E6492
:10468000696E67202000416B6B75206C6565720058
:104690004C6F77204261742E20004C6F772042616E
:1046A00074742E0020204F534420416E7A65696750
:1046B0006520536574757020200020204F534420DE
:1046C00073637265656E20736574757020202000B9
:1046D0004F7574312F32206E656769657274203AA8
:1046E000004F7574312F3220696E7665727465647F
:1046F0003A004F7574312F3220466F726D61743AF3
:10470000004F7574312F3220666F726D61743A00FC
:104710004E6176696461746120616E205356323A4D
:10472000004E6176696461746120746F2053563263
:104730003A004E61766964617461206F702053564F
:10474000323A006D2E2053696E6B72617465206D74
:104750002F733A006D2E66616C6C73706565642012
:104760006D2F733A00566172696F6D6574657220C2
:10477000426565703A00766172696F6D6574657245
:1047800020626565703A00766172696F6D65746567
:104790007220706965703A006D4168205761726ED1
:1047A000756E67203E203A006D4168207761726E19
:1047B000696E67203E203A006D4168207761617222
:1047C0007363682E3E203A004F534420416E7A6551
:1047D0006967657661723A004F534420736372656E
:1047E000656E6D6F64653A004D4B20566F6C74209A
:1047F00042616C6B656E3A004D4B20766F6C742095
:1048000062617267726170683A0042617564205734
:10481000693233322F42543A0020466F6C6C6F7706
:10482000204D6520536574757020200020202020C5
:10483000205265667265736820203A00476573638D
:104840006877696E6469676B6569743A0020202037
:104850002053706565642020202020203A0020200D
:1048600020536E656C68656964202020203A0054EE
:104870006F6C6572616E7A205261646975733A007B
:10488000546F6C6572616E746965205261642E3A72
:1048900000546F6E61757367616265204572772E93
:1048A0003A00736F756E6420657874656E73696F16
:1048B0006E3A00736F756E6420657874656E736907
:1048C000653A00486172647761726520506965706D
:1048D00065723A006861726477617265206265652D
:1048E0007020203A00686172647761726520706997
:1048F000657020203A004C6175747374E4726B65C6
:1049000020202020203A00766F6C756D65202020D5
:104910002020202020203A0073657269656C6C6548
:10492000204B616EE46C652053657475700073658F
:104930007269616C206368616E6E656C207365746A
:104940007570004C69706F204D657373756E673AB2
:10495000004C69706F20636865636B20203A004BE0
:10496000616E616C2020202020202020202020202B
:1049700020202020004368616E6E656C202020207E
:104980002020202020202020202000536572766FD8
:1049900073636872697474653A2020007365727677
:1049A0006F73746570732020203A2020002020202F
:1049B0002020202020536572766F20312020202077
:1049C0002020002020202020202020536572766F98
:1049D00020322020202020200052657665727365E9
:1049E0003A004C696E6B733A006C656674683A0005
:1049F0006C696E6B733A005265636874733A007247
:104A0000696768743A007265636874733A004D6947
:104A10007474653A006D6964646C653A006D69642C
:104A200064656E3A00546573742050756C736CE461
:104A30006E676520202020007465737420667261A3
:104A40006D65776964746820202000205365727654
:104A50006F207A756D2054657374656E2000207325
:104A60006572766F20746F20746573742020202027
:104A70000020736572766F207465207465737465A9
:104A80006E202000202020202020506572696F6455
:104A90006520202020200020202020202066726118
:104AA0006D6520202020202020005465737420662E
:104AB0006F72746C617566656E6420200074657336
:104AC0007420636F6E74696E7565732020202000FA
:104AD0007465737420636F6E74696E752020202076
:104AE00020200045696E7A656C736368726974741E
:104AF00020202020200073696E676C652073746528
:104B0000702020202020202000416E7A61686C20D7
:104B10002020202020202020202020007465737475
:104B200020636F756E7420202020202020200074C8
:104B30006573742061616E74616C202020202020D8
:104B40002000506175736520456E64706F736974E1
:104B5000696F6E2000706175736520656E64706F9B
:104B6000736974696F6E2000706175736520656983
:104B70006E64706F73697469652000506175736548
:104B80002070726F20496E632E2020202000475035
:104B900053204D617573203A00475053206D6F7557
:104BA00073653A00475053206D756973203A00478A
:104BB0005053204254204D61757320312020202015
:104BC0002000475053204254204D6F7573652031AB
:104BD0002020202000475053204254204D756973F7
:104BE000203120202020200047505320506F732E6A
:104BF00020766F6D204D4B202020004750532070B1
:104C00006F732E2066726F6D204D4B202000475031
:104C10005320706F732E2076616E204D4B20202024
:104C200000537469636B206D696E2E205765727432
:104C30003A202000737469636B206D696E2E2076B4
:104C4000616C75653A2000737469636B206D696EE1
:104C5000207761617264653A2000537469636B2048
:104C60006D61782E20576572743A20200073746944
:104C7000636B206D61782E2076616C75653A20003B
:104C8000737469636B206D6178207761617264650C
:104C90003A20005269636874756E673A20202000DC
:104CA000646972656374696F6E3A2020007269638B
:104CB0006874696E673A20202000537469636B74CE
:104CC0007970653A202000737469636B747970653C
:104CD0003A2020004E65757472616C697369657263
:104CE000656E643A006E65757472616C697A696E9E
:104CF000673A006E65757472616C69736572656E92
:104D0000643A004C69706F204D657373756E673A35
:104D10002020202020004C69706F206D6561737524
:104D200072656D656E743A20004C69706F206D6518
:104D300074696E673A20202020202000506F74692B
:104D4000202000706F7469202000546173746572B4
:104D50000073776974636800202020504B54205AF8
:104D60006569742020536574757020202000202010
:104D700020504B542074696D6520736574757020E4
:104D8000202020005A6569747A6F6E6520202855AE
:104D900054432B2D293A0074696D65207A6F6E6536
:104DA00020285554432B2D293A00536F6D6D6572A1
:104DB0007A656974203A0073756D6D657220746947
:104DC0006D653A004F53442D20756E6420424C2D82
:104DD000446174656E004F53442D20616E6420421F
:104DE0004C206461746100204D4B204665686C6501
:104DF000726C6973746500204D4B206572726F721E
:104E00006C697374002055736572204750532D44AC
:104E10006174656E002055736572204750532D6490
:104E200061746100206C65747A746520506F7369D9
:104E300074696F6E00206C61737420706F73697495
:104E4000696F6E00202020414C4C45204461746500
:104E50006E00202020414C4C2064617461006CF68F
:104E6000736368656E3F0064656C6574653F0077C9
:104E7000697373656E3F007A65696765204D4B2DD8
:104E800053657474696E673A0073686F77204D4B91
:104E90002073657474696E673A00576C616E2065A3
:104EA000696E6765626175743A00576C616E206265
:104EB00075696C7420696E203A00576C616E2069C8
:104EC0006E6765626F7577643A005750412076656A
:104ED0007277656E64656E203A0075736520575071
:104EE00041202020202020203A0075736520575053
:104EF00041202020202020203A00536963686572F9
:104F000068656974202020203A00736563757269B2
:104F100074792020202020203A007365637572691F
:104F200074792020202020203A004B616E616C2093
:104F300020202020202020203A006368616E6E65CA
:104F40006C202020202020203A006368616E6E656E
:104F50006C202020202020203A0047656E65726179
:104F60006C004E617669676174696F6E00456C65AF
:104F70006374726963004D4B2D53746174757300D3
:104F80005573657220475053003344204C61676568
:104F90000053746174697374696373004F534430D0
:104FA000004F534431004F534432004C61737472CC
:104FB000696E670050504D202020202020202020A6
:104FC00020202020005370656B7472756D202020A6
:104FD0002020202020005370656B7472756D20486E
:104FE000695265732020005370656B7472756D2073
:104FF0004C6F5265732020004A6574692020202080
:105000002020202020202020004143542044534CC5
:1050100020202020202020202000484F54542020F1
:10502000202020202020202020200046757475623A
:105030006120534255532020202020005573657273
:1050400020202020202020202020202000000001DF
:105050001003010101000001100404040400000118
:10506000100103030300000110020202020003000A
:1050700020050505050003002006060606000300BE
:10508000200707070700030020080808080003009E
:105090002009090909000300200A0A0A0A0003007E
:1050A000200B0B0B0B000300200C0C0C0C0007005A
:1050B0001E640000000002000871000000000200F1
:1050C0000470000000000600062701010100020034
:1050D0004071000000010200010D0000000102000B
:1050E000200D010101010200080D01010101020072
:1050F000100D000000010200047000000001020019
:10510000400D010101010200800D000000010200BC
:10511000040D00000002000014170A080602000037
:10512000141810100A020100FF19060604020100FB
:10513000FF61000000030200016E00000003020096
:10514000026E000000030200046E00000003020073
:10515000086E000000030100FF3B32323203000002
:10516000F73C5A5A5A030000F73D3232320300002E
:10517000F7414E4E4E030000F7424E4E4E040200E1
:10518000010D000000040200017000000004020094
:10519000020D010101040200027001010104070077
:1051A0001F10000000040000F70E1E1E1E04010068
:1051B000FF110F0F0F040100FF0F1E1E1E04010040
:1051C000FF13000000040100FF689696960400009B
:1051D000F7120F0F0F040000F7140808080401006D
:1051E000FF15404040040000A01600000004070026
:1051F0001C6C000000040000F76D0909090501009E
:10520000FF2D808080050100F72E3232320502002A
:105210008071000000050200016F0000000502001F
:10522000046F000000050000F72F0F0F0F050000AE
:10523000F730E6E6E6050000196A00000005010007
:10524000FF31808080050000F7325555550502007A
:10525000026F000000050000F733464646050000D7
:10526000F734DCDCDC050000196B000000050002EF
:105270000835040404050000F7363C3C3C050500F5
:10528000F737000000050100FF387D7D7D05010036
:10529000FF397D7D7D050100FF3A7D7D7D060200A1
:1052A000200D010101060800205100000006010048
:1052B000FF52646464060000F75B080808060000FB
:1052C000F75A060606060100FF535A5A5A0601000D
:1052D000FF545A5A5A060100FF555A5A5A060100FD
:1052E000FF564B4B4B060100FF5755555506010025
:1052F000FF584B4B4B060100FF5900000006010010
:10530000FF5C5A5A5A060100FF5D2A2A2A0601004C
:10531000FF5EF5F5F5060100FF5F8C8C8C06000042
:10532000F760050505060200207000000006020077
:105330000271000000060000F7660000000704008C
:10534000FF4A5F5F5F070100FF4B14141407020060
:10535000206E000000070200106E0101010702002C
:105360002071000000070100FF500000000704004A
:10537000FF4CF3F3F3070100FF4D14141407020070
:10538000406E000000070200806E0101010704006A
:10539000FF4EAAAAAA070400FF4FAAAAAA08000063
:1053A000F71A080808080000F71BE6E6E6080100FF
:1053B000FF1D4040400807001F6300000008020076
:1053C0004070000000080000F7242121210802009D
:1053D0000870000000080000F7265A5A5A0800001A
:1053E000F7252D2D2D080000F767000000080000AC
:1053F0000C690000000802001070000000080200A4
:105400000471000000080200807000000008020023
:105410000171000000080200107100000009010085
:10542000FF1E5A6464090100FF1F787878090100A3
:10543000FF200A0A0A090100FF215A6464090100D9
:10544000FF22787878090100FF45464646090200A8
:10545000800D000000090000F71C1B1B1B09000049
:10546000F743202020090100FF2810101009000038
:10547000F74400000009000010230606060900009A
:10548000F7650000000A0100FF290000000A010082
:10549000FF2A0000000A0100FF2B0000000A0100A3
:1054A000FF2C0000000A0100FF460000000A010076
:1054B000FF470000000A0100FF480000000A010049
:1054C000FF490000000B0200400D0000000B01002E
:1054D000FF3E5A5A5A0B0100FF3F3737370B010086
:1054E000FF404646460C050017620000000D020012
:1054F000010D0000000D0100FF10FFFFFF0D000077
:10550000A0160000000D0200200D0101010D010098
:10551000FF51FEFEFE0D020020700000000D000095
:10552000F7660000000D0100FF630000000D02009F
:1055300040700000000D00000C640000000D05002C
:1055400017620000004761732020202020202020C7
:10555000202020005468726F74746C652020202015
:1055600020200047617320202020202020202020A0
:105570002000476965722020202020202020202044
:105580000047696572202020202020202020200054
:105590004769657220202020202020202020004EF6
:1055A00069636B20202020202020202020004E69CD
:1055B000636B20202020202020202020004E6963C3
:1055C0006B2020202020202020202000526F6C6C97
:1055D0002020202020202020202000526F6C6C20D2
:1055E00020202020202020202000526F6C6C2020C2
:1055F000202020202020202000506F74692031209E
:105600002020202020202000506F7469203120208D
:1056100020202020202000506F746920312020207D
:10562000202020202000506F74692032202020206C
:105630002020202000506F7469203220202020205C
:1056400020202000506F746920322020202020204C
:10565000202000506F74692033202020202020203B
:105660002000506F7469203320202020202020202B
:1056700000506F746920332020202020202020003B
:10568000506F7469203420202020202020200050DA
:105690006F74692034202020202020202000506FAB
:1056A00074692034202020202020202000506F7496
:1056B000692035202020202020202000506F746990
:1056C0002035202020202020202000506F746920C9
:1056D00035202020202020202000506F74692036A3
:1056E000202020202020202000506F7469203620A8
:1056F0002020202020202000506F74692036202098
:1057000020202020202000506F7469203720202086
:10571000202020202000506F746920372020202076
:105720002020202000506F74692037202020202066
:1057300020202000506F7469203820202020202055
:10574000202000506F746920382020202020202045
:105750002000506F74692038202020202020202035
:10576000004D6F746F7220536963682E5363680035
:105770004D6F742E5361666574792053772E004DFA
:105780006F742E7361662E736368616B2E004D6FAC
:10579000746F72205377692E4D6F6465004D6F747E
:1057A0006F72205377692E4D6F6465004D6F746F73
:1057B00072205377692E4D6F6465004572772E20F5
:1057C0005369672E2050722E2000456E682E20539C
:1057D00069672E436865636B00556974672E53696A
:1057E000672E436865636B00456D7066E46E6765A0
:1057F0007220547970200052656365697665722065
:105800005479706520004F6E7476616E672E205457
:10581000797065200053706B20616C6C2045766553
:105820006E74730053706B20616C6C204576656EEE
:1058300074730053707265656B20616C6C657320C6
:10584000200048F668656E726567656C6572202099
:10585000004374726C20416C746974756465200037
:105860004374726C20486F6F677465202020004776
:10587000505320202020202020202020200047508E
:10588000532020202020202020202020004750537B
:105890002020202020202020202020004B6F6D7011
:1058A0006173732020202020202000436F6D7061E1
:1058B000737320202020202020004B6F6D706173B7
:1058C0002020202020202020004B6F6D7046657323
:1058D0007420417573722E00436F6D704F7269654D
:1058E0006E742E466978004B6F6D7061732076611F
:1058F0007374202020004572772E205369672E2074
:1059000050722E200053656E732E52637653696772
:1059100056616C00457874526563205369676E6107
:10592000616C004163687328652E296B6F70706C21
:105930002E004178697320436F7570696E6720206F
:10594000004173206B6F7070656C696E672020007A
:1059500044726568726174656E626567722E00528A
:105960006F7452617465206C696D69742E00526F9A
:105970007452617465206C696D69742E00486561AC
:1059800064696E6720486F6C642020004E69636B09
:105990002F526F6C6C2020202020004B6F6572739B
:1059A000207661737420202020004E69636B2F5293
:1059B0006F6C6C2050202020004E69636B2F526F5B
:1059C0006C6C2050202020004E69636B2F526F6C4E
:1059D0006C2050202020004E69636B2F526F6C6C3E
:1059E0002044202020004E69636B2F526F6C6C2086
:1059F00044202020004E69636B2F526F6C6C204452
:105A0000202020004769657220502020202020207F
:105A1000202000476965722050202020202020206F
:105A2000200047696572205020202020202020205F
:105A30000045787465726E65204B6F6E74722E002F
:105A400045787465726E204374726C202020004586
:105A5000787465726E20436F6E74726F6C004C6F59
:105A60006F70696E67206F62656E2020004C6F6FEB
:105A700070696E6720757020202020004C6F6F7059
:105A8000696E67206F6D686F6F67004C6F6F70692C
:105A90006E6720756E74656E20004C6F6F70696E56
:105AA0006720646F776E2020004C6F6F70696E679F
:105AB0002062656E65642E004C6F6F70696E6720A2
:105AC0006C696E6B7320004C6F6F70696E67206C31
:105AD0006566742020004C6F6F70696E67206C697A
:105AE0006E6B7320004C6F6F70696E672072656318
:105AF000687473004C6F6F70696E672072696768B5
:105B00007420004C6F6F70696E67207265636874F3
:105B10007300476173204C696D6974202020202038
:105B2000005468726F74746C65204C696D69740000
:105B3000476173204C696D69657420202020004105
:105B40006E737072656368736368772E20005265A8
:105B500073702E205468726573682E20004472653D
:105B60006D70656C7761617264652000487973744B
:105B70006572657365202020202000487973746564
:105B800072657369732020202000487973746572F0
:105B9000657365202020202000556D6B656872704C
:105BA0002E204E69636B20005475726E6F7665729D
:105BB000204E69636B20004E69636B206765696ED8
:105BC000766572742E00556D6B656872702E20526A
:105BD0006F6C6C20005475726E6F76657220526F18
:105BE0006C6C2000526F6C6C206765696E76657214
:105BF000742E0048F668656E726567656C756E6731
:105C00002000416C746974756465204374726C2063
:105C100000486F6F67746520436F6E74726F6C001D
:105C20004A3A484265672C4E3A566172696F00598C
:105C30003A4C696D482C4E3A566172696F00593A78
:105C40004C696D482C4E3A566172696F0053636817
:105C5000616C74657220662E20482E007573652075
:105C600053772E20662E5365747000536368616B02
:105C70002E20486F6F6774652000616B7573742EFA
:105C800020566172696F20200061636F75737469BB
:105C90006320566172696F00416B6F6573742E20CB
:105CA000566172696F2000536F6C6C68F6686520EE
:105CB000202020202000536574706F696E742020AE
:105CC0002020202000476577656E73746520686F1B
:105CD0006F6774004D696E2E20476173202020206D
:105CE0002020006D696E2E207468726F74746C656C
:105CF00020004D696E696D61616C206761732020C1
:105D00000048F66865205020202020202020200018
:105D1000416C74697475646520502020202000480F
:105D20006F6F6774652050202020202020004C7564
:105D30006674647275636B20442020200042617297
:105D40006F6D657472696320442020004261726F38
:105D50006D6574722E2044202020005A2D4143434B
:105D600020202020202020202000414343205A20B2
:105D7000202020202020202000414343205A2020A2
:105D800020202020202020004D61782E2048F66819
:105D9000652020202020004D61782E20416C746900
:105DA0007475646520004D61782E20686F6F67748C
:105DB00065202020005665727374E4726B756E67FF
:105DC0002F5220006761696E2F7261746520202058
:105DD00020200056657273742E2F72617465202026
:105DE000200053636877656265676173202B2F2DF0
:105DF00000686F6F7665722076617269612E20008F
:105E0000686F6F7665722076617269612E20004737
:105E10005053205A202020202020202020004750AE
:105E200053205A202020202020202020004750539B
:105E3000205A202020202020202020005374696335
:105E40006B204E657574722E205000737469636BFD
:105E5000206E657574722E205000537469636B2038
:105E60006E657574722E2050004175746F20532F2B
:105E70004C204368616E2E004175746F20532F4C87
:105E8000204368616E2E004175746F20532F4C20A3
:105E90004368616E2E004C616E64652047657363D4
:105EA0006877692E006C616E64696E672073706537
:105EB000656420006C616E64696E6720737065654F
:105EC0006420004E69636B20532E20416E73742E44
:105ED00020006E69636B2073657276206374726C48
:105EE000006E69636B2073657276206374726C0058
:105EF0004E69636B204B6F6D70656E732E20006E64
:105F000069636B20636F6D70656E732E20006E6920
:105F1000636B20636F6D70656E732E2000436F6D31
:105F200070656E732E20206175732000436F6D7055
:105F3000656E732E20206F66662000436F6D70655E
:105F40006E732E20206F666620004E69636B2055AD
:105F50006D6B656872656E20006E69636B20696E9B
:105F6000762E206469722E006E69636B20696E76EE
:105F70002E726963682E004E69636B2053657276DA
:105F80006F2072656C006E69636B20736572766F4B
:105F90002072656C006E69636B20736572766F208A
:105FA00072656C004E69636B20536572766F206D6D
:105FB000696E006E69636B20736572766F206D6920
:105FC0006E006E69636B20736572766F206D696E0B
:105FD000004E69636B20536572766F206D617800A7
:105FE0006E69636B20736572766F206D6178006EE9
:105FF00069636B20736572766F206D6178004E69FE
:10600000636B20536572762046696C74004E696339
:106010006B20536572762046696C74004E69636B21
:1060200020536572762046696C7400526F6C6C2048
:10603000532E20416E73742E2000726F6C6C20738F
:10604000657276206374726C00726F6C6C2073657D
:106050007276206374726C00526F6C6C204B6F6DA3
:1060600070656E732E2000726F6C6C20636F6D70A4
:10607000656E732E2000726F6C6C20636F6D70659F
:106080006E732E2000526F6C6C20556D6B656872BC
:10609000656E2000726F6C6C20696E762E206469CC
:1060A000722E00726F6C6C206F6D6B6572656E2066
:1060B0002000526F6C6C20536572766F206D696E94
:1060C00000726F6C6C20736572766F206D696E0064
:1060D000726F6C6C20736572766F206D696E005202
:1060E0006F6C6C20536572766F206D617800726FF3
:1060F0006C6C20736572766F206D617800726F6CC6
:106100006C20736572766F206D617800526F6C6CD5
:1061100020536572762046696C7400526F6C6C2057
:10612000536572762046696C7400526F6C6C205314
:106130006572762046696C7400416E73742E204738
:1061400065736368772E2000736572766F207265C1
:1061500066726573682000536572766F207265669B
:106160007265736820004D616E75656C6C652047C3
:1061700065736368006D616E75656C6C2053706546
:1061800065642000536E656C682E68616E6462659C
:10619000642E0043616D205269636874756E6720D8
:1061A000200043616D204F7269656E7420202020AD
:1061B0000043616D6572612072696368742E20000E
:1061C000536572766F20332020202020202000533A
:1061D0006572766F20332020202020202000536518
:1061E00072766F20332020202020202000536572FB
:1061F000766F2034202020202020200053657276E6
:106200006F20342020202020202000536572766FDC
:1062100020342020202020202000536572766F201B
:10622000352020202020202000536572766F2035F5
:106230002020202020202000536572766F203520FA
:1062400020202020202000475053202020202020E4
:10625000202020202000656E61626C65204750532D
:106260002020202000656E61626C6520475053201D
:1062700020202000475053204D6F647573205374C5
:106280002E2000475053206D6F646520636F6E743D
:106290007200475053206D6F646520636F6E747297
:1062A00000475053205665727374E4726B2E2000C1
:1062B000475053204761696E20202020202000474E
:1062C000505320766572737465726B2E20004750B0
:1062D000532053742E20536368772E200047505369
:1062E00020737469636B2074687265004750532093
:1062F00073742E206472656D702E004D696E2E20B1
:106300005361742E2020202020004D696E2E2053D2
:1063100061742E2020202020004D696E2E205361B4
:10632000742E2020202020004750532D5020202064
:10633000202020202020004750532D5020202020B6
:106340002020202020004750532D502020202020A6
:1063500020202020004750532D492020202020209D
:10636000202020004750532D49202020202020208D
:106370002020004750532D4920202020202020207D
:1063800020004750532D4420202020202020202072
:10639000004750532D442020202020202020200082
:1063A0004750532D44202020202020202020005022
:1063B000204C696D697420202020202020004C6929
:1063C0006D6974202050202020202020004C696D11
:1063D00069657420205020202020200049204C692D
:1063E0006D697420202020202020004C696D697484
:1063F000202049202020202020004C696D696574F0
:1064000020204920202020200044204C696D697400
:1064100020202020202020004C696D697420204419
:10642000202020202020004C696D696574202044C4
:10643000202020202000475053204163632020204B
:10644000202020200047505320416363202020203B
:10645000202020004750532041636320202020202B
:106460002020004750532057696E646B6F72722E64
:1064700020004750532057696E6420436F72722E7C
:10648000004750532057696E6420436F72722E008C
:106490004272656D737769726B756E672020005369
:1064A0007065656420636F6D70656E732E00526554
:1064B0006D7765726B696E6720202020004750530E
:1064C000206D61782E205261642E200047505320A9
:1064D0006D61782E72616469757300475053206D49
:1064E00061782E7261646975730047505320576953
:1064F0006E6B656C204C692E0047505320616E67AF
:106500006C2E6C696D69740047505320686F656B21
:10651000206C696D2E20005048204C6F67696E20FA
:1065200074696D6520005048206C6F67696E207437
:10653000696D6520005048206C6F67696E20746932
:106540006A64200044796E616D69632050482020A0
:1065500020200044796E616D69632050482020201E
:10656000200044796E616D6973636865205048202E
:1065700000475053206D2E20526164206450480023
:10658000475053206D2E20526164206450480047CC
:106590005053206D2E2052616420645048004348BF
:1065A0002048F66865202020202020200043482035
:1065B000416C74697475646520202000434820484C
:1065C0006F6F6774652020202020004C45443120E7
:1065D0004269746D61736B6520004F7574312042A0
:1065E00069746D61736B20200055697467312042B6
:1065F0006974706174722E00202020202054696D0F
:10660000696E67202020004F7574312054696D69D0
:106610006E672020200055697467312054696D69C8
:106620006E672020002020202020736F666F727418
:1066300020616E0041637469762020202020202094
:106640002020004469726563742061616E202020FF
:10665000200020202020206E2E6D2E4D6F746F7232
:10666000004163742E2077692E204D6F746F720085
:10667000416B742E206D6F746F7220756974006D9C
:1066800069742057502D4576656E74202000636F25
:106690006D622E2057502D4576656E7400636F6DC8
:1066A000622E2057502D4576656E74004175746FCB
:1066B00054722E206D2F506F7469004175746F54A1
:1066C000722E206D2F706F7469004175746F547253
:1066D0002E206D2F706F7469004C45443220426942
:1066E000746D61736B6520004F757432204269745C
:1066F0006D61736B202000556974673220426974A4
:10670000706174722E00202020202054696D696E03
:1067100067202020004F7574322054696D696E67C0
:106720002020200055697467322054696D696E67B6
:106730002020002020202020736F666F727420615B
:106740006E004163746976202020202020202020C4
:10675000004469726563742061616E20202020000E
:1067600020202020206E2E6D2E4D6F746F72004100
:1067700063742E2077692E204D6F746F7200416B09
:10678000742E206D6F746F7220756974004F75746C
:106790003120566D696E2E5761726E004F757431DF
:1067A00020756E646572766F6C740055697467311C
:1067B000206F6E64657273702E004F7574322056B0
:1067C0006D696E2E5761726E004F75743220756E52
:1067D000646572766F6C74005569746732206F6EF1
:1067E00064657273702E004D696E2E2047617320B0
:1067F0002020202020006D696E2E207468726F7436
:10680000746C6520004D696E696D61616C20676113
:10681000732020004D61782E2047617320202020B6
:106820002020006D61782E207468726F74746C651E
:1068300020004D6178696D61616C20676173202073
:10684000004B6F6D706173737769726B756E670063
:10685000636F6D7061737320656666656374004B6A
:106860006F6D7061732065666665637420004361B7
:106870007265667265652053742E20200043617234
:106880006566726565204374726C200043617265B1
:1068900066726565204374726C200054656163689C
:1068A00061626C6520436172650054656163686173
:1068B000626C652043617265005465616368616262
:1068C0006C65204361726500556E7465727370610A
:1068D0006E6E756E672000756E646572766F6C748F
:1068E0006167652020004F6E6465727370616E6E23
:1068F000696E672000566F6C74205265666572651C
:106900006E7A2000566F6C74205265666572656EF3
:106910007A20005265662E207370616E6E696E6714
:1069200020004E6F7420476173205A6569742020DF
:1069300000456D6572672E5468722E54696D65004E
:106940004E6F6F64206761732074696A6420004E23
:106950006F74204761732020202020202000456D87
:106960006572672E5468726F74746C65004E6F6F39
:106970006420676173202020202020004661696C1C
:10698000732E2043482054696D65004661696C731D
:106990002E2043482054696D65004661696C732E52
:1069A0002043482054696A64004661696C732E2054
:1069B0004368616E6E656C004661696C732E20439E
:1069C00068616E6E656C004661696C732E20436869
:1069D000616E6E656C006B2E53756D6D6572206F08
:1069E0002053656E006E20626565702061637420BF
:1069F000545820004765656E2062656570207A20D6
:106A0000545800566172696F206661696C20416C50
:106A10007400566172696F206661696C20416C7404
:106A200000566172696F206661696C20416C740068
:106A3000436F6D70617373204572726F72200043F3
:106A40006F6D70617373204572726F7220004B6FAF
:106A50006D706173204572726F722020006B2E532F
:106A600074617274206F2E53442D4B006E2073742A
:106A70002E207774686F2053442000472E73746172
:106A80007274207A2E20534420006B2E537461724E
:106A900074206F2E47505320006E2073742E207781
:106AA00074686F2047505300472E737461727420CE
:106AB0007A2E20475053004779726F2050202020B3
:106AC0002020202020004779726F20502020202095
:106AD00020202020004779726F2050202020202085
:106AE000202020004779726F20492020202020207C
:106AF0002020004779726F2049202020202020206C
:106B000020004779726F204920202020202020205B
:106B1000004779726F204420202020202020200070
:106B20004779726F20442020202020202020004719
:106B300079726F20442020202020202020004769E7
:106B4000657220502020202020202020004C6163EE
:106B50006574205020202020202020004769657285
:106B6000205020202020202020200047696572200E
:106B7000492020202020202020004C6163657420C3
:106B800049202020202020200047696572204920CC
:106B9000202020202020200044796E616D697363DD
:106BA00068652053742E0064796E616D696320738B
:106BB000746162692E0044796E616D69732E207371
:106BC0007461622E0044726568726174656E6265FC
:106BD000672E2000526F7452617465206C696D6974
:106BE000742E00546F6572656E74616C206C696DF3
:106BF0002E004143432F4779726F2046616B2E2050
:106C0000004143432F4779726F204661637420002F
:106C10004143432F4779726F2046616374200041DE
:106C200043432F4779726F204B6F6D702E00436F77
:106C30006D70204143432F4779726F2000436F6D81
:106C400070204143432F4779726F2000486175706F
:106C5000747265676C6572204920004D61696E2011
:106C600049202020202020202000486F6F66647279
:106C70006567656C2E20492000447269666B6F6DF4
:106C800070656E7361742E00647269667420436F60
:106C90006D70656E732E00447269667420636F6D4B
:106CA00070656E732E004779726F20737461622E67
:106CB00020202020004779726F2073746162696C14
:106CC000697479004779726F2073746162696C69C5
:106CD000742E004D6F746F7220736D6F6F74682027
:106CE00020004D6F746F7220736D6F6F7468202079
:106CF000004D6F746F7220736D6F6F746820200089
:106D0000506172616D6574657220312020200050E1
:106D10006172616D657465722031202020005061C0
:106D200072616D657465722031202020005061729F
:106D3000616D65746572203220202000506172619F
:106D40006D65746572203220202000506172616D83
:106D500065746572203220202000506172616D657B
:106D6000746572203320202000506172616D65745B
:106D70006572203320202000506172616D6574655A
:106D800072203320202000506172616D657465723D
:106D9000203420202000506172616D65746572207E
:106DA0003420202000506172616D6574657220345A
:106DB00020202000506172616D657465722035205D
:106DC000202000506172616D65746572203520204D
:106DD0002000506172616D6574657220352020203D
:106DE00000506172616D657465722036202020004C
:106DF000506172616D6574657220362020200050EC
:106E00006172616D657465722036202020005061CA
:106E100072616D65746572203720202000506172A8
:106E2000616D6574657220372020200050617261A9
:106E30006D65746572203720202000506172616D8D
:106E400065746572203820202000506172616D6584
:106E5000746572203820202000506172616D657465
:106E600065722038202020004163687328652E2930
:106E70006B6F70706C2E0028446529436F75706CC1
:106E80002041786573004173206B6F7070656C6989
:106E90006E672020004769657220706F732E204B4B
:106EA0006F707000526574726F6163206C6163650E
:106EB0007420004769657220706F732E206B6F70AD
:106EC0002E004E69636B2F526F6C6C204B6F70708D
:106ED00000526574726F20726F756C2F74616E0052
:106EE0004E69636B2F526F6C6C206B6F702E004776
:106EF000696572204B6F7272656B74757200436FB7
:106F00007272656374206C61636574200047696503
:106F10007220636F72726563746965004F72696590
:106F20006E74696572756E672020004F7269656EB8
:106F300074696572756E672020004F7269656E74A2
:106F400061746965202020200048F668656E7265CE
:106F500067656C756E672000416C74697475646553
:106F6000204374726C2000486F6F67746520436F14
:106F70006E74722E2000536F6C6C68F6686520206A
:106F80002020202000536574706F696E74202020CB
:106F900020202000476577656E73742E686F6F67D9
:106FA000746500537469636B204E657574722E208E
:106FB0005000737469636B206E657574722E205077
:106FC00000537469636B206E657574722E205000D7
:106FD0004750532020202020202020202020006502
:106FE0006E61626C65204750532020202000456E62
:106FF00061626C6520475053202020200047505389
:10700000204D6F6475732053742E20004750532019
:107010006D6F646520636F6E747200475053206D0E
:107020006F646520636F6E74720044796E616D6980
:1070300063205048202020200044796E616D6963F0
:10704000205048202020200044796E616D69632023
:107050005048202020200043482048F66865202022
:1070600020202020200043482048696768202020F5
:107070002020202000434820686F6F67746520201F
:107080002020200043617265667265652053742E6E
:107090002020004361726566726565204374726CDE
:1070A00020004361726566726565204374726C20CE
:1070B00000546561636861626C65204361726500BC
:1070C000546561636861626C652043617265005458
:1070D0006561636861626C652043617265004D6F34
:1070E000746F7220536963682E536368004D6F7428
:1070F0002E5361666574792053772E004D6F742E80
:107100007361662E736368616B2E004F7269656EE2
:1071100074696572756E672020004F7269656E74C0
:107120006174696F6E202020004F7269656E746112
:1071300074696520202020004B616EE46C6520207E
:10714000202020202020004368616E6E656C202086
:107150002020202020004B616E61616C20202020C7
:1071600020202020004B6F6E66696775726174691C
:107170006F6E20006D61696E20202020202020206D
:10718000202000436F6E66696775726174696520BF
:107190002000537469636B202020202020202020B1
:1071A00000737469636B20202020202020202000A1
:1071B000537469636B202020202020202020004C65
:1071C0006F6F70696E6720202020202020004C6F98
:1071D0006F70696E6720202020202020004C6F6F88
:1071E00070696E67202020202020200048F6686506
:1071F0002020202020202020202000416C74697451
:1072000075646520202020202000486F6F6774651A
:107210002020202020202020004B616D65726120FD
:10722000202020202020200043616D6572612020F5
:107230002020202020200043616D657261202020E5
:107240002020202020004E6176694374726C20203B
:1072500020202020004E6176694374726C2020202B
:10726000202020004E6176694374726C202020201B
:1072700020200041757367E46E6765202020202080
:1072800020004F75747075747320202020202020FA
:107290000055697467616E67656E202020202000AC
:1072A000566572736368696564656E657320004432
:1072B00069766572732020202020202020004469F8
:1072C00076657273656E2020202020200047797239
:1072D0006F20202020202020202020004779726F5E
:1072E00020202020202020202020004779726F209D
:1072F0002020202020202020200042656E75747AF6
:1073000065722020202020200055736572202020E7
:1073100020202020202020004765627275696B655F
:1073200072202020202000416368736B6F70706CA6
:10733000756E67202000436F75706C20417865730F
:1073400020202020004B6F7070656C696E672041B3
:10735000737320004D697865722D536574757020C4
:10736000202000436F6E666967204D6978202020D9
:107370002000436F6E6669672E204D697865722024
:1073800000456173792053657475702020202000BA
:10739000436F6E6669672045617379202020004342
:1073A0006F6E6669672E20656173792020005769CA
:1073B000726B6C696368204B6F70696572656E3FB4
:1073C000004B6F706965727420756E6420416B7438
:1073D00069766965727400282020202D20202029DC
:1073E0002028643A20202029005374642E0028307D
:1073F0002D3234372D50382928643A506F20290017
:107400005374642E00506F202900506F002A002A08
:10741000001D00200020001D00312D5331322F5758
:107420002F3C2F7C2F3E2028643A202029005374C3
:10743000642E004368616E6E656C2020202000532E
:107440006572436820202020005750204576656EE5
:10745000742020004D696E696D756D2020004D69A6
:1074600064646C65202020004D6178696D756D2025
:1074700020004F66662020202020202000446973D1
:107480002C312D5331322F572F4F2028643A202092
:1074900029005374642E0044697361626C65642032
:1074A00020004368616E6E656C20202020005365CB
:1074B00072436820202020005750204576656E7466
:1074C0002020004F666620202020202020004F6EC4
:1074D000202020202020202000442C312D53313228
:1074E0002F572F462F432F5028643A2029005374DA
:1074F000642E0044697361626C65642020004368F7
:10750000616E6E656C2020202000536572436820F8
:10751000202020005750204576656E7420200046BC
:107520007265652020202020202000434820202054
:107530002020202020005048202020202020202013
:1075400000201920202020301149202020456E6481
:10755000652020204F4B0031003000120020001227
:1075600000130012002500200020500020204A00B7
:1075700020204E00430053004F66660044697300AC
:10758000575045004D696E004D6964004D617800AB
:107590004F666600204F6E004672656500204348C6
:1075A000002050480050504D005370650053704803
:1075B0000053704C004A65740041435400486F54B6
:1075C000005342550055535200130012001300009F
:1075D00014BE88E10FB6F8948093600010926000AA
:1075E0000FBE11241FBECFEFD0E4DEBFCDBF13E02E
:1075F000A0E0B1E0E2E9FAEE01E00BBF02C00790C3
:107600000D92A834B107D9F716E2A8E4B3E001C09F
:107610001D92AC33B107E1F70E9477DB0C9447F57C
:107620000C940000A0E1B0E0E8E1FBE30C94F0F082
:107630002B013C0169014A3029F5EE24E394F12C39
:10764000EC0EFD1E6AE0862E912CA12CB12C1701A8
:10765000C301B201A50194010E94B3F0842D805DA5
:107660009AE0299F80191124F70181937F01CF01AE
:107670008219930929013A014114510461047104EA
:1076800039F730C0FE01319620E030E001C09C01A6
:10769000D301C2018F709927AA27BB27482F0A97C9
:1076A000A105B10510F480E301C081E4840F81934A
:1076B000C901019644E076946794579447944A959B
:1076C000D1F7411451046104710409F7FE01E80F78
:1076D000F91F48E74183FE01E20FF31F80E3838334
:1076E000C90103960197F60120E030E0015011092D
:1076F000A1E0B0E0AC0FBD1FA80FB91F4C914193A2
:107700002F5F3F4F1816190624F4019720173107F1
:107710007CF3F601E20FF31F1082C9016096E2E1EB
:107720000C940CF10F931F9350E000E010E09801CF
:1077300039C0642F60536A3060F4F4E0000F111F09
:10774000221F331FFA95D1F700531109210931097E
:107750001FC0642F6156663060F4E4E0000F111F13
:10776000221F331FEA95D1F7075511092109310965
:107770000FC0642F6154663080F474E0000F111F55
:10778000221F331F7A95D1F70753110921093109B7
:10779000040F111D211D311D05C0483741F4511141
:1077A00006C051E0FC014191CF014111C2CFB801A7
:1077B000C9011F910F910895CF93FC0120E030E0A3
:1077C000A90112C08C2F80538A3088F4AAE0B0E05F
:1077D0000E9467F09B01AC01205331094109510916
:1077E0002C0F311D411D511DC191C111EBCFB901AC
:1077F000CA01CF9108950C94C05708950C94A457D2
:1078000008950C94CB57089520918D0A30918E0ADB
:107810004091980A5091990A241735076CF4E09129
:107820008B0AF0918C0AE20FF31F80832F5F3F4F8A
:1078300030938E0A20938D0A0E94A45781E0089508
:10784000CF93DF93EC0170932F1460932E1409C033
:107850000E94D857892B29F00E947257888381E0B3
:1078600007C080912E1490912F14892B89F780E006
:10787000DF91CF910895A1E0B0E0E1E4FCE30C9446
:10788000FEF08C01B801CE010196DADF8111FACF4A
:107890002196E4E00C941AF1A1E0B0E0E2E5FCE30B
:1078A0000C94F6F07C016B01FC019490911012C0D5
:1078B00081E01CC08981891103C00F5F1F4F05C083
:1078C000881102C0850101C08701F80194909110D0
:1078D00007C0EECF8C01892C5C01FFEFAF1ABF0A05
:1078E000B601CE010196ACDF8111E4CF2196ECE028
:1078F0000C9412F1A1E0B0E0E0E8FCE30C94F5F0A8
:107900007C015A0100E010E04B0182E0881A9108E6
:107910006B0181E0C81AD10837C079808DE07812F8
:1079200026C0B501CE0101968BDF89818A3041F4F2
:10793000E114F104C1F1F701E00FF11F108233C02F
:10794000E114F104A1F00815190544F4F701E00F62
:10795000F11F708281830E5F1F4F09C00C151D053A
:1079600034F4F701E00FF11F70820F5F1F4F0C1509
:107970001D0554F4E114F10439F0F701E00FF11F93
:10798000898180830F5F1F4FB501CE01019658DFBB
:107990008111C3CFE114F10421F0F701E00FF11FD1
:1079A000108200E010E0C8012196EDE00C9411F186
:1079B000A1E0B0E0EEEDFCE30C94FCF043C0898163
:1079C0008C3309F03FC08093480309E413E0EE24B0
:1079D000E39401C0EF2C64EF71E0CE01019630DF3B
:1079E000811102C080E036C08981F80181938F0146
:1079F000FE2CF3948E3311F564EF71E0CE01019605
:107A00001FDF882379F38981803261F7AF2DB0E0E1
:107A1000A85BBC4F8C93E394E394EE2DF0E0E85B1D
:107A2000FC4F108281E08093580344EF51E060E006
:107A300070E080E090E05EDF81E00CC0FCE0FF12CF
:107A4000C9CFD0CF64EF71E0CE010196F9DE81118C
:107A5000B6CFC8CF2196E6E00C9418F120915803D8
:107A6000211101C0A5CFBC0188E493E015CF1F937D
:107A7000CF93DF938091890A811160C084EC99E0F3
:107A800024EF31E0F9013197F1F70197D9F78FE948
:107A900092E00E94CB5784EC99E024EF31E0F901A9
:107AA0003197F1F70197D9F762E370E083EA92E04A
:107AB000F3DE8823A1F080915803811130C08DE05E
:107AC0000E94A45782E390E0C9DF811128C08DE0B5
:107AD0000E94A45782E390E0C1DF811120C08DE0B5
:107AE0000E94A45782E390E0B9DF8823F9F017C021
:107AF000FE013197F1F70197D9F789EA92E00E94E8
:107B0000CB5784EC99E0FE013197F1F70197D9F753
:107B100062E370E08DEA92E0BFDE882321F081E02D
:107B20008093890A0CC0115039F003C012E0C4EFF1
:107B3000D1E084EC99E0DCCF80E001C081E0DF910E
:107B4000CF911F9108958091890A882359F08091DF
:107B5000900A9091910A01969093910A8093900ACD
:107B600081E0089584DF8111F2CF08958091890A20
:107B7000882369F088E593E00E94CB5764EF71E0B9
:107B80008EE593E089DE882321F01092890A81E056
:107B9000089580E008958091900A9091910A01974C
:107BA0009093910A8093900A892B09F4DFCF81E0AA
:107BB0000895CF93C8DF882399F084E393E00E946F
:107BC000CB5764EF71E08AE393E066DE882329F007
:107BD00084EF91E043DFC1E001C0C0E0DCDF01C021
:107BE000C0E08C2FCF91089568E473E00E9432F4D6
:107BF00021E0892B09F420E0822F0895A1E0B0E074
:107C0000E4E0FEE30C94F7F0B82EC92ED62E7A01EC
:107C10000DB71EB78DB79EB7E3E06E9F801991092F
:107C200011249EBF8DBF2DB73EB72F5F3F4F922EC1
:107C3000A32EAB2DBC2DF90120E007C010828D9141
:107C40009D91928381832F5F33962D11F7CFB701DA
:107C5000CE010196F5DD81112AC08FEF2FC011965C
:107C6000ED91FC9112974491941301C00DC0F9015C
:107C700060817181FB014491941729F012967C93E5
:107C80006E93119706C0FB0131961296FC93EE930A
:107C900011971196ED91FC911297E49113962E5F36
:107CA0003F4FEE2359F08F5F8D1589F2D8CF998120
:107CB0002B2D3C2DA92DBA2D80E0F6CF1EBF0DBF78
:107CC0002196EBE00C9413F1A8E2B0E0EAE6FEE3C3
:107CD0000C9400F1CE01C096282F892F6FA5653135
:107CE00008F064E1E22FF82FDE01119680E090E0C9
:107CF000262F30E005C0419151914D935D9301963F
:107D000082179307C4F34DA55EA5CE01019676DFD9
:107D1000282F332727FD3095932FA896E2E00C9467
:107D20001CF1A4E0B0E0E7E9FEE30C94FCF08C0168
:107D30007B0182E493E09A83898388E493E09C83C7
:107D40008B8344EF51E062E0CE01019657DF813032
:107D500081F0811106C044EF51E0B701C801CADDCE
:107D600006C0A7016EE473E0C8010E94C7F380E07B
:107D700001C081E02496E6E00C9418F1A0E1B0E0A7
:107D8000E4ECFEE30C94F9F06C017B018A01B22E65
:107D9000DADE882309F442C0C6010E94CB570115E0
:107DA0001105B1F080E20E94A457B11006C00CC0CA
:107DB000803211F48091960A27DDF8010F5F1F4F82
:107DC00084918111F5CF1BC0C8010E94CB5717C009
:107DD000E114F104A1F080E20E94A457B11006C0A2
:107DE0000BC0803211F48091960A0EDDF70181916B
:107DF0007F018111F6CF03C0C7010E94C0578DE0FB
:107E00000E94A45760E170E0CE0101968ADF182F2E
:107E100080E090E023DEBFDE812F01C080E060962D
:107E2000E9E00C9415F1ABE0B0E0E9E1FFE30C947C
:107E3000FCF07C01CB01BA01422F0BE010E09E0167
:107E40002F5F3F4FEFDB20E040E050E0BE016F5F6F
:107E50007F4FC70193DF2B96E6E00C9418F1ABE05F
:107E6000B0E0E5E3FFE30C94FCF07C01CB01BA0148
:107E7000422F0BE010E09E012F5F3F4FD3DB20E04D
:107E800040E050E0BE016F5F7F4FC70177DF91E0B8
:107E9000811101C090E0892F2B96E6E00C9418F137
:107EA000A2E0B0E0E6E5FFE30C9400F1805D898399
:107EB0001A8220E040E050E0BE016F5F7F4F85E610
:107EC00093E05CDF91E0811101C090E0892F229660
:107ED000E2E00C941CF1E0CC0895EF92FF920F9336
:107EE0001F93CF93DF938C01EB017A012CDE882363
:107EF000F1F0000F111F000F111F0A5A1E4FF80159
:107F0000808191810E94CB5764EF71E0F8018281FA
:107F10009381C2DC882351F044EF51E0B701CE01D8
:107F2000E9DC80E090E09ADD36DE03C034DEC4ECAC
:107F3000D2E0CE01CDB7DEB7E6E00C9418F180E0D8
:107F4000AFCF81E0ADCF21E040E050E0BC0181E760
:107F500093E014DF91E0811101C090E0892F089532
:107F60008A3008F49DCF80E008958E3008F08DE0CF
:107F7000482F50E060E070E02AE08FE793E053DFA5
:107F800091E0811101C090E0892F089521E040E047
:107F900050E060E070E08AEA93E0F0DE91E0811169
:107FA00001C090E0892F0895CF9321E040E050E098
:107FB000BC018AE993E0E2DEC82FE8DF81E0C1116D
:107FC00001C080E0CF910895CF93FC012181283733
:107FD00011F0283509F4029620E040E050E0BC01A1
:107FE0008DE893E0CBDEC82FD1DF81E0C11101C065
:107FF00080E0CF910895AB01BC018CE190E06DCFA2
:10800000482F50E060E070E02AE08AEB93E027CF51
:1080100020E040E050E0BC0188EC93E0AFDE91E06E
:10802000811101C090E0892F08958DDD8823F1F042
:1080300087ED93E00E94CB5764EF71E08FED93E002
:108040002BDC811102C0A7DD11C080E593EC24EF89
:1080500031E0F9013197F1F70197D9F71092890AC8
:108060001092910A1092900A81E0089580E008959C
:1080700020E040E050E0BC0188EE93E07FDE91E03C
:10808000811101C090E0892F089520E040E050E088
:10809000BC0184EF93E072DE91E0811101C090E0B9
:1080A000892F08951F93CF93DF93EC01162F109221
:1080B000870A49DD811103C081E08093870A80919E
:1080C000870A811106C0ECDE811103C082E0809333
:1080D000870A8091870A811108C08FE49CE198DFAC
:1080E000811103C083E08093870A8091870A811100
:1080F00008C08FE59CE1C9DF811103C084E0809353
:10810000870A8091870A811107C084E079DF811195
:1081100003C085E08093870A8091870A811107C098
:10812000CE0111DF811103C086E08093870A809120
:10813000870A811107C0812F18DF811103C087E0F2
:108140008093870A36DD811103C088E08093870A17
:1081500022DD811103C089E08093870A66DF809168
:10816000870ADF91CF911F91089520E040E050E011
:10817000BC0183E094E002DE91E0811101C090E057
:10818000892F0895A0E1B0E0E8ECF0E40C9400F150
:108190008330B9F020F4813071F080F406C085306E
:1081A000B1F090F08630C9F403C062E174E011C010
:1081B00067E174E00EC06CE174E00BC061E274E052
:1081C00008C067E274E005C06DE274E002C063E3DA
:1081D00074E0CE0101960E94C0F3B5DC20E040E0DF
:1081E00050E0BE016F5F7F4F8AE394E0C7DD8823D4
:1081F00049F020E040E050E0BE016F5F7F4F88E42F
:1082000094E0BCDD8091E61B0E944F5781E06096B0
:10821000E2E00C941CF10E9458B520E049E554E0DE
:1082200061E080E00E9414B98091E61B8093940A7B
:108230001EDC882349F067C0F9013197F1F70197F7
:10824000D9F780E08170089581E00E944F5720E0C7
:1082500046E654E062E080E00E9414B908DC811137
:1082600052C085E00E944F5720E047E754E062E0AB
:1082700080E00E9414B9FBDB811145C083E00E94BD
:108280004F5720E04AE854E062E080E00E9414B9D1
:10829000EEDB811138C082E00E944F5720E04CE9AC
:1082A00054E062E080E00E9414B9E1DB81112BC050
:1082B00086E00E944F5720E04EEA54E062E080E002
:1082C0000E9414B9D4DB81111EC00E944F5720E0D8
:1082D0004FEB54E062E080E00E9414B9C8DB8111EA
:1082E00012C020E040ED54E062E00E9414B920E0AA
:1082F00040EE54E063E080E00E9414B980E197E230
:1083000024EF31E099CF81E09DCFCF931092890A7D
:108310001092910A1092900A10928F0A10920A0BF2
:1083200081E08093970A8093920A1092950A1092A6
:108330008C0A10928B0A10928E0A10928D0A10925B
:10834000990A1092980A1092860A1092850A109241
:108350009A0A83E00E94DBD080E49CE924EF31E0BC
:10836000F9013197F1F70197D9F755DF811108C06D
:1083700020E043EB52E062E00E9414B9C0E077C015
:108380008091E61BFFDE81110CC020E043EC52E03F
:1083900062E00E9414B98091E61B0E944F57C0E032
:1083A00001C0C1E08091E61B0E944F57CC2309F425
:1083B0004DC020E040E050E060E070E085ED92E0EC
:1083C000DDDC811108C020E04FED52E063E00E9447
:1083D00014B9C0E001C0C1E020E040E050E060E03E
:1083E00070E08FEE92E0CADC811107C020E041E02E
:1083F00053E065E00E9414B9C0E060E570E08AEBEC
:108400009AE0F9DDAC0120E066E080E00E9440B92E
:1084100080914C1C81111AC020E040E153E064E0DF
:108420000E9414B960914E1C80E39CE13BDE8823DE
:1084300069F020E043E253E064E080E00E9414B978
:1084400060E08091870A0E9499BDC0E081E00E94AF
:10845000DBD0C1110BC020E43CE944EF51E0FA014C
:108460003197F1F721503109D1F701C0C1E08C2FCC
:10847000CF910895EF92FF920F931F935DD783EFF3
:1084800094E088D741E2E42E45E0F42E00E115E0C7
:108490002FEF34E040E050E061E081E00E94654B66
:1084A00080912F1C8823B1F183E3E82E85E0F82E1C
:1084B0008701970140E050E061E082E00E94654B57
:1084C00096E4E92E95E0F92E0EE315E028E335E079
:1084D00040E050E061E087E00E94654B29E6E22E33
:1084E00025E0F22E0EE515E02FE435E040E050E007
:1084F00061E084E00E94654B36E9E32E35E0F32E1F
:1085000006E815E027E735E04EE354ED61E085E04D
:108510000E94654B1F910F91FF90EF900895ABE083
:10852000B0E0E5E9F2E40C94FAF0A4DF54EFC52ED4
:10853000DD24D39480E00E943E4ED7D7853009F4E5
:1085400095C0E6D7182F109237088130F9F4F090D3
:108550002F1CEE24E39407E02BED41E050E060E0B7
:1085600070E08F2D90E00E94957E80932F1CF8166E
:1085700009F3882341F0C9DE882319F01093461CC3
:1085800002C01092461CF9D675DFD4CF823011F5A7
:108590004BE050E060E37CE1CE0101960E94C955BA
:1085A00025EA35E043E06AE0CE0101960E941A8296
:1085B00080913708813009F0BDCF85E694E10E94B3
:1085C000E1554BE050E065E674E180E39CE10E94F8
:1085D00023F4B0CF873081F4EE24E39400E02EED55
:1085E0004DE050E061E070E080914E1C90E00E9410
:1085F000957E80934E1C9ECF843009F09BCF0E94C5
:1086000058B58091E61B8093940A0E944F5720E052
:108610004BEB55E063E080E00E9414B976DE20E089
:10862000813049F446EC55E063E080E00E9414B9E3
:108630000E945DC40FC043ED55E063E080E00E94FE
:1086400014B91092461C40E060E470E088EE93E0BC
:108650000E94DD7288EA91E6F6013197F1F7019701
:10866000D9F78091940A0E944F5764CF86D62B96F3
:10867000E8E00C9416F1CF93C82F20E047E057E0D4
:1086800063E080E00E9497B960E08C2F0E9499BD62
:10869000C0935B0340E060E470E084EF91E00E94EF
:1086A000DD7288E893E124EF31E0F9013197F1F7C9
:1086B0000197D9F7CF9108951F93CF93DF93D82FC8
:1086C000C62F8FEF67FD0AC00E94AE5982E00E945C
:1086D000AE598D2F0E94AE598C2F0DC00E94AE59FD
:1086E00083E00E94AE598D2F0E94AE598EEF0E94FA
:1086F000AE598C2F80580E94AE591AE0C4EFD1E0D9
:108700000E94FF5890E028EE33E0FE013197F1F728
:1087100021503109D1F7009719F4115089F702C09F
:108720000697D1F020E049E157E062E080E00E9446
:1087300097B940E060E470E088EE93E00E94DD725B
:1087400080E29EE424EF31E0F9013197F1F70197DF
:10875000D9F72FEF30E002C020E030E0C901DF910F
:10876000CF911F9108951F93CF93DF93C82F0E943D
:10877000FF588FEF0E94AE5982E00E94AE598EEFF3
:108780000E94AE598C2F0E94AE5984EF91E024EFE5
:1087900031E0F9013197F1F70197D9F710E0C4EF13
:1087A000D1E00E94FF58682F70E048EE53E0FE01D0
:1087B0003197F1F741505109D1F71F5F61157105EC
:1087C00019F41A3071F708C01A3031F066307105AB
:1087D00031F4282F30E005C020E030E002C02FEF58
:1087E00030E0C901DF91CF911F910895A1E0B0E081
:1087F000ECEFF3E40C94FEF0182F0E947B5920E07C
:1088000043EE55E061E080E00E9497B91230A1F09C
:1088100028F4112349F0113011F50AC01430A1F0E9
:1088200078F01530E1F414C020E045EF55E013C0B6
:1088300020E04CEF55E00FC020E043E056E00BC0D5
:1088400020E04AE056E007C020E041E156E003C0E6
:1088500020E048E156E061E086E00E9497B988E7B1
:1088600090E081DF082F20E0482F62E080E09983CC
:108870000E9472BD202F9981392FA90141505109C1
:108880004E3F510528F482E080935C0310935A0315
:10889000C9012196E4E00C941AF1CF93DF93C82F1D
:1088A0000E94515B5E9820ED37E044EF51E0FA0101
:1088B0003197F1F721503109D1F70E9458B58C2F2B
:1088C0000E947B5920E04FE156E060E080E00E948A
:1088D00097B98C2F8BDFEC01009721F081E080931A
:1088E0005C03D6C080E082DFEC01009709F0D0C0C5
:1088F00081E07CDFEC01009709F0CAC082E076DFFE
:10890000EC01009709F0C4C083E070DFEC01009730
:1089100009F0BEC084E06ADFEC01009709F0B8C03E
:1089200085E064DFEC01009709F0B2C0A1C0F90155
:108930003197F1F70197D9F7C0E0D0E01AC00E9453
:1089400058B520E043E456E060E080E00E9497B92B
:1089500040E060E470E088EE93E00E94DD7280E227
:108960009EE424EF31E0F9013197F1F70197D9F74F
:10897000E3CFCE0101978E3F910508F077C00E94AA
:1089800058B580915A030E947B5980915C038130D5
:1089900039F420E048E556E060E080E00E9497B9B5
:1089A00080915C03823009F04FC01092831B20E05D
:1089B00046E656E060E080E00E9497B96091E61BD1
:1089C00083E07ADE892B39F46091E61B8EE474DE55
:1089D000892BC9F021C020E04CE756E061E080E03F
:1089E0000E9497B940E060E470E088EE93E00E9456
:1089F000DD7280E29EE424EF31E0F9013197F1F776
:108A00000197D9F7E1CF8091E61B0E947B598091B5
:108A1000E61B8093940A18C020E04DE856E063E01E
:108A200080E00E9497B940E060E470E088EE93E057
:108A30000E94DD7280E29EE424EF31E0F90131977B
:108A4000F1F70197D9F7DFCF45E161E080E00E94BF
:108A50009EB920E040EA56E061E080E00E9497B9CC
:108A600020E04C2F61E089E00E9472BD5E9A15C043
:108A70000E9458B520E043E356E060E080E00E94A9
:108A800097B910925C0380E29EE424EF31E04FCF6F
:108A9000CF3FD10509F06DCF52CFDF91CF9108952F
:108AA0000F931F93CF93DF93C82F85E00E9442D28C
:108AB0008091940AF2DE80915C03882309F491C1CD
:108AC00020E049EA56E062E080E00E9497B95E98B3
:108AD00020ED37E084EF91E0FC013197F1F7215070
:108AE0003109D1F70E94515B6EE781E5E5DD892B05
:108AF00049F020E04DEB56E064E080E00E9497B939
:108B0000D1E001C0D0E06091751B80E0D5DD892BFC
:108B100011F081E0B0DD0D2F0F5F20E04FEB56E04C
:108B200064E08D2F0E9497B96091751B8BE4C4DDC2
:108B3000892B11F082E09FDD1D2F1E5F20E041ECAC
:108B400056E064E0802F0E9497B96091751B81E028
:108B5000B3DD892B11F083E08EDD0D2F0D5F20E05A
:108B600043EC56E064E0812F0E9497B96091751B39
:108B70008CE4A2DD892B11F084E07DDD1D2F1C5FCC
:108B800020E045EC56E064E0802F0E9497B960E059
:108B90008DE092DD892B11F085E06DDD0D2F0B5FEF
:108BA00020E047EC56E064E0812F0E9497B963E033
:108BB00082E082DD892B11F086E05DDD1D2F1A5FDA
:108BC00020E049EC56E064E0802F0E9497B9609164
:108BD000781B85E071DD892B11F087E04CDD0D2FCE
:108BE000095F20E04BEC56E064E0812F0E9497B9CA
:108BF0006091781B80E560DD892B11F088E03BDD1A
:108C00001D2F185F20E04DEC56E064E0802F0E949D
:108C100097B96091791B89E04FDD892B11F089E0CC
:108C20002ADD0D2F075F20E04FEC56E064E0812F36
:108C30000E9497B96091791B84E53EDD892B11F084
:108C40008AE019DD1D2F165F20E041ED56E064E05B
:108C5000802F0E9497B96091771B84E02DDD892BCE
:108C600011F08BE008DD0D2F055F20E043ED56E0AD
:108C700064E0812F0E9497B96091771B8FE41CDD1F
:108C8000892B11F08CE0F7DC1D2F145F20E045EDFF
:108C900056E064E0802F0E9497B961E088E00CDD27
:108CA000892B11F08DE0E7DC0D2F035F20E047ED0D
:108CB00056E064E0812F0E9497B961E08BE0FCDC14
:108CC000892B11F08EE0D7DC1D2F125F20E049EDDB
:108CD00056E064E0802F0E9497B96091761B86E091
:108CE000EBDC892B11F08FE0C6DC0D2F015F20E05B
:108CF0004BED56E064E0812F0E9497B96091761B9E
:108D000081E5DADC892B11F08FE0B5DC1D2F105FD7
:108D100020E04DED56E064E0802F0E9497B96C2F63
:108D200083E0CADC892B11F080E1A5DCDF5E20E066
:108D30004FED56E064E0812F0E9497B920ED37E0B7
:108D400044EF51E0FA013197F1F721503109D1F7A1
:108D50006C2F8EE4B1DC892B11F081E18CDC20E0FA
:108D600041EE56E064E08D2F0E9497B95E9A8091A3
:108D70005B0320E08823E9F043EE56E062E080E008
:108D80000E9497B960E080915B030E9499BD40E02A
:108D900060E470E088EE93E00E94DD7220E23EE441
:108DA00044EF51E0FA013197F1F721503109D1F741
:108DB0000CC045EF56E062E080E00E9497B90E9447
:108DC00055C460E08C2F0E9499BD8C2F0E947B5966
:108DD00080E29EE424EF31E0F9013197F1F7019749
:108DE000D9F7DF91CF911F910F910895CF93DF9322
:108DF00010926203109261031092600310925E035E
:108E000010925F0310925D03E091110BF091120B31
:108E100011AA10AAAFE7BCE1E4E9FCE189E691E020
:108E20002FEFEF012997188214961D921D921D9223
:108E30001C9217971D921D921D921C9213971896C3
:108E40001D921D921D921C921B971E969C938E93B1
:108E50001D97EF0126971882EF0125971882EF01E1
:108E600022972883EF012497188210825E967E96BF
:108E700030E2A132B307A9F681E0DF91CF910895E6
:108E8000B5CF089580915F030895882379F090917C
:108E90005F03981758F090E001974EE1489F9001CA
:108EA000499F300D11242158334E02C020E030E09C
:108EB000C9010895CF93DF93EC018A89982F9150CF
:108EC0009F3108F06DC090E001972EE1289FF001DE
:108ED000299FF00D1124EE56F34E2081213091F19F
:108EE000D8F02F3F09F046C02B89222321F02130F2
:108EF00009F040C006C0209160032F5F20936003FB
:108F000005C020915E032F5F20935E0320915F03D5
:108F10002F5F20935F032EC02B89213041F02F3F1C
:108F200049F52091600321502093600315C02091E2
:108F30005E032F5F20935E032091600321502093F6
:108F4000600318C02B89222359F02F3F99F42091F8
:108F50005E03215020935E0320915F032150D9CFFF
:108F6000209160032F5F2093600320915E032150C6
:108F700020935E032EE1289FD001299FB00D11247C
:108F8000A158B34EFE0101900D922A95E1F7E091B0
:108F9000110BF091120B8091600381AB8A8901C0A3
:108FA00080E0DF91CF910895CF93DF931092620319
:108FB00080915D03811103C020E030E05CC010921D
:108FC000610380915F03882309F441C0E2E9FCE179
:108FD000DF0180E09C918F5F911108C0ED01279720
:108FE0009881992319F08093620303C05E968F31B4
:108FF00089F780916203A091110BB091120B882325
:1090000099F091E0D0969C9390E001972EE1289FF3
:10901000F001299FF00D1124E457F34E80819181D6
:1090200097FF1AC081950CC0D0961C9280E0908169
:109030008F5F913041F4DF0117979C91992319F0CC
:109040008093610309C07E968F3189F705C0E09156
:10905000110BF091120B10AA80916203882309F47E
:10906000ABCF90E001974EE1489F9001499F300DB2
:1090700011242158334EC901DF91CF910895CF9328
:10908000DF93109262031092610380915D0381115E
:1090900003C020E030E05DC080915F03882309F4C5
:1090A00044C0E6E1F0E2DF0181E09C9191110AC049
:1090B000ED0127979881992329F090E2981B9093CE
:1090C000620304C08F5F5E97803279F780916203FC
:1090D0008823C9F0E091110BF091120B909160037D
:1090E00090AB90E001972EE1289FF001299FF00DB1
:1090F0001124E457F34E8081918197FF1BC0819525
:109100008093610317C081E09081913051F4DF01B9
:1091100017979C91992329F090E2981B90936103F3
:1091200004C08F5F7E97803279F7E091110BF09148
:10913000120B10AA80916203882309F4AACF90E051
:1091400001974EE1489F9001499F300D112421580D
:10915000334EC901DF91CF91089580915D0388233B
:1091600009F448C0809162038F31E8F59EE1989F31
:10917000900111242F58344EF901EF5DFE4F4081CC
:109180008F5F41111EC0F901E65EFE4F2081222350
:10919000C1F080936203E091110BF091120B90A942
:1091A0009F5F90AB90E001972EE1289FF001299FEF
:1091B000F00D1124E457F34E2081318137FF08C0B0
:1091C00003C08F31A1F60FC021952093610302C027
:1091D000109261034EE1489F9001499F300D112488
:1091E0002158334E09C0E091110BF091120B10AAD7
:1091F0001092610320E030E0C9010895882321F036
:1092000081E080935D03D0CE10925D0310926103E4
:1092100008958091610339CE823069F018F481306D
:10922000C9F405C0833059F08430A1F40CC022E0A9
:1092300044E257E00BC022E044E357E007C022E0DD
:1092400044E457E003C022E044E557E063E083E0F4
:109250000E9414B940E06FE070E088EE93E00C9457
:10926000DD72982F4091000147FD10C020E131E0F0
:109270004203F001439FF00D1124ED5EF44F618134
:1092800070E040E050E020E030E00EC081E0C4DF5C
:109290000FC0DF01A40FB51F9096AC912F5F3F4F19
:1092A000415F5F4F9A1729F0822F261737078CF3FB
:1092B0008FEF08954091000120E131E04203F00179
:1092C000439FF00D1124ED5EF44F80819381282F90
:1092D000291B27FD03C0263014F085508383089591
:1092E00087E00E947DB622E044E657E067E080E038
:1092F0000E9414B980E197E224EF31E0F90131973F
:10930000F1F70197D9F787E00C949EB640910001E0
:1093100020E131E04203F001439FF00D1124ED5EA6
:10932000F44F8781882339F040E06FEF7FEF89E1C8
:1093300090E00C94DD720895CF93DF93409100018B
:1093400046301CF082E068DF15C04F5F409300019B
:1093500020E131E04203F001439FF00D1124ED5E66
:10936000F44FEF01C90119920197E9F715821682AE
:1093700081E08783DF91CF9108958091000187FF7D
:1093800002C081E049CF815080930001089580930D
:10939000630308954091000147FF02C081E03CCF84
:1093A00020E131E04203F001439FF00D1124ED5E16
:1093B000F44F9287818781E0808708954091000172
:1093C00047FF02C081E028CF20E131E04203F001F5
:1093D000439FF00D1124ED5EF44F92878187108634
:1093E00008954091000147FF02C081E015CF20E1C0
:1093F00031E04203F001439FF00D1124ED5EF44F84
:10940000858308954091000147FF02C081E004CFA9
:1094100020E131E04203F001439FF00D1124ED5EA5
:10942000F44F878308954091000147FF02C081E017
:10943000F3CE20E131E04203F001439FF00D11240F
:10944000ED5EF44F868308951F931091000117FF7E
:1094500003C081E0E1DE47C0843081F420E131E0E7
:109460001203F001139FF00D1124ED5EF44F81E023
:10947000848776876587508B478735C0883681F427
:1094800020E131E01203F001139FF00D1124ED5E95
:10949000F44F81E0818B738B628B558B448B23C09F
:1094A000853081F420E131E01203F001139FF00DCB
:1094B0001124ED5EF44F81E0868B708F678B528FA5
:1094C000418F11C0893679F420E131E01203F001B7
:1094D000139FF00D1124ED5EF44F81E0838F758FA3
:1094E000648F578F468F1F9108954091000147FF69
:1094F00004C081E091DE80E0089520E131E0420384
:10950000F001439FF00D1124ED5EF44F8385089523
:109510004091000147FF04C081E07EDE80E00895B5
:1095200020E131E04203F001439FF00D1124DF01FF
:10953000AD5EB44F8C919FE0899FE00DF11D112429
:10954000ED5EF44F80A10895A1E0B0E0EAEAFAE40C
:109550000C9400F1698385DE698187FD14C0409118
:10956000000120E131E04203F001439FF00D11249E
:109570009FE08902E00DF11D1124ED5EF44F81E0C2
:10958000611180E082A32196E2E00C941CF1A1E03D
:10959000B0E0EDECFAE40C9400F1698362DE6981DD
:1095A00087FD11C04091000120E131E04203F0014C
:1095B000439FF00D11249FE08902E00DF11D11245D
:1095C000ED5EF44F63A32196E2E00C941CF1A1E060
:1095D000B0E0EDEEFAE40C9400F1698342DE6981BB
:1095E00087FD11C04091000120E131E04203F0010C
:1095F000439FF00D11249FE08902E00DF11D11241D
:10960000ED5EF44F64A32196E2E00C941CF1A0E01F
:10961000B0E0EDE0FBE40C9400F17E81609100018C
:1096200067FF02C081E00EC040E151E06403900199
:10963000659F300D1124F901ED5EF44F41814031F9
:1096400018F083E0E9DD3EC0F9018FE0489FE00DAE
:10965000F11D1124ED5EF44F8F8180A3888581A3D5
:1096600012A213A289859A8596A785A78D8185A3C5
:1096700076A3CE010B96FC018FE0489F200D311D93
:1096800011242D5E344F80E090E060E00AC04191EB
:109690005191D901A80FB91F96965C934E93959757
:1096A0006F5F02966713F3CF4091000120E131E034
:1096B0004203F001439FF00D1124ED5EF44F8181D0
:1096C0008F5F8183E2E00C941CF1EF92FF920F9385
:1096D0001F93FF92EF921F930F933F932F935F93EC
:1096E0004F936F938F9383E08F9381E08F938FDFFE
:1096F0008DB79EB70C969EBF8DBF1F910F91FF90A7
:10970000EF900895EF92FF920F931F93FF92EF92C5
:109710001F930F933F932F935F934F936F938F9369
:1097200083E08F931F9273DF8DB79EB70C969EBF19
:109730008DBF1F910F91FF90EF9008953F932F934E
:109740005F934F936F938F9381E08F938F935FDF3E
:109750008DB79EB708969EBF8DBF08953F932F93F8
:109760005F934F936F938F9381E08F931F924FDF9F
:109770008DB79EB708969EBF8DBF0895A1E0B0E05B
:10978000E4ECFBE40C94F0F0182F8091000187FFCB
:1097900003C081E041DD6EC2113009F0BCC000E0C1
:1097A0002FE246E068E080E00E947BB72FE342E0D2
:1097B00060E08DE70E947BB74091000120E131E03D
:1097C0004203F001439FF00D1124ED5EF44F21851B
:1097D00032852115310509F446C0909163038085D7
:1097E000992349F1882329F03F932F938AE797E043
:1097F00004C03F932F9381E897E09F938F931F922C
:109800001F9282E08F931F921F920E94E7BDDEBFDE
:10981000CDBF40910001552747FD5095A12CCC2488
:10982000C39462E0E62E00E021E030E060E080E0FA
:109830000E94BFBE1FC0882329F03F932F9388E862
:1098400097E004C03F932F938EE897E09F938F9308
:109850001F921F9282E08F931F921F920E94E7BD7A
:10986000DEBFCDBF07C001E027E040E860E080E058
:109870000E947BB781E090E00E943EDE20E0AC01D8
:1098800067E080E00E9414B94091000120E131E0DE
:109890004203F001439FF00D1124ED5EF44F8485E7
:1098A0008823A9F085859685009789F09F938F93EB
:1098B00084E997E09F938F931F921F921F9287E0F6
:1098C0008F9381E18F930E94E7BDDEBFCDBF4091B2
:1098D000000120E131E04203F001439FF00D11242B
:1098E000ED5EF44F86898823B1F02789308D2115EC
:1098F000310589F03F932F9388E997E09F938F93E9
:109900001F921F921F9287E08F938CE08F930E948B
:10991000E7BDDEBFCDBF4091000120E131E0420351
:10992000F001439FF00D1124ED5EF44F86818823F2
:1099300059F0113039F400E028E048E160E086E6B3
:109940000E947BB70E94D0B488E0682E11E09FE0AF
:10995000D92E22EB222E27E0322ECC24C3943EEBCC
:10996000432E37E0532E4CE9842E47E0942E58EADC
:10997000E52E57E0F52E80910001992787FD9095FF
:10998000E0E1F1E08E9F90018F9F300D9E9F300DA2
:109990001124F901ED5EF44F43814150410F518193
:1099A000451708F010C1508145130CC0F901D49E31
:1099B000E00DF11D1124ED5EF44F22A1222321F0D0
:1099C000A5E103C0A0E201C0ADE1242F30E060E1D9
:1099D00071E0869FF001879FF00D969FF00D112496
:1099E000D49EE00DF11D1124ED5EF44F43A1411111
:1099F00002C0B0E201C0BAE2D29EF001D39EF00DE7
:109A0000112460E171E0869FA001879F500D969F11
:109A1000500D1124E40FF51FED5EF44FB1A072E07C
:109A2000B71611F000E201C00DE1D29EF001D39E05
:109A3000F00D112460E171E0869FA001879F500D19
:109A4000969F500D1124E40FF51FED5EF44F74A0A6
:109A500071100FE1D29EF001D39EF00D112460E150
:109A600071E0869FA001879F500D969F500D112495
:109A7000E40FF51FED5EF44F46A1413019F0A090C0
:109A8000741B01C0A12CD29EB001D39E700D112475
:109A9000E0E1F1E08E9FA0018F9F500D9E9F500D41
:109AA0001124FB01E40FF51FED5EF44FE5A1EE2359
:109AB000E9F1F2E0BF1611F0772021F11F920F9328
:109AC000D29EA001D39E500D1124FA01EA0DF11D82
:109AD000EA0DF11D40E151E0849F9001859F300D1A
:109AE000949F300D1124E20FF31FED5EF44F80A51B
:109AF0008F9387A18F931F92BF931F92AF939F92D3
:109B00008F923CC0FB01EA0DF11DEA0DF11DE40F3F
:109B1000F51FED5EF44F80A58F9387A18F931F9261
:109B2000BF931F92AF93FF92EF9245C0E2E0BE1643
:109B300011F0772069F11F920F93D29EA001D39E5E
:109B4000500D1124FA01EA0DF11DEA0DF11D40E15D
:109B500051E0849F9001859F300D949F300D11241A
:109B6000E20FF31FED5EF44F80A58F9387A18F93D3
:109B70001F92BF931F92AF933F922F921F921F92FB
:109B80001F921F93CF920E94E7BDDEBFCDBF22C0C0
:109B9000FB01EA0DF11DEA0DF11DE40FF51FED5E6D
:109BA000F44F80A58F9387A18F931F92BF931F922D
:109BB000AF935F924F921F921F921F921F93CF926B
:109BC0000E94E7BDE2CF00E027E04AE7662D86E08D
:109BD0000E947BB71F5F98E0690E173009F0CBCE6B
:109BE00000910001112707FD109580E191E0089F89
:109BF000F001099FF00D189FF00D1124ED5EF44F58
:109C000081818730B8F1E82EF12C8EE091E0B70128
:109C10000E94A0F0362F6E3208F03DE280E191E024
:109C2000089FF001099FF00D189FF00D1124ED5EC3
:109C3000F44F23814DE250E0431B5109249FC001A2
:109C4000259F900D1124B701665071090E94A0F064
:109C5000162F00E02DE241E069E080E039830E94A8
:109C60007BB7612F675F01E03981232F41E080E0FE
:109C70000E947BB72196E2E10C940CF1A0E0B0E0E9
:109C8000E4E4FEE40C94F7F0982E4091000147FFC5
:109C900002C081E00DC020E131E04203F001439FAA
:109CA000F00D1124ED5EF44F8181811104C084E038
:109CB000B3DAD0E02FC1992019F08481811112C04C
:109CC00080EF0E94997281E059DD4091000120E10E
:109CD00031E04203F001439FF00D1124ED5EF44F9B
:109CE00081E0848300E111E07FE0F72EE4E0EE2ED6
:109CF000F8E6DF2EA9E6CA2EB5E0BB2E20910001C2
:109D00002003F001219FF00D1124ED5EF44F138626
:109D10000E94BF8DC1E0811101C0C0E080E40E94BB
:109D20009972882399F0209100012003F001219F6E
:109D3000F00D1124ED5EF44F4081242F30E081813D
:109D400090E001972817390744F00AC062E080E4E8
:109D50000E94D1728111E7CF0AC04F5F408306C0D5
:109D60008581882311F0108201C0D0DAA3DA80E85F
:109D70000E949972882369F0209100012003F0016C
:109D8000219FF00D1124ED5EF44F808181110CC0F4
:109D900007C062E080E80E94D1728111EDCF09C056
:109DA0008581882321F081818150808301C0AEDAD2
:109DB00081DA209100012003F001219FF00D112490
:109DC000ED5EF44FA08080E10E94A372882359F1D8
:109DD000209100012003D001219FB00D1124FD012D
:109DE000FA9CE00DF11D1124ED5EF44F82A1882351
:109DF00011F076DA18C005A4F6A5E02D309709F029
:109E000008C0AD5EB44F1F96ED91FC91509730970E
:109E100031F0099580EF0E949972C1E004C01B9651
:109E2000EC92D1E001C0D0E0209100012003F001CC
:109E3000219FF00D1124ED5EF44F81898823E9F014
:109E400080E10E94B8728823C1F0209100012003B4
:109E5000D001219FB00D1124AD5EB44F5496ED9109
:109E6000FC915597309731F0099580EF0E949972D7
:109E7000C1E003C01B96DC92D2E0209100012003D8
:109E8000F001219FF00D1124ED5EF44F838D8823A6
:109E9000E9F080E20E94B8728823C1F020910001AD
:109EA0002003D001219FB00D1124AD5EB44F5E960A
:109EB000ED91FC915F97309731F0099580EF0E940A
:109EC0009972C1E003C01B96CC92D2E080E20E945E
:109ED000A3728823C1F0209100012003D001219FAB
:109EE000B00D1124AD5EB44F5996ED91FC915A9787
:109EF000309731F0099580EF0E949972C1E003C05C
:109F00001B96BC92D2E08C2F39DCD11103C0992072
:109F100009F4F4CE8D2FCDB7DEB7EBE00C9413F13E
:109F200087E00E947DB622E048EC57E067E080E0E1
:109F30000E9414B980E197E224EF31E0F9013197F2
:109F4000F1F70197D9F787E00C949EB6CF93DF9392
:109F5000D62FC42F20E04EED57E0682F8C2F0E94A3
:109F600014B920E040EE57E06D2F8C2F0E9414B9F9
:109F7000DF91CF910895EF92FF920F931F93CF93AC
:109F8000DF93182F062FF42ED22F622F822FDEDFC1
:109F9000CD2F80E40E949972E82E61E080E40E9457
:109FA000D1728E2929F0C01710F4CF5F01C0C02FE5
:109FB00080E80E949972E82E61E080E80E94D172E8
:109FC0008E2929F01C1710F4C15001C0C12FCD17E4
:109FD00029F04F2D6C2F8D2FB9DFDC2F80E30E94ED
:109FE00099728823B1F285FDCFEF8C2FCDB7DEB704
:109FF000E6E00C9418F1A0E0B0E0E1E0F0E50C94AC
:10A00000FBF0182FF62ED42FE22E41E06D2F8D2F6E
:10A010009DDFCD2F80E40E949972D82E61E080E40C
:10A020000E94D1728D2939F0CF1510F4CF5F03C093
:10A03000013011F1CF2D80E80E949972D82E61E095
:10A0400080E80E94D1728D2941F01C1710F4C15094
:10A0500004C081E0E81691F0C12FCD1729F041E04E
:10A060006C2F8D2F73DFDC2F80E30E949972882381
:10A0700089F285FD05C005C0CEEF03C0CDEF01C05C
:10A08000CFEF8C2FCDB7DEB7E7E00C9417F1A0E04F
:10A09000B0E0EDE4F0E50C94FBF0182FF62ED42F91
:10A0A000E22E41E06D2F8D2F51DFCD2F80E40E94F5
:10A0B0009972D82E61E080E40E94D1728D2941F01E
:10A0C000CF1510F4CF5F04C0013009F441C0CF2D8B
:10A0D00080E80E949972D82E61E080E80E94D172D7
:10A0E0008D2941F01C1710F4C15004C081E0E8161E
:10A0F00089F1C12F80E20E94B872882329F080EF95
:10A100000E949972CAEF27C080E10E94B87288232A
:10A1100029F080EF0E949972CBEF1DC080E20E946F
:10A12000A372882329F080EF0E949972CCEF13C0AC
:10A13000CD1729F041E06C2F8D2F08DFDC2F0E9416
:10A14000D0B480E10E94A372882309F4AFCF03C08A
:10A15000CEEF01C0CDEF8C2FCDB7DEB7E7E00C948A
:10A1600017F1A0E0B0E0E7EBF0E50C94F8F07C012B
:10A17000162F10927311C62FD0E086E3B82E92E10D
:10A18000A92E6E0181E0C81AD10810926703809150
:10A190006603882339F020E042EE57E061E081E079
:10A1A0000E9414B91092670331C02091660330E019
:10A1B000260F311D2C173D0794F4B29EA001B39ECB
:10A1C000500D11244E0D5F1D8091741BA89E400DF3
:10A1D000511D11246F5F20E083E00E9414B980912B
:10A1E0006703853071F48091660390E005968C15C5
:10A1F0009D053CF420E044EE57E066E081E00E94DB
:10A2000014B9809167038F5F809367036091670340
:10A21000663058F28091640381111CC080916603FE
:10A2200081110FC0173030F001E020E040910101B2
:10A2300065E005C000E020E040910101612F81E070
:10A2400006C001E021E04091010165E082E0D3DE3B
:10A2500080937311809164038130B9F42091660377
:10A2600030E02A5F3F4F2C173D0734F000E021E03B
:10A270004091010166E005C001E021E0409101014B
:10A2800065E082E0B8DE80937311809173118E3F98
:10A2900051F4809166038F5F8093660381E0809321
:10A2A000640385E00AC08D3F59F4809166038150B4
:10A2B000809366031092640382E08093010165CF6E
:10A2C000CDB7DEB7EAE00C9414F1CF93C82F26E1A6
:10A2D000829FC00111240E942DF1909375118093EB
:10A2E00074110097F1F40E9458B520E046EE57E053
:10A2F00063E081E00E9414B920E047EF57E064E09A
:10A3000081E00E9414B940E063E373E384EF91E0DD
:10A310000E94DD7280E20E94A3728823D9F380E05C
:10A320000BC0C09376111092771110927811109291
:10A33000791110927F1181E0CF910895809174116D
:10A3400090917511009711F00E94C8F1109275114B
:10A350001092741108958091771190917611891758
:10A3600070F4E0917411F091751196E1899FE00D00
:10A37000F11D11249AE090838F5F809377110895E7
:10A38000FF920F931F93CF93DF93F62E9091771147
:10A39000609176119617E0F4C0917411D091751107
:10A3A00066E1969FC00DD11D112489019A0145E1F6
:10A3B00065E871E15AD145E150E065E871E1CE010F
:10A3C0000196E7D3F882809177118F5F80937711A0
:10A3D000CDB7DEB7E5E00C9419F1A0E0B0E0E3EF13
:10A3E000F1E50C9400F1CE0108969C014E815F814D
:10A3F0006D8181E0C5DFE2E00C941CF1A0E0B0E0EB
:10A40000E4E0F2E50C9400F1CE0108969C014E8147
:10A410005F816D8180E0B4DFE2E00C941CF1843058
:10A4200041F481E08093791145E050E08AE791E1C1
:10A4300009C0883641F481E080937F1145E050E007
:10A4400080E891E1A6C30895FF920F931F93CF93E5
:10A45000DF9310E0C0E0D0E086E1F82E2091741187
:10A460003091751180917811AE01480F511DCA01CC
:10A470004091771150E08417950714F5F89EF0018C
:10A48000F99EF00D1124E20FF31F20812A3081F490
:10A4900000E027E048E7612F86E00E947BB7612F4C
:10A4A0006D5F01E0262F4DE786E00E94CBB60FC01E
:10A4B000AF014F5F5F4F6C2F81E00E9440B907C032
:10A4C00000E027E048E7612F86E00E947BB72196F5
:10A4D000185F183319F6E0917711F0E081E891E008
:10A4E000BF010E94A0F0C62F683308F0C7E3209197
:10A4F000781147E350E04C1B5109249FC001259F70
:10A50000900D1124BF01675071090E94A0F0D62F51
:10A5100000E027E341E060E080E00E947BB701E0DB
:10A520002C2F41E06D2F80E00E947BB781E090E00E
:10A530000E943EDE20E0AC0167E080E00E9414B99A
:10A5400080917911882321F020E04AE751E107C08A
:10A5500080917F1120E0882339F040E851E167E0E5
:10A5600081E10E94C7B806C043E058E067E081E19E
:10A570000E9414B9CDB7DEB7E5E00C9419F1CF9382
:10A580008091741190917511892B09F467C05CDF7B
:10A590000E94BF8D882319F00E9458B555DF80E4D2
:10A5A0000E949972882361F040917811242F30E045
:10A5B0008091771190E007972817390744F00CC075
:10A5C00062E080E40E94D1728111EECF0CC04F5F37
:10A5D0004093781139DF07C040E06FEF7FEF89E1EA
:10A5E00090E00E94DD7280E80E949972882329F031
:10A5F00080917811811108C00CC062E080E80E944F
:10A60000D1728111F5CF0CC08150809378111CDF7D
:10A6100007C040E06FEF7FEF89E190E00E94DD72BC
:10A6200080917911811102C0C0E006C080E10E94D2
:10A63000A3728823C9F3C4E080917F11882329F095
:10A6400080E10E94B8728111C8E680E20E9499728E
:10A65000811105C0CC2309F49BCF01C0C0E080EF7D
:10A660000E9499728C2FCF910895A0E1B0E0EBE3A6
:10A67000F3E50C94F0F06B01B42E882361F040E513
:10A6800050E0B9018AE991E10E94C7F31092E91103
:10A690008AE991E101C0C9011982BB2009F448C2CD
:10A6A0001C017601A12CC12CD12C4B2C512C2EE25B
:10A6B000622E9E012F5F3F4F3A8729879981911122
:10A6C00013C0D1018C91853259F488E0E985FA856F
:10A6D00011928A95E9F781E0898380E2888727C013
:10A6E000D7018D937D0117C2913009F052C0F1015D
:10A6F0008081803339F4FAEECF16F1E1DF0631F4D0
:10A7000088870EC2803330F08A33B0F4D6018D933F
:10A710006D0106C28E3281F48D8181113AC09D8314
:10A72000F60110828AEE91E10E9490F38B839AEEFB
:10A73000C92E91E1D92EF4C18C3619F481E08E83B3
:10A74000EFC1843681F0853771F0883761F0823649
:10A7500051F08F3641F0833731F0833521F0833665
:10A7600011F08532B1F48A831982D6011C928D8151
:10A77000811108C08AEE91E10E9490F38B838111D0
:10A7800006C007C08AEE91E10E9490F38C8381E0BD
:10A790008F838A81843649F0853739F0883729F0EC
:10A7A000823619F08F3609F067C19E81992309F42A
:10A7B00054C08F3609F441C030F4823691F18436AA
:10A7C00009F08EC006C08537A1F0883709F088C02F
:10A7D0001CC04801B4E08B0E911CF80160817181AE
:10A7E000828193812AE030E041EF51E10E9492F4AE
:10A7F00076C04801F4E08F0E911CD8016D917D91D7
:10A800008D919C912AE030E023C04801B4E08B0E8A
:10A81000911CF801608171818281938120E130E097
:10A8200017C04801F4E08F0E911CD8016D917D9105
:10A830008D919C9122E030E00BC04801B4E08B0E7A
:10A84000911CF801608171818281938128E030E060
:10A8500041EF51E10E94CCF442C08F3699F128F4C7
:10A86000823621F18436E1F505C0853789F08837D5
:10A87000B9F515C04801F2E08F0E911C4AE050E096
:10A8800061EF71E1D8018D919C910E9473F427C012
:10A890004801B2E08B0E911C4AE050E00DC0480127
:10A8A000F2E08F0E911C40E150E012C04801B2E08E
:10A8B0008B0E911C42E050E061EF71E1F801808164
:10A8C00091810BC04801F2E08F0E911C48E050E0EE
:10A8D00061EF71E1D8018D919C910E94EFF48401A8
:10A8E00061E08091F1118D3209F060E08B812C8163
:10A8F000A22FA80F91E03D81311101C090E0A90F76
:10A90000E1EFF1E101900020E9F73197E15FF141DA
:10A910007F81772389F090E0AF0155274C01820EAB
:10A92000911C841695061CF481E090E007C0262F48
:10A9300030E028173907C4F780E090E0892B99F4BC
:10A940001BC08D81882331F08B81981303C0F701E0
:10A95000608204C08AE2882EF70180822FEFE21A1B
:10A96000F20A9F5F01C090E0892F8A0D9A1709F4BF
:10A97000D4C08B1530F3DDC09E2E711101C0AE2FF7
:10A98000762E662331F09A9442EF51E15C874B8733
:10A9900004C081EF91E19C878B8788248394B1E088
:10A9A0008A2F90E0FC01EA0DF11DFE87ED87292D2D
:10A9B00030E0388B2F8758C06B2F61502B2F30E041
:10A9C0004D855E85421B530B441655060CF44BC057
:10A9D0004D81442351F04C81641307C0FC01E21BFC
:10A9E000F30BEE0DFF1D60823EC0981488F0EF85DA
:10A9F000F889E819F1094B855C85E40FF51F408162
:10AA0000FC01E21BF30BEE0DFF1D408383942BC072
:10AA10004C81442389F0641738F070E050E04F5FB8
:10AA20005F4F6417750741F4FC01E21BF30BEE0D59
:10AA3000FF1D50E3508317C0FC01E21BF30B9F0185
:10AA4000772061F04885403211F0BA1307C0F70152
:10AA5000E20FF31F2DE22083712C05C04885F7011A
:10AA6000E20FF31F4083BF5FAB1708F0A5CFE80EDE
:10AA7000F91E8A2F8A0D51C0833731F0833551F08A
:10AA8000833609F043C017C0D801ED91FC910E5FE9
:10AA90001F4F1BC04801B2E08B0E911CF801608172
:10AAA000718140E550E081EF91E10E94C7F310927F
:10AAB0004012840108C0D8018C918093F11110924A
:10AAC000F2110E5F1F4FE1EFF1E12B81DF010D90DD
:10AAD0000020E9F71197AE1BBF0B8F81811101C0D8
:10AAE0002A2F2A0D8A2D30E20EC08B1558F4908142
:10AAF000D701992319F09C93319601C03C93BFEF85
:10AB0000EB1AFB0A8F5F8213F0CF07C0853241F446
:10AB1000F70181937F018A2D8F5F8B1550F4A82E4A
:10AB2000D1018D911D018111C9CD80E090E003C05C
:10AB300076018FEF9FEFF701E80FF91F1082609603
:10AB4000E2E10C940CF1A0E0B0E0E9EAF5E50C9448
:10AB5000FEF0CE010C968C012A853B8549856F81DC
:10AB6000788580E082DDE4E00C941AF1A0E0B0E0AA
:10AB7000ECEBF5E50C94FEF0CE010C968C012A85E9
:10AB80003B8549856F81788581E06FDDE4E00C9439
:10AB90001AF1DB01FC0190E060E20AC02D91222352
:10ABA00011F0992319F0608391E001C02083319660
:10ABB0002E2F281B30E02417350780F331971082A1
:10ABC0000895FC0101900020E9F7E81BF90B32978A
:10ABD000E80FF91F01C03197E817F90721F48081C8
:10ABE000803229F406C020812032A9F3F8CF8111E8
:10ABF000319610820895ACE0B0E0E1E0F6E50C9407
:10AC0000F8F02CE0EAECF1E0DE01119601900D92F3
:10AC10002A95E1F700912D1C10912E1C28E0FB01D4
:10AC2000DC0101900D922A95E1F7DC011696AD90BA
:10AC3000BC901797A114B10409F4ABC01596AC9160
:10AC4000AA2309F4A6C0AD3008F0A3C0FC014081DE
:10AC5000518162817381E02FE10F30E1E32E3EE00C
:10AC6000F32E2E2F870120036001219FD00C112489
:10AC7000EE24D7FCE094FE2C4C0D5D1D6E1D7F1D57
:10AC8000413831E5530731E06307710534F040582E
:10AC9000514561407109B1E009C077FF06C04058D5
:10ACA0005E4A6E4F7F4FBFEF01C0B0E0FC014083B2
:10ACB00051836283738314814B2F552747FD509531
:10ACC000652F752F410F511D611D711D0A2F10E059
:10ACD0007E01E00EF11EF701C080DD24C7FCD09498
:10ACE000ED2CFD2CC416D506E606F706ACF01416BE
:10ACF000150616061706B4F0A130B1F0AE014150AA
:10AD00005109400F511FFA014081552747FD5095C9
:10AD1000652F752FBFEF0DC0B1E041E050E060E05E
:10AD200070E007C0B0E005C0BFEF4FE150E060E069
:10AD300070E0FC0144834B2F552747FD5095652F4C
:10AD4000752F4A0F511D611D711D4D305105610553
:10AD5000710539F0411551056105710541F0E0E0DB
:10AD60000BC0E1E041E050E060E070E005C0EFEFD3
:10AD70004CE050E060E070E0DC0115964C931597D4
:10AD800095012E0F311DE7FD3A9517963C932E93B2
:10AD900016972C96EAE00C9414F11F920F920FB6BE
:10ADA0000F9211240BB60F922F938F939F93EF93D3
:10ADB000FF938091C8009091CE008871E0916B0361
:10ADC000EF5F20916A03E2130BC0809141129091D2
:10ADD00042120196909342128093411282E006C083
:10ADE000E0936B03F0E0E259FC4F9083809369039A
:10ADF000FF91EF919F918F912F910F900BBE0F902C
:10AE00000FBE0F901F9018951F920F920FB60F92C2
:10AE100011240BB60F928F939F93EF93FF93909112
:10AE20006D0380916C03981769F0E0916C03EF5FFC
:10AE3000EF73E0936C03F0E0E259F84F8081809368
:10AE4000CE0005C08091C9008F7D8093C900FF911D
:10AE5000EF919F918F910F900BBE0F900FBE0F90AF
:10AE60001F90189510926D0310926C0310926B0353
:10AE700010926A03109242121092411297FF04C07E
:10AE800022E02093C8009F779093CD008093CC0060
:10AE900088E98093C90086E08093CA0008958330D2
:10AEA000B9F020F4813071F080F406C08530B1F043
:10AEB00090F08630B1F403C087E092E011C083E0E7
:10AEC00091E00EC081E890E00BC080E490E008C003
:10AED0008FE190E005C084E190E002C08AE090E05C
:10AEE000C1CF089590916B0380916A03981781F008
:10AEF000E0916A03EF5FE0936A03F0E0E259FC4FF0
:10AF0000808190916903392F20E0280F311D02C004
:10AF100020E031E0C901089590916B0380916A03AC
:10AF2000981771F0E0916A03EF5FF0E0E259FC4F8F
:10AF3000808190916903392F20E0280F311D02C0D4
:10AF40002FEF3FEFC901089590916D039F5F9F73AD
:10AF500020916C039217E1F3E92FF0E0E259F84FEA
:10AF6000808390936D039091C90090629093C90083
:10AF700090916903392F20E0280F311DC9010895F0
:10AF8000CF93DF93EC0101C0DFDF89918111FCCF0A
:10AF9000DF91CF910895CF93DF93EC0101C0D4DF0F
:10AFA000FE01219684918111FACFDF91CF9108950E
:10AFB00080916B0320916A0390E081509C4F821B2B
:10AFC00091096FEF73E00C94A0F080916A03809375
:10AFD0006B030895CF93DF939C01FB013197E80F3A
:10AFE000F91F1082CAE0D0E0CA01BE010E948CF0B5
:10AFF000805D8293AB016115710519F02E173F0733
:10B0000098F3CF01DF91CF9108951F920F920FB661
:10B010000F9211240BB60F922F933F934F935F9390
:10B020006F937F938F939F93AF93BF93CF93EF9340
:10B03000FF9380917C0A853009F402C0843081F549
:10B040004091C6008091BA079091BB072091B80744
:10B050003091B907821B930B97FF02C0805C9F4F12
:10B06000CF970CF0B8C0E091BA07F091BB074083CE
:10B070008091BA079091BB0701969093BB0780938C
:10B08000BA078091BA079091BB078C5F974009F08F
:10B09000A2C08CEB97E09093BB078093BA079BC04C
:10B0A000C091C60080914408882331F08091DE1B56
:10B0B000882311F08C2F48DF8091B70781118BC056
:10B0C0008091FC0781110EC0C33279F4C093431202
:10B0D00081E08093FC0783E290E09093FE078093E9
:10B0E000FD0779C0843B08F069C0482F50E0CD309F
:10B0F00091F0FA01ED5BFD4EC0838F5F8093FC07FA
:10B100002091FD073091FE072C0F311D3093FE0773
:10B110002093FD0760C0DA01AF5BBD4E6C91FA0170
:10B12000EE5BFD4E90812091FD073091FE07261BBE
:10B130003109291B3109B9017F707093FE076093B3
:10B14000FD079C91A6E076956795AA95E1F7635C6B
:10B15000691326C090812F733327235C291320C0E5
:10B16000FA01ED5BFD4EC0838F5F8093B60790912F
:10B170007E0A8091451298131EC081E08093B70724
:10B18000809145128235B9F42CE088E190E00FB649
:10B19000F894A895809360000FBE209360000BC0C8
:10B1A0008091B1079091B20701969093B207809376
:10B1B000B1071092B7071092FC070DC08091AF073E
:10B1C0009091B00701969093B0078093AF071092CB
:10B1D000FC071092B707FF91EF91CF91BF91AF910C
:10B1E0009F918F917F916F915F914F913F912F919F
:10B1F0000F900BBE0F900FBE0F901F9018952091CF
:10B20000BA073091BB078091B8079091B90728170A
:10B210003907C9F0E091B807F091B9078081209112
:10B22000B8073091B9072F5F3F4F3093B90720938C
:10B23000B8072C5F374041F42CEB37E03093B90767
:10B240002093B807089580E008954091BA0750917F
:10B25000BB072091B8073091B90742175307D1F0C7
:10B26000E091B807F091B9072081FC01208380911B
:10B27000B8079091B90701969093B9078093B807E2
:10B280008C5F974049F48CEB97E09093B9078093DB
:10B29000B80702C080E0089581E008959093C5004A
:10B2A0008093C4008091C0008D7F8093C00086E0B1
:10B2B0008093C2008091C1008B7F8093C10002C047
:10B2C0008091C6008091C00087FDFACF8091C100B7
:10B2D00088618093C1008091C10080688093C10023
:10B2E0008CEB97E09093B9078093B8079093BB07D6
:10B2F0008093BA0708958330B9F020F4813071F05B
:10B3000080F406C08530B1F090F08630B1F403C00F
:10B3100087E092E011C083E091E00EC081E890E008
:10B320000BC080E490E008C08FE190E005C084E1AC
:10B3300090E002C08AE090E0B1CF0895E1ECF0E047
:10B340008081877F808323982B980895239A2B9858
:10B35000E1ECF0E080818860808308959091C000E6
:10B3600095FFFCCF8093C6000895CF93DF93EC0147
:10B3700001C0F4DF89918111FCCFDF91CF91089555
:10B38000CF93DF93EC0102C0E9DF2196FE018491A7
:10B390008111FACFDF91CF910895A0E0B0E0E3ED05
:10B3A000F9E50C94FAF08C850D8593E290931613D1
:10B3B0008F59809317138B8580931813FE013E9647
:10B3C000002341F04E855F85828193810150FE010B
:10B3D000729604C080E090E040E050E010E023E08E
:10B3E00030E072C0DA01A10FB11DEC901F5F019730
:10B3F00079F4002309F4AEC040815181DF01149635
:10B4000082819381015010E0009709F4A4C001C02B
:10B41000DF01FA01E10FF11D60811F5F019789F4DF
:10B42000002309F499C04D915C911197FD01349668
:10B4300012968D919C911397015010E0009799F00E
:10B4400001C0FD01DA01A10FB11DFC901F5F019742
:10B4500059F4002349F04081518182819381015048
:10B46000349610E001C0F12C7E2D76957695735CB4
:10B47000D901AA5EBC4E7C93762F72957F70BE2D4B
:10B48000B370A0E1BA9F600111247C29735CD901DB
:10B49000A95EBC4E7C936F70A4E06A9FB00111243A
:10B4A0007F2D7295769576957370762B735CD901A6
:10B4B000A85EBC4E7C936F2D6F73635CD901A75E51
:10B4C000BC4E6C932C5F3F4F009709F08BCF80E010
:10B4D00090E060E007C0FA01EA5EFC4E4081840F14
:10B4E000911D6F5F462F50E042175307A0F3AC0148
:10B4F0005F70B6E056954795BA95E1F7435CF90160
:10B50000EA5EFC4E40838F739927835CF901E95E04
:10B51000FC4E8083F901E85EFC4E8DE080832D5F58
:10B520003F4F1092020140E00CC08091C00085FFA7
:10B53000FCCFE42FF0E0EA5EFC4E80818093C600F1
:10B540004F5F842F90E08217930778F381E0809318
:10B55000020106C0DF0160E0FD0180E090E083CFE2
:10B56000E8E00C9416F1A2E0B0E0E9EBFAE50C9407
:10B57000FEF0182F062F4A83E9DE8A816AE00E94D6
:10B5800080F089831F9291E09F939E012F5F3F4F30
:10B590003F932F939F930F931F93FFDEDEBFCDBF8B
:10B5A000809102018823E1F3C9DE2296E4E00C9445
:10B5B0001AF17091B607765063E0A3E048C0EA2F15
:10B5C000F0E0ED5BFD4E4081EA2FEF5FF0E0ED5BD8
:10B5D000FD4E20812D53EA2FEE5FF0E0ED5BFD4E36
:10B5E00090819D53EA2FED5FF0E0ED5BFD4EB08161
:10B5F000BD53AC5FE62FF0E0822F82958F704D53E4
:10B6000034E0439FA0011124842BED5BFD4E808329
:10B61000E62FEF5F7130F1F0F0E080E1289F9001BC
:10B620001124892F86958695822BED5BFD4E8083B4
:10B63000E62FEE5F723071F0F0E020E4929FC001DF
:10B6400011248B2BED5BFD4E80836D5F7350711168
:10B65000B6CF01C06E2F86E492E19093B507809338
:10B66000B40763506093B3070895CF93C0917D0AE8
:10B67000C130A9F48BE172DE8BE170DE85E56EDE10
:10B680008AEA6CDE80E06ADEC0937C0A84EF91E097
:10B6900024EF31E0F9013197F1F70197D9F7CF9114
:10B6A000089585E080937C0A84EF91E024EF31E0F7
:10B6B000F9013197F1F70197D9F70895A1E0B0E0CA
:10B6C000E4E6FBE50C94FFF020917C0A2130D1F4F4
:10B6D00019821F922F93CE0101969F938F932F93E0
:10B6E00012E01F9385E78F9358DE10937C0ADEBF2C
:10B6F000CDBF84EF91E024EF31E0F9013197F1F70C
:10B700000197D9F72196E3E00C941BF1A1E0B0E09A
:10B71000ECE8FBE50C9400F120917C0A2130D9F48F
:10B7200029831F922F93CE0101969F938F932F937E
:10B7300082E08F9385E78F9330DE83E080937C0AED
:10B74000DEBFCDBF84EF91E024EF31E0F901319706
:10B75000F1F70197D9F72196E2E00C941CF1A1E0F2
:10B76000B0E0E5EBFBE50C9400F120917C0A213080
:10B77000D9F432E039831F922F93CE0101969F9323
:10B780008F932F933F9385E78F9307DE84E0809319
:10B790007C0ADEBFCDBF84EF91E024EF31E0F901F8
:10B7A0003197F1F70197D9F72196E2E00C941CF15B
:10B7B000CF92DF92EF92FF92CF93DF936B017C01E8
:10B7C000CFE0D0E0E0E0F0E840E050E8F695E79523
:10B7D0009A01DA010E9455F0C616D706E806F90666
:10B7E00018F44E1B5F0B02C04E0F5F1F219771F7BD
:10B7F0009A01DA010E9455F0C616D706E806F90646
:10B8000010F441505109CA01DF91CF91FF90EF90A0
:10B81000DF90CF9008951F932AE530E0281B390B65
:10B8200037FF05C03195219531091FEF01C011E0A7
:10B83000E8E6F1E0C901BF010E94A0F08B35910557
:10B84000E4F09C012B5531092A35310538F424EBFD
:10B8500030E0A901481B590BCA010FC09C01255BB0
:10B8600031092A35310518F4845B910904C09F0120
:10B87000281B390BC9016FEF01C061E0FC01EE0F1D
:10B88000FF1FEA52FE4F208131811203A001139F56
:10B89000500D112464039001659F300D1124C901DE
:10B8A0001F910895ACE0B0E0E8E5FCE50C94F2F0FF
:10B8B00069837A838B839C8349015A0169817A81E8
:10B8C00077FF03C0719561957109882777FD809591
:10B8D000982F0E9480EE8B013C0120E030E0A9010E
:10B8E000712F972D0E94DEED811105C0B7FEDFC0DC
:10B8F00044EB50E0DEC0B40197FE03C07195619542
:10B900007109882777FD8095982F0E9480EE6B0142
:10B910007C01202F312F462D572D6C2D7D2D8E2D06
:10B920009F2D0E94DEED87FF11C0202F312F462D65
:10B93000572D6C2D7D2D8E2D9F2D0E94E5ED00E065
:10B9400010E0B0E86B2E2FE3722E10C02C2D3D2D91
:10B950004E2D5F2D602F712F862D972D0E94E5EDC6
:10B960008B013C0160E070E080E89FE320E038ED6F
:10B970004BED56E40E946DEF0E944DEE6B017C0191
:10B9800020E038ED4BED56E4602F712F862D972D7A
:10B990000E946DEF0E944DEE2B013C0100E010E093
:10B9A00060E070E0CB01A7019601002E04C056951F
:10B9B0004795379527950A94D2F729873A874B8779
:10B9C0005C87A3019201002E04C0559547953795D9
:10B9D00027950A94D2F72D833E834F835887F80129
:10B9E000EE0FFF1F77FE15C0C21AD30AE40AF50A4C
:10B9F00029853A854B855C85420E531E641E751E53
:10BA0000E85FF74F25913491621B730B810991090F
:10BA100018C02D813E814F815885C20ED31EE41E71
:10BA2000F51E29853A854B855C85421A530A640ABE
:10BA3000750AE85FF74F25913491620F731F811DDE
:10BA4000911D0F5F1F4F0F30110509F0ACCF0E9401
:10BA50007EEE21EE3EE245E652E40E946DEF20E0EC
:10BA600038ED4BED56E40E94E5ED0E9452EEAB013D
:10BA7000BC01181419041A041B0464F084EB90E050
:10BA8000A0E0B0E08C019D01041B150B260B370BC9
:10BA9000B901A80189819A81AB81BC811816190668
:10BAA0001A061B0634F051954195510902C040E039
:10BAB00050E0CA012C96E0E10C940EF10895CF936A
:10BAC000C82F80916F008D7F80936F008091FE1B47
:10BAD000811150C0809181008C7F80938100809182
:10BAE000810084608093810080E18093CA1380E2AA
:10BAF0008093D6131092E3131092E213E091FE1B91
:10BB000088E0E89FF0011124EC54FD4F2681378135
:10BB100040E050E060E07DE281E391E00E94B3F01C
:10BB2000AC2FB0E00E9467F00E947EEE2FE632E17B
:10BB300043E85AE30E946DEF0E9452EE9B0170931E
:10BB4000E5136093E4134091880050918900952F8C
:10BB500080E0840F911D820F931F90938900809342
:10BB6000880080916F00826080936F0081E08093F5
:10BB7000FC130BC0809181008B7F8093810090919A
:10BB80008100936090938100AFCFCF910895E091B1
:10BB9000FE1B28E0E29FF0011124EC54FD4F2681AA
:10BBA0003781AC01429FC001439F900D529F900D81
:10BBB0001124BC0180E090E00E947EEE20E030E0A5
:10BBC00040EA51E40E94E5ED20E030E040E05FE330
:10BBD0000E947AED0E9452EECB010895E091FE1B87
:10BBE00088E0E89FF0011124EC54FD4F8481958199
:10BBF00008959CE0899FF0011124E653FC4E61708A
:10BC0000638308959CE0899FF0011124E653FC4E64
:10BC1000A091FE1B88E0A89FD0011124AC54BD4F19
:10BC200012968D919C911397680F791F7583648389
:10BC300008959CE0899FF0011124E653FC4EA091E9
:10BC4000FE1B88E0A89FD0011124AC54BD4F8D91FC
:10BC50009C91861B970B9783868308959CE0899F10
:10BC6000F0011124E653FC4E7387628744815581AD
:10BC7000A091FE1B88E0A89FD0011124AC54BD4FB9
:10BC800014968D919C911597840F951F268137816D
:10BC9000281B390B660F771F260F371F93E0220FE3
:10BCA000331F9A95E1F764E0369527956A95E1F799
:10BCB000240F351F318720870895EFE6F0E080815B
:10BCC0008D7F80830895482F50E09CE0899FF0018C
:10BCD0001124E653FC4E24813581CB016217730792
:10BCE00008F4C9012CE0249FF001259FF00D1124D8
:10BCF000E653FC4E268137812817390708F4C9011D
:10BD00009283818308951F93CF93DF93182F282F59
:10BD100030E04CE0849FF0011124E653FC4E838117
:10BD2000882371F0E091FE1B58E0E59FF00111249B
:10BD3000EC54FD4F84819581AC01461B570BBA0131
:10BD4000E091FE1B58E0E59FF0011124EC54FD4FFB
:10BD50000480F581E02DCF019695879568177907C6
:10BD600008F58CE0829FD001839FB00D1124A6536B
:10BD7000BC4E1496CD91DC9115979B0140E050E0AC
:10BD8000220F331F441F551F18960D90BC91A02DF4
:10BD9000AC1BBD0B0E9467F09F0140E050E00E9489
:10BDA000D5F022C04CE0429FD001439FB00D11243A
:10BDB000A653BC4E1896CD91DC91199716962D91ED
:10BDC0003C9117972C1B3D0B40E050E0220F331F96
:10BDD000441F551FDB01A81BB90B0E9467F09F0190
:10BDE00040E050E00E94B3F0BE01620F731F812F4C
:10BDF0006ADFDF91CF911F910895CF93DF93CEEF4C
:10BE0000DBE1E88188E0E89FF0011124EC54FD4F6C
:10BE10006481758180E077DFE88188E0E89FF00148
:10BE20001124EC54FD4F6481758181E06CDFDF915A
:10BE3000CF910895CF93C82FE091FE1B88E0E89F33
:10BE4000F0011124EC54FD4F24813581DB010E9467
:10BE500061F024EB30E040E050E00E94B3F0B90123
:10BE60008C2F51DFCF9108951F920F920FB60F9232
:10BE700011240BB60F922F933F934F935F938F93A1
:10BE80009F93EF93FF93E091FF07E23058F49BB14B
:10BE90008CE0E89FF0011124E653FC4E80818095F0
:10BEA00089238BB98091FF078F5F8093FF078230D2
:10BEB00091F010F01092FF078BB1E091FF079CE02A
:10BEC000E99FF0011124E653FC4E9081892B8BB938
:10BED000818192810AC08091E4139091E5132091B1
:10BEE000E2133091E313821B930B40918800509131
:10BEF0008900352F20E0240F311D280F391F309382
:10BF00008900209388002091E2133091E313280FD9
:10BF1000391F3093E3132093E2138091E41390913F
:10BF2000E5132817390720F01092E3131092E2135B
:10BF3000FF91EF919F918F915F914F913F912F9141
:10BF40000F900BBE0F900FBE0F901F901895EF92A1
:10BF5000FF920F931F930E949C498CE499E00E94EA
:10BF6000CA4987E6E82E89E0F82E870126E539E000
:10BF700043EE52E661E081E00E94654B95E8E92ED0
:10BF800099E0F92E870127E739E04FEE5FE562E09F
:10BF900082E00E94654B26E9E22E29E0F22E87011D
:10BFA00020E939E040E253E661E083E00E94654B1E
:10BFB00034EAE32E39E0F32E87012CE939E042E53B
:10BFC00053E661E084E00E94654B80E00E943E4EB3
:10BFD0000E94BD491F910F91FF90EF900895EF923D
:10BFE000FF920F931F930E949C4985E998E00E945D
:10BFF000CA4940EBE42E48E0F42E870125EA38E0F8
:10C0000045EC53E661E081E00E94654B59ECE52E7A
:10C0100058E0F52E87012BEB38E041EB52E661E06A
:10C0200082E00E94654B60EFE62E68E0F62E01EE9E
:10C0300018E025ED38E04FE752E661E083E00E942A
:10C04000654B7DE1E72E79E0F72E0FE019E02DEF4B
:10C0500038E04DE452E661E084E00E94654BECE399
:10C06000EE2EE9E0FE2E87012DE239E04BE152E6AB
:10C0700061E085E00E94654B80E00E943E4E0E9498
:10C08000BD491F910F91FF90EF9008950F93CF93AB
:10C09000DF93EC01A3DD96958795BE01681B790BB4
:10C0A000882777FD8095982F00E020E044E0A9D60E
:10C0B00020E0AC0162E080E10E9440B9BE018091C5
:10C0C000E613CCDD8BDDBC01769567958091E61398
:10C0D0001ADEDF91CF910F9108950F93BC0180E09C
:10C0E00090E000E020E043E08CD620E0AC0162E08C
:10C0F00080E10E9440B90F910895CF92DF92EF92B4
:10C100000F93CF93DF93EC0169DD6C01E12C00E02C
:10C1100025E030E0AE0162E080E10E94EBBEBE01AE
:10C120008091E61386DD8091E61397E0899FF00108
:10C130001124E051F44E9081992311F0C12CD12C9F
:10C14000B601E1DDDF91CF910F91EF90DF90CF90BD
:10C150000895EF920F93CF93DF93EC01E12C00E071
:10C1600025E030E0AC0162E080E10E9423BFBE0127
:10C170008091E61347DDE091E61387E0E89FF00148
:10C180001124E051F44E8081882311F027DD02C094
:10C1900080E090E0BC018091E613B5DDDF91CF91A6
:10C1A0000F91EF900895EF92FF920F93CF93DF934B
:10C1B000EC01BC018091E61386DDE091FE1B26E0D8
:10C1C000E29FF0011124E057FD4F84819581DE014B
:10C1D000A81BB90B4281538120813181B7FF04C074
:10C1E000AC01421B530B02C0481B590B28EE33E035
:10C1F0000E9461F09A01442737FD4095542F0E9418
:10C20000D5F07901CE01C3DC883E23E0920710F41B
:10C2100064DF0DC0BC0180E090E003E023E045E076
:10C22000F0D520E0AC0162E08EE00E9440B9B70199
:10C23000882777FD8095982F01E021E046E0E1D541
:10C2400020E0AC0162E08EE00E9440B9DF91CF9126
:10C250000F91FF90EF900895CF93DF93EC0120E0D2
:10C2600048E258E062E080E00E9414B920E0CD2B63
:10C2700019F447E358E002C04FE258E062E08EE074
:10C280000E9414B9DF91CF910895892B19F48AE1A6
:10C2900090E002C089E190E00E943EDE20E0AC0127
:10C2A00062E081E10C9414B920E0892B19F44CEC84
:10C2B00052E002C041ED52E062E080E10C9440B9EE
:10C2C000009751F48AE190E00E943EDE20E0AC014C
:10C2D00062E081E10C9414B900CFF2CF08950F937E
:10C2E000BC018A30910570F0BC0180E090E001E073
:10C2F00021E043E086D520E0AC0162E080E10E94CD
:10C3000040B908C084E6282F269FC001279F900DC2
:10C310001124E3DE0F91089570CD0895D0DB80E005
:10C320000895A0E0B0E0E7E9F1E60C94FAF0EC0142
:10C330008B016A0180E40E949972882329F0CC1550
:10C34000DD0548F0E8010BC063E080E40E94D17293
:10C350008111F5CF07C081E0809337082196CE0187
:10C36000F701099580E80E949972882329F00C173B
:10C370001D0748F0E6010BC063E080E80E94D1721F
:10C380008111F5CF07C0219781E080933708CE0156
:10C39000F7010995CE01CDB7DEB7E8E00C9416F1B0
:10C3A0006F927F928F929F92AF92BF92CF92DF92C5
:10C3B000EF92FF920F93CF93DF93EC014B013A0181
:10C3C0005901C880D980C601F90109950AC07501D3
:10C3D00002E020E1A301B40188819981A2DF998361
:10C3E000888380E10E949972882331F02881398105
:10C3F0002C153D0551F406C080E20E9499728823F5
:10C4000031F3F4CF1092370803C081E080933708EE
:10C4100081E0C216D30609F480E0DF91CF910F913D
:10C42000FF90EF90DF90CF90BF90AF909F908F9054
:10C430007F906F900895A2E0B0E0E1E2F2E60C9404
:10C4400000F10E9458B585EC90E00E943EDE22E0AB
:10C45000AC0160E080E00E9414B982E090E00E94AC
:10C460003EDE20E0AC0167E080E00E9414B98091DC
:10C47000051C89831A822DE631E648EC50E060E025
:10C4800070E0CE0101968CDF882319F089818093BA
:10C49000051C2296E2E00C941CF1A2E0B0E0E3E57A
:10C4A000F2E60C9400F10E9458B584EC90E00E94F2
:10C4B0003EDE22E0AC0160E080E00E9414B982E040
:10C4C00090E00E943EDE20E0AC0167E080E00E9448
:10C4D00014B98091041C89831A822FE631E644E165
:10C4E00050E064E070E0CE0101965ADF882319F035
:10C4F00089818093041C2296E2E00C941CF1A2E056
:10C50000B0E0E5E8F2E60C9400F18091031C898329
:10C510001A820E9458B583EC90E00E943EDE22E031
:10C52000AC0160E080E00E9414B982E090E00E94DB
:10C530003EDE20E0AC0167E080E00E9414B92DE609
:10C5400030E644E650E061E070E0CE01019628DF7D
:10C55000882319F089818093031C2296E2E00C94D1
:10C560001CF1A2E0B0E0E7EBF2E60C9400F10E94CF
:10C5700058B58091021C89831A8282EC90E00E9457
:10C580003EDE22E0AC0160E080E00E9414B982E06F
:10C5900090E00E943EDE20E0AC0167E080E00E9477
:10C5A00014B920E631E644E150E060E070E0CE01ED
:10C5B0000196F6DE882319F089818093021C229669
:10C5C000E2E00C941CF1A2E0B0E0E9EEF2E60C949B
:10C5D00000F10E9458B58EEB90E00E943EDE22E012
:10C5E000AC0160E080E00E9414B982E090E00E941B
:10C5F0003EDE20E0AC0167E080E00E9414B980914B
:10C60000011C5DDAE091FE1B86E0E89FF001112439
:10C61000E057FD4F848195819A83898342815381BC
:10C620006081718123ED30E6CE010196B9DEF89488
:10C6300084E145DA7894E1DB2296E2E00C941CF187
:10C64000A2E0B0E0E6E2F3E60C9400F10E9458B5F7
:10C650008FEB90E00E943EDE22E0AC0160E080E0E3
:10C660000E9414B982E090E00E943EDE20E0AC011E
:10C6700067E080E00E9414B98091E61389831A82F2
:10C680002CE231E641E050E060E070E0CE0101963E
:10C6900087DE882319F089818093E6132296E2E0F1
:10C6A0000C941CF1A2E0B0E0E8E5F3E60C9400F194
:10C6B0000E9458B580EC90E00E943EDE22E0AC0182
:10C6C00060E080E00E9414B982E090E00E943EDECB
:10C6D00020E0AC0167E080E00E9414B98091011C69
:10C6E00089831A822DE630E64EE150E06AE070E080
:10C6F000CE01019655DE882319F089818093011CB3
:10C700002296E2E00C941CF197FF04C0A901461B9D
:10C71000570B02C0421B530BCA010895282F30E06B
:10C720002330310514F48F5F01C080E0F901E45734
:10C73000FD4F9081E82FF0E0E457FD4F8081DB0151
:10C74000A90FB11DA90FB11DFB01E80FF11DE80FE5
:10C75000F11D2D913C91808191818217930714F0F6
:10C7600081E008958FEF08950F93682F70E080E0C7
:10C7700090E000E020E044E044D320E0AC0162E03F
:10C7800080E10E9440B90F910895A6E0B0E0EBEC83
:10C79000F3E60C94F7F08091011C91D90E9458B5F2
:10C7A00081EC90E00E943EDE22E0AC0160E080E09F
:10C7B0000E9414B982E090E00E943EDE20E0AC01CD
:10C7C00067E080E00E9414B98091031CCDDF1A82DB
:10C7D000198204DA969587959C838B83FFD99E8373
:10C7E0008D838E010F5F1F4FB80180E097DFC82E49
:10C7F00080918C02F801E80FF11DE80FF11DE08037
:10C80000F180B090031CDD24D394A02E912E4BC058
:10C81000B7018091E61377DAED2DF0E0E457FD4F94
:10C820008081EA2DF92DE80FF11DE80FF11D00813F
:10C830001181E016F10621F14091021C5C2D540398
:10C84000900111242E0D3F1DC7FE04C02017310793
:10C8500044F005C0CC2019F00217130714F0411161
:10C8600089012091011C30E02F5F3F4F8091051C12
:10C87000A901480F511DCA010E948972780113C095
:10C880006A2D792D8D2D4ADFC82E52E05D1538F0C6
:10C89000D11003C0BA948B2D67DFD39401C0D12C83
:10C8A0008091041C45D480E10E949972882331F064
:10C8B000F89484E104D97894A0DA07C080E20E9459
:10C8C0009972882309F4A4CFF3CF2696EBE00C9459
:10C8D00013F1A2E0B0E0EFE6F4E60C94FFF08AEB8F
:10C8E00090E00E943EDE20E0AC0162E080E00E9429
:10C8F00014B982E090E00E943EDE20E0AC0167E0E7
:10C9000080E00E9414B984E1DAD8A091E61317E020
:10C910001A9FD0011124A051B44E8C9189831A82A0
:10C9200025E431E641E050E060E070E0CE010196A0
:10C9300037DD882351F08091E6136981189FF0015B
:10C940001124E051F44E608354D957DA2296E3E083
:10C950000C941BF10E9458B58091E613811103C01D
:10C9600088EB90E002C089EB90E00E943EDE22E07E
:10C97000AC0160E080E00C9414B9ECDFAACFA2E037
:10C98000B0E0E5ECF4E60C94FFF08BEB90E00E9455
:10C990003EDE20E0AC0162E080E00E9414B982E05B
:10C9A00090E00E943EDE20E0AC0167E080E00E9463
:10C9B00014B984E184D812D9BC018091E613A3D9BB
:10C9C000E091E61317E01E9FF0011124ED50F44EA4
:10C9D000808191819A838983E091FE1B8CE0E89F9E
:10C9E000F0011124E456FD4F468157816481758121
:10C9F0002DE730E6CE010196D3DC8823A1F08091AB
:10CA0000E613189F900111242F58344EF901EE5768
:10CA1000FF4F49815A8151834083F901EC57FF4F01
:10CA2000608171811BD9E9D92296E3E00C941BF156
:10CA300091DFA5CFA2E0B0E0E0E2F5E60C94FFF0D4
:10CA40008CEB90E00E943EDE20E0AC0162E080E0F2
:10CA50000E9414B982E090E00E943EDE20E0AC012A
:10CA600067E080E00E9414B984E129D860E070E0BA
:10CA70008091E61348D9E091E61317E01E9FF0017C
:10CA80001124EF50F44E808191819A838983E09143
:10CA9000FE1B8CE0E89FF0011124E456FD4F42811B
:10CAA00053816081718129EA30E6CE01019678DCFC
:10CAB0008823A1F08091E613189F900111242F582C
:10CAC000344EF901E058FF4F49815A815183408328
:10CAD000F901EC57FF4F60817181C0D88ED9229641
:10CAE000E3E00C941BF136DFA5CFA2E0B0E0EBE76A
:10CAF000F5E60C94FFF08DEB90E00E943EDE20E026
:10CB0000AC0162E080E00E9414B982E090E00E94F3
:10CB10003EDE20E0AC0167E080E00E9414B984E1D1
:10CB20000E945F5D5BD8BC01769567958091E613A6
:10CB3000EAD8A091E61317E01A9FD0011124AB5058
:10CB4000B44E8D919C919A838983E091FE1B8CE079
:10CB5000E89FF0011124E456FD4F4285538560851E
:10CB6000718526E430E6CE0101961ADC882359F05F
:10CB7000E091E6131E9FF0011124EB50F44E8981E1
:10CB80009A819183808339D92296E3E00C941BF13A
:10CB9000E1DEABCF0F931F93CF93DF93082FC1EF4D
:10CBA000DBE110E028813981011115C03695279508
:10CBB00036952795398328832A813B813695279599
:10CBC000369527953B832A832C813D813695279581
:10CBD0003695279516C0220F331F220F331F398336
:10CBE00028832A813B81220F331F220F331F3B836F
:10CBF0002A832C813D81220F331F220F331F2D5F8B
:10CC00003F4F3D832C8368817981812F0E94025E92
:10CC10006A817B81812F0DD86C817D81812F1ED807
:10CC20001F5F2796123009F0BDCFE7D8DF91CF9173
:10CC30001F910F910895A2E0B0E0E1E2F6E60C94B6
:10CC400000F10E9458B587EB90E00E943EDE22E0A2
:10CC5000AC0160E080E00E9414B987EB90E00E9494
:10CC60003EDE20E0AC0162E080E00E9414B982E088
:10CC700090E00E943EDE20E0AC0167E080E00E9490
:10CC800014B98091FE1B89831A8224E531E641E0C4
:10CC900050E060E070E0CE01019682DB882349F02D
:10CCA000F89489818093FE1B75DF84E10E945F5DAB
:10CCB00078942296E2E00C941CF1EF92FF920F938D
:10CCC0001F938093E6130E949C498FE398E00E9493
:10CCD000CA49E4E5EE2EE8E0FE2E87012CE438E0B8
:10CCE0004DEB54E661E081E00E94654BF7E6EF2EE4
:10CCF000F8E0FF2E02E618E02CE538E048E155E6C2
:10CD000061E082E00E94654BAAE7EA2EA8E0FA2ED5
:10CD100004E718E02DE638E043E755E661E083E0FC
:10CD20000E94654BBEE8EB2EB8E0FB2E07E818E04A
:10CD300021E838E048EC55E661E084E00E94654B6C
:10CD400080E00E943E4E0E94BD491F910F91FF90CE
:10CD5000EF900895EF92FF920F931F930E949C49CA
:10CD60008AEA99E00E94CA4918ECE12E19E0F12EF6
:10CD700087012AEB39E04BE156E661E081E00E9451
:10CD8000654B0CEDE02E09E0F02E870124ED39E033
:10CD900040E050E062E082E00E94654B8CEEE82EBD
:10CDA00089E0F82E870124EE39E040E050E062E0AF
:10CDB00083E00E94654B9EEFE92E99E0F92E8701F2
:10CDC00024EF39E047EA5FE562E084E00E94654BCA
:10CDD00080E00E943E4E0E94754A853059F00E94C4
:10CDE000884A823011F480E003C0833089F781E003
:10CDF00064DFEECF0E94BD491F910F91FF90EF902D
:10CE00000895A8E0B0E0E7E0F7E60C94F0F06B01DD
:10CE10007C01242E922EA42EB12CF501E050F84F67
:10CE200010820217A8F4E22FF0E0E01BF109EE0FE8
:10CE3000FF1FEE0FFF1FE85FF54F259135914591DC
:10CE40005491C701B6010E94D5F069017A01902E74
:10CE5000F7FE0BC0F094E094D094C094C11CD11C98
:10CE6000E11CF11C8824839401C0812C21E030E076
:10CE700005C02F5F3F4F2A30310591F0422FF90155
:10CE8000EE0FFF1FEE0FFF1FE85FF54F85919591A5
:10CE9000A591B491C816D906EA06FB0654F701C05D
:10CEA0004AE081104F5F91104F5F742E7218171473
:10CEB0000CF06EC0472C552447FC5094092D10E00F
:10CEC0004016510629F0C80101964816590621F569
:10CED000F801EE0FFF1FEE0FFF1FEC5FF54F2591DE
:10CEE000359145915491A5E0B0E00E9467F06C0D3A
:10CEF0007D1D8E1D9F1DF801EE0FFF1FEE0FFF1F02
:10CF0000E85FF54F25913591459154910E94D5F0F8
:10CF100069017A01912C3CC04016510624F5F201BA
:10CF2000EE0FFF1FEE0FFF1FEC5FF54F25913591C0
:10CF300045915491A5E0B0E00E9467F06C0D7D1D15
:10CF40008E1D9F1DF201EE0FFF1FEE0FFF1FE85F0A
:10CF5000F54F25913591459154910E94D5F0690185
:10CF60007A01971815C02A9480E090E0222D33278B
:10CF700027FD30952050384F5AE205C0F901E80FDF
:10CF8000F91F50830197422D480F47FFF7CF6EC01E
:10CF90002A9418861F82822D992787FD90959A835F
:10CFA0008983E82DF0E0FE83ED838C010050184F5B
:10CFB0008AE0482E512C612C712C2DC0EF81F88510
:10CFC000E00FF11F992059F0C501891991090197C6
:10CFD0002817390721F48CE28083912C17C0FC8339
:10CFE000EB83C701B601A30192010E94D5F0605DF9
:10CFF000EB81FC81608369017A01C114D104E104F1
:10D00000F10421F4911002C03A9412C08F819885E6
:10D01000019798878F833F80320C29813A81EF8175
:10D02000F8852E0F3F1F8D819E812817390734F612
:10D03000882049F0E32DFF27E7FDF095E050F84FF9
:10D040008DE280833A9480E090E0232D332727FD02
:10D0500030952050384F50E205C0F901E80FF91F14
:10D0600050830197432D480F47FFF7CF80E098E0AA
:10D070002896E2E10C940CF1CF92DF92EF92FF92AE
:10D080001F93CF93DF9300D0CDB7DEB76A017B014A
:10D090004AE050E0BE016F5F7F4F0E9466F29B0145
:10D0A000AC01E981FA8180818E3209F5319616C092
:10D0B000AAE0B0E00E9467F09B01AC01812F90E0F4
:10D0C000C097AA2797FDA095BA2F280F391F4A1F8E
:10D0D0005B1F81E0C81AD108E108F1081191112302
:10D0E00031F0C114D104E104F10411F715C0C114E9
:10D0F000D104E104F10481F0C601880F991F880F63
:10D10000991F885F954FFC01659175918591949168
:10D110000E9471F09B01AC01B901CA010F900F9000
:10D12000DF91CF911F91FF90EF90DF90CF90089506
:10D1300090E044EF51E009C028EE33E0FA01319766
:10D14000F1F721503109D1F79F5F9813F5CF08957A
:10D150004F925F926F927F928F929F92AF92BF9207
:10D16000CF92DF92EF92FF920F93CF93DF93CDB7E1
:10D17000DEB72E97DEBFCDBF4C015B01DC012D91E8
:10D180003D914D915C9113972F83388749875A873A
:10D190001496CD90DD90ED90FC901797DB012D91CA
:10D1A0003D914D915C9113972B873C874D875E870E
:10D1B00014964D905D906D907C90179780913408F7
:10D1C000811138C007E027E04AE0C701B60119DE47
:10D1D00020E0AC0163E080E00E9440B9F40160818E
:10D1E00071818281938127E04AE00BDE20E0AC016F
:10D1F00063E08BE00E9440B9D50114966D917D915A
:10D200008D919C91179727E04AE0FBDD20E0AC016F
:10D2100064E080E00E9440B9F50160817181828103
:10D22000938127E04AE0EDDD20E0AC0164E08BE093
:10D230000E9440B9C701B601640D751D861D971D7A
:10D2400020E03DE241E351E00E94D5F0C9010E9497
:10D250000B5C2FE435E0DC010E9461F04B015C01C6
:10D260006F81788589859A852B853C854D855E857E
:10D27000621B730B840B950B2AE030E040E050E01A
:10D280000E94D5F02F83388749875A87A5019401DA
:10D290006F81788589859A850E9471F020E836E94A
:10D2A00048E950E00E94D5F049015A01A7019601D2
:10D2B0002419350946095709A9E5B4E00E9467F029
:10D2C00020E137E240E050E00E94D5F029013A0128
:10D2D000C501B4010E94525C845E9D4F68E671E016
:10D2E0000E94A0F07C01A5019401C501B4010E9437
:10D2F00071F04B015C01A3019201C301B2010E94D4
:10D3000071F0860E971EA81EB91EC501B4010E94B9
:10D31000D85B4C01A12CB12C80913408811136C00E
:10D3200020E040E35AE065E00E9414B9B701882785
:10D3300077FD8095982F00E020E043E062DD20E05B
:10D34000AC0165E085E00E9440B920E046E35AE088
:10D3500065E088E00E9414B920E048E35AE065E007
:10D3600089E00E9414B901E021E043E0C501B40165
:10D3700048DD20E0AC0165E08FE00E9440B920E08C
:10D380004EE35AE065E084E10E9414B989829A82F2
:10D39000AB82BC82FE82ED82282D3A814B815C817A
:10D3A0006E2D7E8180E090E02E96DEBFCDBFDF91B6
:10D3B000CF910F91FF90EF90DF90CF90BF90AF9003
:10D3C0009F908F907F906F905F904F9008958F9275
:10D3D0009F92AF92BF92CF92DF92EF92FF920F9304
:10D3E000CF93DF93CDB7DEB72697DEBFCDBF6FEE0D
:10D3F00073E183E094E1ACDE29833A834B835C8361
:10D400006D837E8386E0FE013196ADEFB3E101903E
:10D410000D928A95E1F7C090FD13D090FE13E09035
:10D42000FF13F09000146091F7137091F81380913E
:10D43000F9139091FA1380900B1490900C14A09013
:10D440000D14B0900E14681979098A099B0924E615
:10D4500030E040E050E00E94D5F049015A01A701B8
:10D460009601C501B4010E94525C909318148093F8
:10D4700017148091FD139091FE13A091FF13B091AA
:10D48000001488329105A105B10544F0CC97A1059F
:10D49000B1056CF580910F08882349F180910F1434
:10D4A0009091101490930214809301148091F713BB
:10D4B0009091F813A091F913B091FA1340910B14C5
:10D4C00050910C1460910D1470910E14841B950BE7
:10D4D000A60BB70B803A9F40A105B10524F410922A
:10D4E00018141092171481E080930F0802C0109254
:10D4F0000F0880910114909102148E539E4F209139
:10D500000F1430911014821B930B68E671E00E9497
:10D51000A0F0909316148093151420911714309155
:10D52000181437FF04C01092181410921714209189
:10D53000171430911814253B310534F024EB30E0FA
:10D540003093181420931714843B910594F0845B56
:10D550009109909316148093151484EB90E0209118
:10D56000171430911814821B930B90931814809306
:10D570001714609115147091161480E00E941A5FC0
:10D58000609117147091181481E00E941A5F8091C5
:10D590003408811123C020E040E45AE066E00E9494
:10D5A00014B94091151450911614E12C01E023E0B8
:10D5B00030E066E086E00E94EBBE20E046E45AE000
:10D5C00066E08BE00E9414B9409117145091181432
:10D5D00023E030E066E081E10E94EBBE2696DEBFEC
:10D5E000CDBFDF91CF910F91FF90EF90DF90CF9063
:10D5F000BF90AF909F908F900895A1E0B0E0E3E0DE
:10D60000FBE60C94F0F011E01093FC1322E04BEDDC
:10D610005AE062E080E00E9414B944E161E080E0F9
:10D620000E949EB90E94355B8FE480937E0A198226
:10D630001F921F93EE24E394F12CEC0EFD1EFF923B
:10D64000EF921F931F9284E68F930E94CD598AE038
:10D6500089831F921F93FF92EF921F9382E08F9313
:10D660008FE68F930E94CD5988EC90E0909323141D
:10D6700080932214909325148093241410923E08D2
:10D68000DEBFCDBF712CD12C08EC10E09AE0692EE2
:10D690003E2C2F2C22E0522E3FE6432E8091B707DE
:10D6A000882309F4F1C010932314009322140E94DC
:10D6B000D95A8091B4079091B50790931A1480932A
:10D6C000191441E061E082E10E9433A591E0D91292
:10D6D00004C061E080E00E9472A5809119149091CD
:10D6E0001A14FC01EC5BFF4F208127FD15C17394D8
:10D6F000E2E37E1691F0F9E17F1204C022E041EFEF
:10D700005AE006C081E0781209C020E044E05BE006
:10D7100061E080E00E9414B901C0712C1092B7073B
:10D72000D12C9BC0FC01ED5BFF4F208123FF37C054
:10D73000FC01478D50A161A172A140930314509345
:10D740000414609305147093061443A154A165A1B9
:10D7500076A14093071450930814609309147093B2
:10D760000A1447A150A561A572A540930B145093CC
:10D770000C1460930D1470930E1486AD97AD9093B6
:10D78000101480930F141092FC131092B70720E02E
:10D7900047E15BE061E080E00E9414B95CC020E0FA
:10D7A0004AE25BE061E080E00E9414B952C0FC01F3
:10D7B0003196AFEEB3E12DE001900D922A95E1F79D
:10D7C000FC01A3A8B4A860910B1470910C14809173
:10D7D0000D1490910E140E9480EE6B017C0120EAE2
:10D7E0003FE0D5010E9461F00E9480EE20E030E031
:10D7F00044EB51E40E94E5ED4B015C016091F713AD
:10D800007091F8138091F9139091FA130E9480EEB1
:10D810009B01AC01C501B4010E947AEDA7019601FC
:10D820000E9479ED20E030E040EA50E40E94E5ED0E
:10D830009B01AC01C701B6010E947AED0E944DEE3A
:10D840006093F7137093F8138093F9139093FA137E
:10D85000BEDD1092B707DD24D394809124149091FB
:10D860002514892B89F469821F9281E08F932F926E
:10D870003F928F935F924F920E94CD59109325143F
:10D8800000932414DEBFCDBF809122149091231405
:10D89000892B31F481E00E94879781E080933E08D4
:10D8A00080E147D6811105C080913E08882309F4A4
:10D8B000F5CE45E161E080E00E949EB945E162E07D
:10D8C00080E00E949EB945E163E080E00E949EB93D
:10D8D00045E164E080E00E949EB945E165E080E0BA
:10D8E0000E949EB945E166E080E00E949EB9809169
:10D8F0003E088130B1F420E04DE35BE062E080E07F
:10D900000E9414B980E29EE424EF31E0F9013197DE
:10D91000F1F70197D9F705C02091FC13211102CF2F
:10D9200046CF81E02196E2E10C940CF18F929F9218
:10D93000AF92BF92CF92DF92EF92FF92CF93DF939D
:10D94000EB01FC01C080FAE0CF9E6001112420EEC3
:10D95000C21A21E0D20AFC012181C20ED11CF0E3DF
:10D96000CF1AD108EE24D7FCE094FE2C46E050E01C
:10D9700060E070E0029680DB4B015C01A70196013C
:10D9800060E876E988E990E00E9471F06B017C0123
:10D99000C501B40126E030E040E050E00E94D5F03F
:10D9A000C20ED31EE41EF51E8881833541F4F09427
:10D9B000E094D094C094C11CD11CE11CF11CB601B0
:10D9C000C701DF91CF91FF90EF90DF90CF90BF9094
:10D9D000AF909F908F9008958F929F92AF92BF9239
:10D9E000CF92DF92EF92FF92CF93DF93EB01FC0196
:10D9F0002081FAE02F9F90011124205E3140FC012C
:10DA00004181240F311D4AE0429F6001439FD00CA9
:10DA10001124F0EECF1AF1E0DF0AFC012281C20EE0
:10DA2000D11CF0E3CF1AD108EE24D7FCE094FE2CF1
:10DA300046E050E060E070E003961EDB4B015C01C5
:10DA4000A701960160E876E988E990E00E9471F00C
:10DA50006B017C01C501B40126E030E040E050E0FC
:10DA60000E94D5F0C20ED31EE41EF51E88818735B4
:10DA700041F4F094E094D094C094C11CD11CE11CFA
:10DA8000F11CB601C701DF91CF91FF90EF90DF90BD
:10DA9000CF90BF90AF909F908F900895FC0180E051
:10DAA00090E02AE301C09A2F3191A92FB0E0AD5F39
:10DAB000BE4F3C93A92FAF5F813011F0833031F41A
:10DAC000B0E0AD5FBE4F2C93A92FAE5F8F5F863065
:10DAD00051F7EA2FF0E0ED5FFE4F10820895982F86
:10DAE00080538A3058F08153863008F404C0892F5F
:10DAF0008154863010F4865F089580E00895EF9297
:10DB0000FF920F931F93CF93DF9380917008813022
:10DB1000D9F580912726811104C037C0F826CF5F40
:10DB200002C0C1E0F12C80912726C81758F0D0E040
:10DB30008E010E5F1F4F8091272690E0081719076E
:10DB40004CF022C0EC2FF0E0EF58FC4D80818A327F
:10DB500029F7EDCFCF58DC4D8981C1DFE82EF801E0
:10DB6000EF58FC4D8081BBDF90E1E99E90011124CC
:10DB7000822B8F1109C0188262E773E289ED92E26D
:10DB80000E940EF481E001C080E010927008CDB7D1
:10DB9000DEB7E6E00C9418F10F931F93B0DF8823F3
:10DBA00009F4AEC066ED72E089ED92E20E94F0F3F6
:10DBB00068ED72E00E9405F4009709F0A1C06EEDD7
:10DBC00072E080E090E00E94F0F368DF66ED72E0C2
:10DBD00080E090E00E94F0F366ED72E080E090E07B
:10DBE0000E94F0F38C0166ED72E080E090E00E940C
:10DBF000F0F3BC01C8019ADE6093E7137093E81359
:10DC00008093E9139093EA1366ED72E080E090E070
:10DC10000E94F0F38C0166ED72E080E090E00E94DB
:10DC2000F0F3BC01C801D8DE609311147093121494
:10DC3000809313149093141466ED72E080E090E0EA
:10DC40000E94F0F30E9490F38093EB1366ED72E074
:10DC500080E090E00E94F0F30E9490F38093EC1338
:10DC600066ED72E080E090E00E94F0F341E050E069
:10DC700060E070E001DA70931C1460931B1466ED91
:10DC800072E080E090E00E94F0F341E050E060E05C
:10DC900070E0F2D970931E1460931D14009111145A
:10DCA0001091121420911314309114140093031442
:10DCB0001093041420930514309306140091E71375
:10DCC0001091E8132091E9133091EA13009307149F
:10DCD000109308142093091430930A14CB01AA2737
:10DCE00097FDA095BA2F80930B1490930C14A093DA
:10DCF0000D14B0930E141092101410920F1467DBD1
:10DD00001F910F910895A1E0B0E0E9E8FEE60C94C0
:10DD1000F5F081E08093FC1320E04AEA5BE161E0EA
:10DD200080E00E9440B982E00E94DBD08091851B98
:10DD3000813011F40E947FCE20E04CE45AE061E093
:10DD400082E10E9414B98EEB9BE10E9459CB182FFF
:10DD5000813051F420E041E55AE061E082E10E9427
:10DD600014B91093680307C022E046E55AE061E069
:10DD700081E10E9414B9F090680381E0F8121AC1A1
:10DD800022E04BE55AE062E080E00E9414B944E1F1
:10DD900061E080E00E949EB920E041E75AE063E044
:10DDA00080E00E9414B920E043E75AE064E080E09C
:10DDB0000E9414B9109270080E94355B8FE4809322
:10DDC0007E0A19821F92FF928E010F5F1F4F1F93D1
:10DDD0000F93FF921F9284E68F930E94CD598AE0A1
:10DDE00089831F92FF921F930F93FF9282E08F937C
:10DDF0008FE68F930E94CD5988EC90E09093231486
:10DE0000809322149093251480932414DEBFCDBFF9
:10DE100048ECC42ED12C5DE0B52E6AE0A62EFF247E
:10DE2000F394802E712E12E07FE6972E0E9417CF7A
:10DE3000811123C045E161E080E00E949EB945E187
:10DE400062E080E00E949EB945E163E080E00E94CC
:10DE50009EB945E164E080E00E949EB945E165E03D
:10DE600080E00E949EB945E166E080E00E949EB994
:10DE700080916803811196C08EC08091B707882376
:10DE800009F46EC0D0922314C09222140E94D95A71
:10DE9000E091B407F091B507F0931A14E0931914C8
:10DEA0003196AFEEB3E18B2D01900D928A95E1F79B
:10DEB00073DE8091340881113BC022E043E051E0E1
:10DEC00060E08DE00E9440B920E045E75AE061E063
:10DED00080E10E9414B94091EC13E12C01E022E0B2
:10DEE00030E050E061E083E10E94EBBE20E04AE7D1
:10DEF0005AE061E080E00E9414B94091EB1321E008
:10DF000030E050E061E084E00E94EBBE20E04FE7AB
:10DF10005AE061E086E00E9414B940911B145091D0
:10DF20001C1400E023E030E061E08BE00E945DBF64
:10DF30001092B7078091241490912514892B81F4B5
:10DF4000A9821F92FF927F928F92FF921F939F92BE
:10DF50000E94CD59D0922514C0922414DEBFCDBFAB
:10DF60008091221490912314892B29F480E00E943F
:10DF70008797F0923E0880E1DCD2882309F456CFDF
:10DF800080916803882309F451CF80913E08813045
:10DF900009F44CCF4FCF20E045E85AE062E080E042
:10DFA0000E9414B920E042E95AE063E080E00E9458
:10DFB00014B912C020E04EE95AE064E080E00E940B
:10DFC00014B920E042EB5AE065E080E00E9414B909
:10DFD00080E1AFD28823E1F3109268030E9418CB4E
:10DFE000892B39F420E047EC5AE063E080E00E949E
:10DFF00014B981E00E94DBD081E02196EDE00C9421
:10E0000011F180EF96D20E9458B58091CD1B8111FD
:10E0100006C022E04EE45BE060E00E9414B980910B
:10E02000CD1B813039F422E044E65BE060E080E023
:10E030000E9414B920E04AE75BE067E080E10E94BB
:10E0400014B98091CD1B811101C05DDE8091CD1B83
:10E05000813009F4D2DA80EF6CC21092231410924E
:10E06000221482E084BD85E085BD83EC87BDEEE6A9
:10E07000F0E080818260808308951F920F920FB636
:10E080000F9211245F9A0F900FBE0F901F9018955A
:10E090001F920F920FB60F9211245F980F900FBE30
:10E0A0000F901F9018958091ED1B8130A1F4109274
:10E0B000B0001092B6001092B2008FEF8093B300C0
:10E0C0008091B000836C8093B0008091B10081603A
:10E0D0008093B1000895579A8091B000836880932F
:10E0E000B0008091B10081608093B1008091700098
:10E0F0008660809370008FEF8093B3000895E0E90D
:10E10000F0E0108288EF809395001092940087E0F1
:10E11000809399008FEF8093980080818260808344
:10E12000E1E9F0E0808181608083E1E7F0E08081D7
:10E130008260808308951F920F920FB60F92112470
:10E140000BB60F922F933F934F935F936F937F93F1
:10E150008F939F93AF93BF93EF93FF9340912408C6
:10E1600080B18095842790912B0898239095909367
:10E170002B0820912C082823292720932C08392F9D
:10E1800038233223832F842780932408982F9323C6
:10E1900080912308892B8093230880912D08882360
:10E1A00021F0815080932D0811C089E080932D08C3
:10E1B0008091100890911108019690931108809316
:10E1C0001008809113018F5F80931301332389F02E
:10E1D00080912114811102C00E94C5D081E08093FA
:10E1E000211410921D0810921C0810921B08109206
:10E1F0001A082091731B2223D1F0809121148130C1
:10E20000B1F480911C0890911D08019690931D080F
:10E2100080931C0864E670E00E948CF0822F90E0EE
:10E220006817790721F40E94D0D0109221148091B0
:10E23000EE1B813061F580911408909115080097CC
:10E24000D9F08B30910530F00A97909315088093A0
:10E25000140804C0109215081092140880910D0142
:10E2600090910E0120911408309115088223932378
:10E27000892B09F020C122C18FEF9FEF90930E01EF
:10E2800080930D01109213081092120817C180910B
:10E290002408982F907F19F426E420932E082091CB
:10E2A0002E08215020932E08211107C0382F307FCF
:10E2B00020912208232B20932208911103C021E0F2
:10E2C00020932F0820912F08215019F020932F0818
:10E2D0000AC02FE020932F08382F307F209121088B
:10E2E000232B20932108911103C026E420933008AA
:10E2F00020913008215019F0209330080AC02FE0F7
:10E3000020933008382F307F20912008232B209332
:10E310002008911103C096E4909331089091310840
:10E32000915090933108911115C090911E08913031
:10E3300011F494E107C0923011F498E003C09330D7
:10E3400049F491E090933108807F90911F08982BB9
:10E3500090931F088091221490912314892B49F0E7
:10E360008091221490912314019790932314809309
:10E37000221480912E1490912F14892B49F08091B2
:10E380002E1490912F14019790932F1480932E1494
:10E390008091321490913314892B49F0809132147A
:10E3A0009091331401979093331480933214809199
:10E3B0003B1490913C14892B49F080913B1490912F
:10E3C0003C14019790933C1480933B1480913F142C
:10E3D00090914014892B49F080913F149091401402
:10E3E00001979093401480933F1480913914909139
:10E3F0003A14892B49F08091391490913A1401977D
:10E4000090933A1480933914809130149091311480
:10E41000892B49F080913014909131140197909399
:10E420003114809330148091241490912514892BF9
:10E4300049F080912414909125140197909325140C
:10E44000809324148091250890912608A091270894
:10E45000B09128080196A11DB11D809325089093C5
:10E460002608A0932708B09328086091250870918A
:10E470002608809127089091280824E630E040E0A3
:10E4800050E00E94B3F0672B682B692BD1F4809188
:10E49000261490912714A0912814B0912914019664
:10E4A000A11DB11D8093261490932714A0932814C6
:10E4B000B093291406C00E94AFD0E9CE0E94BAD012
:10E4C000E6CEFF91EF91BF91AF919F918F917F9198
:10E4D0006F915F914F913F912F910F900BBE0F90D5
:10E4E0000FBE0F901F9018952091100830911108C1
:10E4F0002F5F3F4F280F391FC90108952091100841
:10E5000030911108821B930B88279078892F86956C
:10E510000895CF93DF93C0911008D09111082196F0
:10E52000C80FD91FCE01EADF8823E1F3DF91CF9135
:10E5300008952FB7F89490912308892398279093F2
:10E5400023082FBF0895CF93CFB7F8949091240854
:10E5500090958923EEDFCFBFCF9108952FB7F89420
:10E560009091210889239827909321082FBF08951F
:10E570002FB7F89490912208892398279093220826
:10E580002FBFECDFD6CF2FB7F894909120088923C6
:10E590009827909320082FBF909123089095892762
:10E5A000DDCF2FB7F89490911F0889239827909377
:10E5B0001F0860931E082FBF08952091EE1B213085
:10E5C00071F5411107C02091120830911308232BD7
:10E5D00031F50EC04130A9F4209112083091130892
:10E5E000232BE9F421E030E0309313082093120844
:10E5F000909315088093140870930E0160930D0199
:10E600000895423061F4109213081092120810928B
:10E6100015081092140810920E0110920D01089521
:10E620008091160890911708019769F440E060E224
:10E6300070E088EE93E0C1DF22E04FE75BE060E04E
:10E6400080E00E9414B9209116083091170840917B
:10E6500011015091120164E6649FC001659F900D05
:10E6600011242817390721F4109217081092160860
:10E670008091160890911708892B49F0809116080F
:10E680009091170801969093170880931608349B71
:10E6900004C0109219081092180834991BC0809178
:10E6A00018089091190801969093190880931808FA
:10E6B00080911808909119080A9761F480911608C2
:10E6C00090911708892B31F481E090E0909317081E
:10E6D00080931608209118083091190840910F0175
:10E6E0005091100164E6649FC001659F900D112454
:10E6F0002817390709F4299808958CE0E7EFF2E12B
:10E70000DF011D928A95E9F7E1E4F4E1A7EFB2E1B8
:10E710008081329686598D9384E1EB34F807C1F7F6
:10E720001F928CE08F9387EF92E19F938F9381E00C
:10E730008F938F9389E78F930E94CD59ADB7BEB762
:10E740001796BEBFADBF0895EF92FF920F931F9330
:10E75000CF93DF938091320890E0880F991FFC01DE
:10E76000EF5BFB4E20813181FC01E75AFB4E0081BB
:10E770001181021713070CF044C0063911050CF083
:10E7800040C046E9E42EF12CB701621B730B8827C9
:10E7900077FD8095982F0E9480EE20E030E040E0E9
:10E7A0005FE30E946DEF9B01AC0160E070E08CE7DD
:10E7B00092E40E9479ED0E9452EED62FC091330868
:10E7C000CF5FB701601B710B882777FD8095982F6D
:10E7D0000E9480EE20E030E040E05FE30E946DEFB9
:10E7E0009B01AC0160E070E08CE792E40E9479ED5F
:10E7F0000E9452EE862F00E024E04D2F6C2F0E94E5
:10E800007BB78091320890E0880F991FFC01EF5B85
:10E81000FB4EC081D181FC01E75AFB4E60817181C2
:10E82000C617D707DCF567397105C4F16659710958
:10E83000882777FD8095982F0E9480EE20E030E0B9
:10E8400040E05FE30E946DEF20E030E04CE752E4EF
:10E850000E947AED0E9452EEF62E109133081F5F4F
:10E86000BE0166597109882777FD8095982F0E940F
:10E8700080EE20E030E040E05FE30E946DEF20E0BA
:10E8800030E04CE752E40E947AED0E9452EE862F6F
:10E8900000E024E04F2D612F0E947BB7E091320809
:10E8A000F0E0EE0FFF1FEF5BFB4E80819181863918
:10E8B0009105CCF0BC0166597109882777FD8095D8
:10E8C000982F0E9480EE20E030E040E05FE30E945D
:10E8D0006DEF0E9452EE462F609133086F5F01E0AA
:10E8E00024E08FE32DC066E970E0681B790B882770
:10E8F00077FD8095982F0E9480EE20E030E040E088
:10E900005FE30E946DEFF62E072F182FD92F812F6E
:10E910000E9452EEE62EC0913308CF5F6F2D702F0C
:10E920009B01412F5D2F60E070E08CE792E40E9434
:10E9300079ED0E9452EE862F01E024E04E2D6C2FDF
:10E940000E947BB726E042E0609133088EE30E948C
:10E950007BB760913308262F2A5F01E043E083E014
:10E960000E94CBB660913308262F2A5F47E187E1EA
:10E970000E94CBB660913308262F2A5F4BE28BE2D0
:10E980000E94CBB660913308262F2A5F43E583E5CA
:10E990000E94CBB660913308262F2A5F47E687E6B0
:10E9A0000E94CBB660913308262F2A5F4BE78BE796
:10E9B0000E94CBB6CDB7DEB7E6E00C9418F1A4E127
:10E9C000B0E0E5EEF4E70C94F0F086E996E9A6E90C
:10E9D0008093411490934214A0934314FE013B96FC
:10E9E00085E0DF011D928A95E9F780911D1C811158
:10E9F00003C01098089802C0109A089A80912C1CA5
:10EA0000811109C080911E1C811103C011980998C1
:10EA100002C0119A099A80911F1C811103C012989B
:10EA20000A9802C0129A0A9A8091201C811103C090
:10EA300013980B9802C0139A0B9AFE013196A0E02E
:10EA4000B0E462E370E017EC24E930E04CE650E01B
:10EA5000B0937C0080917C00807E8A2B80937C0028
:10EA600070932314609322148091221490912314A4
:10EA7000892BD1F710937A0080917A0086FDFCCF24
:10EA800080917800909179009695879596958795D5
:10EA900099278D3691051CF45183408308C0843931
:10EAA00091051CF49183808302C03183208380917F
:10EAB0007C00807E8A2B80937C0080917A00806429
:10EAC00080937A0080917A0086FDFCCF8091780057
:10EAD00090917900969587959695879599278D368B
:10EAE00091051CF45183408308C0843991051CF4BE
:10EAF0009183808302C031832083AF5F3296A4303C
:10EB000009F0A6CF80917C00807E80937C0080916C
:10EB10007A00806480937A000E9458B562E085E9AB
:10EB20009BE00E941FB983E090E00E943EDE20E05F
:10EB3000AC0167E080E00E9414B920E04AEA5BE0A3
:10EB400067E082E10E9414B91CE01093330801E0F1
:10EB500026E048E7612F83E00E94BDB96091330849
:10EB6000262F2A5F47E187E10E94CBB660913308E8
:10EB7000262F2A5F4BE28BE20E94CBB626E042E0D2
:10EB8000609133088EE30E947BB760913308262F93
:10EB90002A5F43E583E50E94CBB660913308262FB8
:10EBA0002A5F47E687E60E94CBB6185F143369F602
:10EBB00086E990E090934214809341141C861B8652
:10EBC0009093461480934514188A1F8690934A1494
:10EBD000809349141C8A1B8AB12CAA24AA94442429
:10EBE0004394512C612CACE37A2E812CB4EC9B2EF7
:10EBF00018E7E12EF12C08E8C02EDD24DA9406E9AE
:10EC000010E08CE1282E80917A0086FD21C18B2DA9
:10EC100090E0FC01EE5DF34E2081AC01440F551FE6
:10EC20002223C1F02091780030917900FA01EF5B46
:10EC3000FB4EA1E0B0E0AC0FBD1FA40FB51F369591
:10EC40002795369527954D915C91421B510951832B
:10EC5000408318C02091780030917900FA01EF5B71
:10EC6000FB4E36952795369527953327A1E0B0E0E2
:10EC7000AC0FBD1FA40FB51F4D915C91241B350B2C
:10EC8000318320839C01220F331FF901EF5BFB4E80
:10EC9000408151814938BFEF5B071CF4D182C082AB
:10ECA00005C04837510514F0F182E082FC01E95DAE
:10ECB000F34E4081411162C0F901EF5BFB4E408190
:10ECC000518157FF02C0495F5F4FF3E0559547956B
:10ECD000FA95E1F7BC01660F771FA1E0B0E0AC0F39
:10ECE000BD1FA60FB71FFA0157FF04C0EE27FF276D
:10ECF000E41BF50B4E9F90014F9F300D5E9F300D32
:10ED000011241A964D915C911B97240F351FAC016D
:10ED1000440F551F2130E4EC3E074CF4E1E0F0E0F5
:10ED2000EC0FFD1FE60FF71F938682860FC0E1E010
:10ED3000F0E0EC0FFD1FE40FF51F21156CE3360723
:10ED40001CF43387228702C073866286FA01EF5B68
:10ED5000FB4EA1E0B0E0AC0FBD1FA40FB51F1A968B
:10ED60002C911A971B963C9137FF02C021583F4FB8
:10ED7000220F232F221F330B318320839C01220F6C
:10ED8000331FF901EF5BFB4E408151814A565F4FC3
:10ED900051834083D901A75FB34E6D917C91641775
:10EDA000750708F00AC0DC01AA0FBB1FAD5EB34EA9
:10EDB0006D917C914617570710F071836083F901BC
:10EDC000EF5BFB4ED901A75ABB4E408151812D917B
:10EDD0003C914217530739F0D20102C0AA0FBB1F62
:10EDE0008A95E2F7AA2AB394B3E0BB1224C08091BB
:10EDF000251C882319F0039B03C007C0039B05C093
:10EE00008091191C90911A1C04C080910F1C909144
:10EE1000101C90934814809347142091471430910C
:10EE2000481480915F14909160142817390711F0ED
:10EE3000E8E0AE2AB12C90917C008B2D8F71907EF2
:10EE4000892B80937C0080917A00806480937A0083
:10EE500080E46FDB382E63E080E4A3DB8329C9F113
:10EE600080912B1C2091261C811121C08091491476
:10EE700090914A14211102C0019601C0019790930C
:10EE80004A14809349142091491430914A14809176
:10EE9000111C9091121C8217930708F013C08091E7
:10EEA0001B1C90911C1C2817390780F00BC02111E6
:10EEB00005C080911B1C90911C1C04C08091111CEA
:10EEC0009091121C90934A148093491420E1A22A35
:10EED00040C080E82EDB382E63E080E862DB8329C7
:10EEE000C1F180912B1C2091261C811121C08091A1
:10EEF000491490914A14211102C0019701C0019652
:10EF000090934A14809349142091491430914A14E3
:10EF10008091111C9091121C8217930708F013C066
:10EF200080911B1C90911C1C2817390780F00BC086
:10EF3000211105C08091111C9091121C04C0809178
:10EF40001B1C90911C1C90934A148093491430E12F
:10EF5000A32A80912B1C882389F0809149149091D9
:10EF60004A148639910551F0069B08C0079B06C0DC
:10EF700010934A140093491460E1A62A80E1D9DA7B
:10EF80008823F9F010934214009341141C861B86C9
:10EF90001093461400934514188A1F8610934A1440
:10EFA000009349141C8A1B8A88EC90E09093150802
:10EFB0008093140880E890E090930E0180930D01F7
:10EFC00003C0AA2009F471C08CE08093330810922A
:10EFD0003208BADB8091320890E0880F991FFC015B
:10EFE000E75AFB4EDC01AF5BBB4E8D919C91918348
:10EFF0008083A4E1A0933308B1E0B09332088091FC
:10F000002C1C811101C0A0DB8091320890E0880F98
:10F01000991FFC01E75AFB4EDC01AF5BBB4E8D91A3
:10F020009C919183808320923308E2E0E093320840
:10F030008BDB8091320890E0880F991FFC01E75A22
:10F04000FB4EDC01AF5BBB4E8D919C919183808325
:10F0500084E28093330883E08093320875DB8091EB
:10F06000320890E0880F991FFC01E75AFB4EDC0143
:10F07000AF5BBB4E8D919C91918380838CE280939A
:10F08000330884E0809332085FDB8091320890E09F
:10F09000880F991FFC01E75AFB4EDC01AF5BBB4EAA
:10F0A0008D919C919183808328DB80E242DAA12CB0
:10F0B000882309F4A8CD80EF3CDA80912C1C8130A4
:10F0C00011F40E94E4B36496E2E10C940CF1A0E028
:10F0D000B0E0EDE6F8E70C94F2F00E9458B522E0BB
:10F0E0004EEA5BE060E080E00E9497B920E044ECEB
:10F0F0005BE061E080E00E9497B9C9E0DCE183E178
:10F10000C82E8CE1D82E9DE1A92E9CE1B92E27E2D4
:10F11000822E2CE1922E32E2632E3CE1732E80E0AF
:10F1200090E02C012FEF421A520AF82E182F1E5F82
:10F13000E12C00E021E030E0A201612F80E00E949C
:10F14000EBBE4991599123E030E0612F82E00E94AB
:10F15000EBBEF601419151916F0123E030E0612F48
:10F1600086E00E94EBBEF50181915F0120E08111F4
:10F1700003C04AED5BE002C04FED5BE0612F8AE027
:10F180000E9497B9F30181913F0120E0811103C0F2
:10F1900044EE5BE002C049EE5BE0612F8FE00E942D
:10F1A00097B9F40181914F0120E0811103C04DEE28
:10F1B0005BE002C04FEE5BE0612F84E10E9497B9F3
:10F1C000F1E0FF120BC080912C1C813039F420E05B
:10F1D00041EF5BE0612F83E00E9497B9C201853067
:10F1E000910509F09ECF20E044E05CE067E082E119
:10F1F0000E9414B980E19DD98823E1F3CDB7DEB731
:10F20000E0E10C940EF1A0E0B0E0E9E0F9E70C9445
:10F21000F4F0C82E0E949C4987E09CE00E94CA49F5
:10F220004BE2E42E4CE0F42E0DE11CE020E13CE04A
:10F2300040E050E061E081E00E94654B54E5E52E3E
:10F240005CE0F52E06E41CE029E33CE040E050E001
:10F2500061E082E00E94654B67E6E62E6CE0F62EE8
:10F26000870122E63CE040E050E061E083E00E945C
:10F27000654B7FE7E72E7CE0F72E05E71CE02CE6E8
:10F280003CE040E050E061E084E00E94654BE4EA4D
:10F29000EE2EECE0FE2E07E91CE028E83CE040E022
:10F2A00050E061E085E00E94654B8C2D90E09C0170
:10F2B0002F58344E590146EBA40EB11C4901E1EB25
:10F2C0008E0E911C3901FCEA6F0E711CEC01CC0F03
:10F2D000DD1FCD5ED34E6C01CC0CDD1C89E09CE1C2
:10F2E000C80ED91E80E00E943E4E0E94754A8530AD
:10F2F00009F456C00E94884A813081F4EE24E394D8
:10F3000000E029EC4CE251E060E070E0F601808121
:10F3100091810BD5F60191838083E4CF823071F423
:10F32000EE24E39400E02AEC4CE251E060E070E06F
:10F3300088819981FAD499838883D4CF833071F4FA
:10F34000EE24E3940DE02CEC41E050E060E070E04E
:10F35000F301808190E0E9D4F30120C0843071F49E
:10F36000EE24E39409E02BEC41E050E060E070E033
:10F37000F401808190E0D9D4F40110C0853009F007
:10F38000B1CFEE24E39407E02DEC41E050E060E0E3
:10F3900070E0F501808190E0C8D4F5018083A2CFB0
:10F3A0000E94BD49CDB7DEB7EEE00C9410F1EF92AC
:10F3B000FF920F931F93CF93DF930E949C4983EB9F
:10F3C0009CE00E94CA49BDECEB2EBCE0FB2E8701FD
:10F3D00023EC3CE040E050E061E081E00E94654BBE
:10F3E000CDEDEC2ECCE0FC2E870125ED3CE040E09D
:10F3F00050E062E082E00E94654BDDEEED2EDCE045
:10F40000FD2E870125EE3CE040E050E062E083E025
:10F410000E94654B1DEFE12E1CE0F12E870125EFC8
:10F420003CE040E050E062E084E00E94654B0DE08B
:10F43000E02E0DE0F02E870125E03DE040E050E0B9
:10F4400062E085E00E94654B8DE1E82E8DE0F82EAC
:10F45000870125E13DE040E050E062E086E00E9467
:10F46000654B97E4E92E9DE0F92E05E31DE025E2CA
:10F470003DE040E050E061E087E00E94654BC4EF72
:10F48000D1E080E00E943E4E0E94754A853009F42A
:10F4900045C00E94884A813011F419DEF2CF8230D3
:10F4A00011F480E027C08330D1F480912C1C81308E
:10F4B000A1F40E9458B58EEC90E00E943EDE22E05E
:10F4C000AC0163E080E00E9414B980E197E2FE01A4
:10F4D0003197F1F70197D9F7D4CF81E00BC0843091
:10F4E00011F482E007C0853011F483E003C0863058
:10F4F00019F484E088DEC5CF873009F0C2CFEE244E
:10F50000E39407E02EEC41E050E060E070E0809191
:10F510002C1C90E00AD480932C1CB3CF0E94BD49D0
:10F52000CDB7DEB7E6E00C9418F10E9458B580EF35
:10F5300000D887E490E00E943EDE20E0AC0162E06B
:10F5400080E00E9414B988E490E00E943EDE20E052
:10F55000AC0163E080E00E9414B986E490E00E9470
:10F560003EDE20E0AC0167E08CE00E9414B980E14F
:10F570000E949972882321F00E948EC429980895D0
:10F5800080E20E949972882391F380EF0C94997223
:10F5900040E06FEF7FEF8CE390E00FD820E047E58D
:10F5A0005DE067E083E10E9414B902C00E94BF8D54
:10F5B00080E10E9499728823C9F380EF0C949972BC
:10F5C0001F93CF93DF930E9458B583E890E00E9489
:10F5D0003EDE22E0AC0160E080E00E9414B920E051
:10F5E00041E75DE061E080E00E9414B920E049E776
:10F5F0005DE064E080E00E9414B920E04AEA5BE14B
:10F6000062E080E00E9440B9CEEBDBE110E049917E
:10F6100020E065E0812F0E9448B91F5F1C30B9F7D8
:10F62000B7DFDF91CF911F9108958091821B8111E7
:10F6300013C00E9458B522E04AE55DE060E080E03A
:10F640000E9414B922E046E65DE061E080E00E949D
:10F6500014B99EDF80E0089581E00895CF92EF9283
:10F660000F93CF93E2DF882309F43EC18091C31B3F
:10F67000803321F08091C41B8033D1F40E9458B5AF
:10F6800022E046EE5DE060E080E00E9414B922E0F6
:10F6900045EF5DE061E080E00E9414B980E29EE405
:10F6A00024EF31E0F9013197F1F70197D9F71CC147
:10F6B0000E9458B58AEA9BE19F938F9380EE92E077
:10F6C0009F938F931F921F9282E08F931F921F929E
:10F6D0000E94C7BD0E9408D18DB79EB709969EBFF4
:10F6E0008DBF8091851B81110E947FCE20E043E079
:10F6F0005EE061E080E00E9414B98EEB9BE10E9425
:10F7000059CB81110BC00E9420D120E042E15EE084
:10F7100062E080E00E9414B93BDFE6C081E08093A4
:10F72000680300E020E140E868E080E00E947BB7E9
:10F7300020E044E25EE067E083E10E9414B920E04B
:10F7400047E25EE061E080E00E9414B920E04DE213
:10F750005EE061E08BE00E9414B920E044E35EE0EB
:10F7600062E080E00E9414B920E04AE35EE062E0DB
:10F770008BE00E9414B922E041E45EE063E080E0A7
:10F780000E9414B920E047E55EE066E080E00E9458
:10F7900014B910927008C1E0C09334080E9417CFCA
:10F7A000811103C01092680374C00E94CC6D409117
:10F7B000EC13E12C00E022E030E050E061E085E075
:10F7C0000E94EBBE40916C0824E030E050E061E024
:10F7D00081E10E94EBBE4091EB1322E030E050E06B
:10F7E00062E085E00E94EBBE40911B1450911C1416
:10F7F0004115510541F420E04DE55EE062E080E115
:10F800000E9414B908C0E12C00E024E030E062E07E
:10F8100080E10E945DBF2091E7133091E813409191
:10F82000E9135091EA13C12CE12C00E064E080E080
:10F830000E94CAC0209111143091121440911314E7
:10F840005091141464E08CE00E94CAC040911D14D1
:10F8500050911E1425E030E066E085E00E945DBF17
:10F8600020E043E65EE066E08BE00E9414B920E011
:10F8700043E051E066E08DE00E9440B980E10E94E3
:10F880009972882309F488CF80916803882309F44A
:10F8900083CF0E9458B5109234088091680381117B
:10F8A0000DC020E045E65EE061E00E9414B940E052
:10F8B00060E870E080E991E00E94DD7220E042E7BC
:10F8C0005EE063E080E00E9414B920E04EE75EE075
:10F8D00064E080E00E9414B910926803109234082A
:10F8E0000E9418CB0E9420D1CF910F91EF90CF9022
:10F8F00008950F931F93CF93DF9397DE882309F426
:10F900005EC080916D08811112C00E9458B520E040
:10F910004EE75DE063E080E00E9414B920E044E936
:10F920005DE064E080E00E9414B932DE48C00E94CD
:10F930009C498CE99DE00E94CA4910E002E21CC08B
:10F94000019FE00111249E01295F3B4D40E050E002
:10F9500061E0812F0E94AE4B4EE050E06EEB7BE108
:10F96000CE01855E9B4D0E9415F4009721F461E065
:10F97000812F0E94C74A1F5F80916D08181700F3FE
:10F9800080E00E943E4E8130C1F40E94884A92E29B
:10F99000899FE0011124BE01655E7B4D4EE050E081
:10F9A0008EEB9BE10E9423F4BE01695F7B4D44E135
:10F9B00050E08AEA9BE10E9423F40E94BD49DF9156
:10F9C000CF911F910F910895CF9340E06FEF7FEF9C
:10F9D0008CE390E00E94DD720E9458B58091AA1BD2
:10F9E000803281F0882371F022E04DEA5DE060E032
:10F9F00080E00E9414B920E04AEA5BE161E080E027
:10FA00000E94C7B820E043EC5DE064E081E00E9422
:10FA100014B98DE190E00E943EDE20E0AC0167E089
:10FA20008BE00E9414B980E20E949972811102C099
:10FA3000C2E001C0C1E080E10E949972811117C04B
:10FA4000C23089F3F2DD882391F00E9458B520E09E
:10FA500046ED5DE060E080E00E9414B90E9408D1AC
:10FA60000E947FCE0E94A8CE0E9420D142DFCF917B
:10FA70000895AF92BF92CF92DF92EF920F93CF9300
:10FA8000DF93EC015B016A01E22FF0E0E031F10568
:10FA900008F032C1EA5BFF4F0C9427F1E12C00E043
:10FAA00023E030E004C0E12C00E025E030E0AE01CE
:10FAB00062E080E10E94EBBE1FC1E12C00E023E088
:10FAC00030E0AC0162E080E10E945DBF15C10097AB
:10FAD00029F08130910509F00FC104C020E04EE803
:10FAE0005EE006C120E048E95EE002C1009729F02F
:10FAF0008130910509F000C103C083E490E002C0A9
:10FB000084E490E00E943EDE20E0AC01E2C0009779
:10FB100029F08130910509F0EFC003C08AE190E03F
:10FB20000FC089E190E00CC0009729F08130910569
:10FB300009F0E2C003C08EE590E002C08DE590E0E0
:10FB40000E943EDE20E0AC0162E081E1D3C000977C
:10FB500029F08130910509F0CFC003C084E490E022
:10FB6000A4C085E490E0A1C0E12C00E023E030E0F7
:10FB7000AC0162E080E10E94EBBECC15DD0580F0B7
:10FB800040E060E870E088EC90E00E94DD7223E0E5
:10FB900030E0A60162E080E10E94EBBEE60113C006
:10FBA000E12C00E023E030E0AE0162E080E10E9461
:10FBB000EBBEF8942B9881E80E944AB58C2F0E94E6
:10FBC0004AB52B9A7894E12C00E023E030E0AE01B6
:10FBD00062E080E1CA15DB0551F40E94EBBE40E013
:10FBE00060E870E088EC90E00E94DD7285C00E94C1
:10FBF000EBBEF8942B9881E80E944AB58C2F0E94A6
:10FC00004AB52B9A789478C083309105D9F028F4BE
:10FC10008130910579F090F409C085309105D1F0DB
:10FC2000A8F08630910509F067C018C020E042EACC
:10FC30005EE04FC020E049EA5EE04BC020E040EBD0
:10FC40005EE047C020E047EB5EE043C020E04EEBC3
:10FC50005EE03FC020E045EC5EE03BC020E04CECC5
:10FC60005EE037C08130910549F028F0823091057F
:10FC700009F042C006C089E490E005C08AE490E043
:10FC800002C08BE490E00E943EDE20E0AC0162E026
:10FC90008AE030C0009721F08130910569F503C0FA
:10FCA0008FEC90E002C080ED90E00E943EDE20E00C
:10FCB000AC0162E08EE01EC0009721F0813091051A
:10FCC000D9F404C020E043ED5EE003C020E049ED3C
:10FCD0005EE062E08FE00EC0009739F08130910560
:10FCE00059F420E04FED5EE003C020E045EE5EE019
:10FCF00062E08CE00E9414B9DF91CF910F91EF90F8
:10FD0000DF90CF90BF90AF900895EF920F93213086
:10FD100049F4E12C00E023E030E0AC0162E082E154
:10FD20000E9423BF0F91EF900895A1E0B0E0EBE9AE
:10FD3000FEE70C94F2F02C016B015A0150927C14F6
:10FD400040927B1429830E9458B5898190E00E94DB
:10FD50003EDE20E0AC0162E080E00E9414B9202F7A
:10FD6000A501B601C20185DE82E090E00E943EDE80
:10FD700020E0AC0167E080E00E9414B9F12C45015D
:10FD80008E189F0811E037016C0C7D1C80E40E94E6
:10FD90009972882321F08414950488F007C062E0EA
:10FDA00080E40E94D1728111F6CF09C01093370808
:10FDB0004E0C5F1C202FA501B601C2015ADE80E85F
:10FDC0000E949972882321F04614570488F007C0D6
:10FDD00062E080E80E94D1728111F6CF09C01093D1
:10FDE00037084E185F08202FA501B601C20141DE79
:10FDF00080E10E94997281110EC080E20E94997286
:10FE0000882321F280EF0E94997210923708409067
:10FE10007B1450907C14C2012196E0E10C940EF109
:10FE2000EF92FF920F931F930E949C4980E59FE001
:10FE30000E94CA4980E8E82E8FE0F82E0FE61FE006
:10FE400020E63FE044EE5CE761E082E00E94654B23
:10FE500090EBE92E9FE0F92E00EA1FE02EE83FE04C
:10FE600049E75CE761E081E00E94654B23EEE22E0A
:10FE70002FE0F22E03ED1FE022EC3FE040EE5AE7C8
:10FE800061E085E00E94654B30E1E32E30E1F32E26
:10FE900002E010E125EF3FE040E050E061E083E068
:10FEA0000E94654B4FE3E42E40E1F42E0EE210E198
:10FEB0002EE130E140E050E061E084E00E94654BDB
:10FEC0005AE5E52E50E1F52E870120E530E14EE2BE
:10FED0005BE761E086E00E94654B80E00E943E4E59
:10FEE0000E94754A853021F10E94884A833079F456
:10FEF000EE24E39404E026EC41E050E060E070E0A2
:10FF00008091CD1B90E011DF8093CD1BE6CF843034
:10FF100021F7EE24E39407E024E841E050E060E0BC
:10FF200070E08091CC1B90E000DF8093CC1BD5CF9C
:10FF30000E94BD491F910F91FF90EF900895A1E09D
:10FF4000B0E0E5EAFFE70C94F2F02C016B015A01F6
:10FF500050927C1440927B1429830E9458B5898169
:10FF600090E00E943EDE20E0AC0162E080E00E9472
:10FF700014B9202FA501B601C201C7DE82E090E0CE
:10FF80000E943EDE20E0AC0167E080E00E9414B9F0
:10FF9000F12C45018E189F0811E036016E0C7F1C74
:10FFA00080E40E949972882321F0841495048CF0D7
:10FFB00007C062E080E40E94D1728111F6CF09C0CF
:10FFC000109337084E0C5F1C202FA501B601C2010B
:10FFD0009CDE80E80E949972882321F04614570421
:10FFE0008CF007C062E080E80E94D1728111F6CFE8
:10FFF00009C0109337084E185F08202FA501B601DD
:020000021000EC
:10000000C20183DE80E10E94997281110EC080E2FC
:100010000E949972882321F280EF0E9499721092B7
:10002000370840907B1450907C14C2012196E0E187
:100030000C940EF1CF93DF93C82F80937B14109212
:100040007C140E9458B584E290E00E943EDEAC0130
:1000500020E061E080E00E9414B985E290E00E9417
:100060003EDEAC0120E062E080E00E9414B98091A5
:10007000811B811156C084E290E00E943EDE20E0A8
:10008000AC0160E080E00E9414B986E290E00E943A
:100090003EDE20E0AC0161E080E00E9414B987E21E
:1000A00090E00E943EDE20E0AC0162E080E00E9431
:1000B00014B988E290E00E943EDE20E0AC0163E0EB
:1000C00080E00E9414B989E290E00E943EDE20E0C8
:1000D000AC0164E080E00E9414B98AE290E00E94E2
:1000E0003EDE20E0AC0165E080E00E9414B98BE2C6
:1000F00090E00E943EDE20E0AC0166E080E00E94DD
:1001000014B98FE090E00E943EDE20E0AC0167E091
:100110008CE00E9414B980E20E9499728823D9F37E
:1001200077C0CC2319F0C13079F404C020E04BEE45
:100130005EE006C082E490E00E943EDEAC0120E07A
:1001400062E08EE00E9414B982E090E00E943EDE00
:10015000AC0120E067E080E00E9414B9D091811BDF
:10016000D13009F04FC080E40E949972882391F049
:10017000C11110C0D093370882E490E00E943EDEA7
:1001800020E0AC0162E08EE00E9414B986E00E949B
:1001900042D2C1E080E80E949972882379F0C13090
:1001A00069F4C093370820E041EF5EE062E08EE042
:1001B0000E9414B985E00E9442D2C0E080E10E9412
:1001C00099728823F9F08CE290E00E943EDEAC0147
:1001D00020E064E080E00E9414B98DE290E00E948B
:1001E0003EDEAC0120E065E080E00E9414B942E10F
:1001F00067E080E00E949EB980E10E9499728823A6
:10020000D9F30DC080E20E949972882309F4A6CF29
:1002100080EF0E94997210923708C0917B148C2F46
:10022000DF91CF910895A0E0B0E0E9E1F1E80C940E
:10023000FBF0182FD62EF42EC22F80937B14109231
:100240007C14682F70E080E090E00E9480EE23E351
:1002500033E343E250E40E946DEF0E9452EE60935C
:10026000B3000E9458B58C2F90E00E943EDE20E043
:10027000AC0162E080E00E9414B9E12C00E023E0D0
:1002800030E0412F50E062E080E10E94EBBE20E0D0
:1002900047EF5EE062E081E10E9414B982E090E005
:1002A0000E943EDE20E0AC0167E080E00E9414B9CD
:1002B000C4E6D0E0E12C00E023E030E0412F50E044
:1002C00062E080E10E94EBBE20E8129FC001112491
:1002D000BE010E94A0F0462F01E026E060E280E02F
:1002E0000E947BB780E40E949972882319F01F1541
:1002F00040F023C063E080E40E94D1728111F7CF07
:100300001CC01F5F1F1548F040E060E870E088ECFB
:1003100090E00E94DD721F2D10C0612F70E080E020
:1003200090E00E9480EE23E333E343E250E40E9436
:100330006DEF0E9452EE6093B30080E80E949972C4
:10034000882319F0D116A8F507C063E080E80E9461
:10035000D1728111F7CF2DC0812F90E00197969532
:10036000982F882797958795BE010E94A0F0862F29
:1003700000E026E040E860E20E947BB711501D11CA
:1003800008C040E060E870E088EC90E00E94DD7218
:1003900010C0612F70E080E090E00E9480EE23E3C7
:1003A00033E343E250E40E946DEF0E9452EE60930B
:1003B000B30080E10E9499728823A9F0612F70E058
:1003C00080E090E00E9480EE23E333E343E250E4D8
:1003D0000E946DEF0E9452EE6093B30010937D1B5C
:1003E0001092370821C080E20E949972882309F494
:1003F00061CF80EF0E9499721092370860917B1450
:1004000070917C1480E090E00E947EEE23E333E361
:1004100043E250E40E946DEF0E9452EE6093B300FD
:1004200010917B1410937D1B812FCDB7DEB7E7E0D1
:100430000C9417F1A1E0B0E0E0E2F2E80C94F2F0E5
:10044000182FB62EF42E690199830E9458B522E028
:10045000A60160E080E00E9414B9812E9981992E56
:1004600045E6C42E44E1D42E8601EE24E39417C061
:1004700020E0F401408163E08E2D0E9448B920E025
:1004800049EF5EE063E08E2D8F5F0E9414B9F401A6
:1004900081914F01F80181938F01E394E394802FC0
:1004A0008C198B1528F301E02AE04AE066E183E02D
:1004B0000E94BDB920E04BEF5EE066E080E00E9464
:1004C00014B920E04AE05FE067E080E00E9414B9E0
:1004D000E12C11E0DD24D394E0E2CE2EF9E3AF2E3F
:1004E000AAE59A2EB1E68B2E81E4782E90E3B92E00
:1004F00024E0622E34EF432E55245394F1E0FF168E
:1005000031F083E0F81619F0E4E0FE1260C080E4F8
:100510000E949972882349F0EE2DF0E0DF01AB597B
:10052000BB4E8C918A3740F026C062E080E40E9486
:10053000D1728111F1CF1FC08F5F803210F08C9388
:1005400001C0CC928C9181528F3008F4BC92EB594F
:10055000FB4E80818A53873008F4708280818B55EE
:10056000863008F4808220E0408163E0812F0E9481
:1005700048B9D092370880E80E949972882349F0E0
:100580008E2D90E0FC01EB59FB4E2081213240F48E
:1005900070C062E080E80E94D1728111F1CF69C021
:1005A000322F3C55363018F02150208301C0908204
:1005B00020812A53273008F4A082FC01EB59FB4E1E
:1005C000808181528F3008F04CC0C0824AC0F2E076
:1005D000FF124FC080E40E949972882349F08E2D4B
:1005E00090E0FC01EB59FB4E2081293340F01DC007
:1005F00061E080E40E94D1728111F1CF16C02F5FBB
:10060000203210F0208301C0C082208121522F307F
:1006100008F4B082FC01EB59FB4E20E0408163E01E
:10062000812F0E9448B9D092370880E80E949972C1
:10063000882341F0EE2DF0E0EB59FB4E80818133B1
:1006400040F417C061E080E80E94D1728111F2CFBE
:1006500010C0982F9B53973018F08150808301C0B1
:10066000A08220E0408163E0812F0E9448B9D092AF
:10067000370880E20E94B872882311F181E0F816F1
:1006800031F0E3E0FE1619F0F4E0FF1205C0EE2DA4
:10069000F0E0EB59FB4EC08282E0F81205C0EE2D6F
:1006A000F0E0EB59FB4EB082EE2DF0E0EB59FB4E43
:1006B00020E0408163E0812F0E9448B9D092370842
:1006C00080E20E94A372882309F447C0E1E0FE1291
:1006D00001C00DC0F2E0FF1203C060927D140AC099
:1006E00083E0F81201C003C0E4E0FE1203C08AE018
:1006F00080937D14212F269530E02F5F3F4F40914E
:100700007D1450E0812F880F810F880F00E024179F
:10071000350784F02AE04AE066E183500E94BDB9C3
:1007200001E02AE04AE066E183E00E94BDB9E12CE5
:1007300011E013C02AE04AE066E183500E94BDB98F
:100740001E5F812F880F810F880F01E02AE04AE0A9
:1007500066E183500E94BDB9E39480E10E949972E2
:10076000882309F4CBCEF1E0FF123AC080916514E2
:100770008032B1F57CEFE72E00E020E04FE15FE052
:1007800065E080E00E9404B940E06FE070EF8CE229
:1007900091E00E94DD7280E29EE4F2013197F1F770
:1007A0000197D9F700E027E04FE764E280E00E947C
:1007B0007BB7812F880F810F880F2AE04AE066E11E
:1007C00083500E94BDB901E02AE04AE066E183E07F
:1007D0000E94BDB980EF0E949972E12C11E097CE82
:1007E00081E02196E0E10C940EF1AF92BF92CF929E
:1007F000DF92EF920F931F93CF93DF93EC015B0196
:100800006A010E9458B585E690E00E943EDE20E035
:10081000AC0162E080E00E9414B986E690E00E949C
:100820003EDE20E0AC0165E080E00E9414B987E67E
:1008300090E00E943EDE20E0AC0166E080E00E9495
:1008400014B9D0936414C0936314E12C00E024E045
:1008500030E0AE0162E080E10E94EBBE82E090E019
:100860000E943EDE20E0AC0167E080E00E9414B907
:100870008AE0C81AD10811E080E40E9499728823A6
:1008800021F0CC15DD05C0F407C062E080E40E94D1
:10089000D1728111F6CF10C0109337086496D093AF
:1008A000D91BC093D81BE12C00E025E030E0AE015D
:1008B00062E080E10E94EBBE80E80E94997288238A
:1008C00021F0AC16BD06C0F407C062E080E80E94CB
:1008D000D1728111F6CF10C0109337086497D0936E
:1008E000D91BC093D81BE12C00E025E030E0AE011D
:1008F00062E080E10E94EBBE80E10E94997281116A
:1009000027C00E94D0B4409158085091590800E087
:1009100020E030E063E088E00E9497BF20E045E3FC
:100920005FE063E083E00E9414B980E20E94997264
:10093000882309F4A1CF80EF0E94997210923708A2
:10094000C0916314D0916414D093D91BC093D81B69
:10095000CE01DF91CF911F910F91EF90DF90CF905B
:10096000BF90AF900895EF92FF920F931F930E9454
:100970009C498FE092E10E94CA49BEE2EB2EB2E1AF
:10098000FB2E05E212E12DE132E140E050E061E0B2
:1009900083E00E94654B1CE3E12E12E1F12E8701FA
:1009A00023E332E140E050E061E08EE00E94654BDD
:1009B00001E5E02E02E1F02E870126E432E140E07D
:1009C00050E061E08FE00E94654B8BE7E82E82E10A
:1009D000F82E0DE612E12DE532E140E050E061E055
:1009E00084E00E94654B80912E26813071F4A7EA45
:1009F000EA2EA2E1FA2E08E912E129E832E140E00C
:100A000050E061E085E00E94654B50EDE52E52E13B
:100A1000F52E03EC12E126EB32E140E050E061E01C
:100A200086E00E94654B61E0E62E63E1F62E0FEE54
:100A300012E12DED32E140E050E061E087E00E94FC
:100A4000654B73E2E72E73E1F72E03E113E19801A2
:100A500040E050E061E08AE00E94654BE3E4EE2E66
:100A6000E3E1FE2E0BE313E123E333E140E050E04A
:100A700061E08CE00E94654BF6E6EF2EF3E1FF2E7D
:100A80000AE513E12DE433E140E050E061E08DE060
:100A90000E94654B80E00E943E4E0E94754A853060
:100AA00009F4CAC00E94884A833079F4EE24E394A2
:100AB0000CE02EE442E050E060E070E08091741BB6
:100AC00090E033D98093741BE5CF8E3089F4809108
:100AD0002D1CEE24E39401E022ED4CE050E064EFA5
:100AE0007FEF992787FD90952ADA80932D1CD2CF2E
:100AF0008F3079F4EE24E39407E023ED41E050E0F9
:100B000060E070E080912E1C90E00FD980932E1C45
:100B1000C1CF843079F4EE24E39400E02FE44EEF6B
:100B200050E060E070E08091731B90E0FED880930D
:100B3000731BB0CF8A3079F4EE24E39407E022EB04
:100B400041E050E060E070E08091EE1B90E0EDD875
:100B50008093EE1B9FCF893079F4EE24E39407E075
:100B600021EB41E050E060E070E08091ED1B90E00F
:100B7000DCD88093ED1B8ECF8B3079F4EE24E39498
:100B800000E023EB42E350E060E070E08091EF1B77
:100B900090E0CBD88093EF1B7DCF863079F4EE24A4
:100BA000E3940AE021E54FE350E060E070E08091DB
:100BB0007C1B90E0BAD880937C1B6CCF873079F493
:100BC000EE24E39409E022E544E050E060E070E0C8
:100BD00080917B1B90E0A9D880937B1B5BCF8530F5
:100BE00049F420E544E660E080917D1B1CDB8093A6
:100BF0007D1B50CF8C3079F4EE24E3940FE024E693
:100C000041E050E060E070E08091DA1B90E08DD828
:100C10008093DA1B3FCF8D3009F03CCF4FE057E295
:100C200060E070E08091D81B9091D91BDEDD90933D
:100C3000D91B8093D81B2ECF0E94BD491F910F91C5
:100C4000FF90EF900895A1E0B0E0E9E2F6E80C949F
:100C5000FFF0182F10937B1410927C1429830E94AC
:100C600058B5898190E00E943EDEAC0120E062E050
:100C700080E00E9414B9113019F0133091F51FC0B3
:100C800021E043E050E063E170E089E590E00E94FC
:100C9000F9B920E043E050E063E170E085E690E0E0
:100CA0000E9471BA21E043E050E063E170E085E624
:100CB00090E00E94F9B921E041E050E00CC021E051
:100CC00043E050E063E170E089E590E00E94F9B90B
:100CD00021E043E050E063E170E085E690E00E94AF
:100CE00071BA82E090E00E943EDEAC0120E067E055
:100CF00080E00E9414B980E40E9499728823A9F0D0
:100D0000113099F421E043E050E063E170E089E5BF
:100D100090E00E94F9B921E043E050E063E170E027
:100D200085E690E00E9471BA13E080E80E94997213
:100D3000882339F1133029F521E043E050E063E1E5
:100D400070E089E590E00E94F9B920E043E050E0CE
:100D500063E170E085E690E00E9471BA21E043E033
:100D600050E063E170E085E690E00E94F9B921E08F
:100D700041E050E063E170E085E690E00E9471BAE6
:100D800011E080E10E949972882329F01093DD1B05
:100D9000109237080FC080E20E949972882309F4EC
:100DA000AACF80EF0E9499721092370810917B149D
:100DB0001093DD1B812F2196E3E00C941BF1EF9241
:100DC0000F930E949C498AE39FE00E94CA4988E6EB
:100DD00090E00E943EDE9C0140E050E061E087E050
:100DE0000E949E4B89EA90E00E943EDE9C0140E01A
:100DF00050E061E088E00E949E4B83E590E00E9415
:100E00003EDE9C0140E050E061E08AE00E949E4BA3
:100E10008AED90E00E943EDE9C0140E050E061E0FF
:100E20008BE00E949E4B87EA90E00E943EDE9C0190
:100E300040E050E061E084E00E949E4B88EA90E050
:100E40000E943EDE9C0140E050E061E085E00E94AF
:100E50009E4B8BEA90E00E943EDE9C0140E050E019
:100E600061E089E00E949E4B85EA90E00E943EDEB0
:100E70009C0140E050E061E081E00E949E4B84EAEA
:100E800090E00E943EDE9C0140E050E061E082E0A4
:100E90000E949E4B86EA90E00E943EDE9C0140E06C
:100EA00050E061E083E00E949E4B80E00E943E4E55
:100EB0000E94754A853009F4B3C00E94884A813087
:100EC00049F425EA43E061E08091DD1BBCDE8093BC
:100ED000DD1BEBCF823081F4EE24E39407E024EABB
:100EE00041E050E060E070E08091DC1B90E00E9407
:100EF000957E8093DC1BD9CF8A3081F4EE24E39475
:100F000006E023E541E050E060E070E08091DB1B0B
:100F100090E00E94957E8093DB1BC7CF8B3081F4DD
:100F2000EE24E39407E02AED41E050E060E070E059
:100F300080917A1B90E00E94957E80937A1BB5CFBA
:100F4000833081F4EE24E39407E026EA41E050E0A8
:100F500060E070E08091DE1B90E00E94957E8093BF
:100F6000DE1BA3CF843081F4EE24E39403E027EA70
:100F700047EF50E060E070E08091DF1B90E00E945E
:100F8000957E8093DF1B91CF853081F4EE24E3942E
:100F900007E028EA41E050E060E070E08091E01B6B
:100FA00090E00E94957E8093E01B7FCF873081F494
:100FB000EE24E39403E028E647EF50E060E270E0BF
:100FC0008091721B90E00E94957E8093721B6DCF82
:100FD000883099F494E6E92E02E029EA40E355E7E7
:100FE00060E070E08091E21B9091E31B0E94957E8F
:100FF0009093E31B8093E21B58CF893009F055CFC3
:10100000EE24E39407E02BEA41E050E060E070E07A
:101010008091E51B90E00E94957E8093E51B45CF73
:101020000E94BD490F91EF9008950F931F9341E0E7
:1010300050E0082E02C0440F551F0A94E2F76627BD
:1010400057FD6095762F0091471C1091481C209108
:10105000491C30914A1C402351236223732391E0A1
:10106000452B462B472B09F490E0692F0E94E74A55
:101070001F910F910895CF92DF92EF92FF920F93FD
:101080001F934091471C5091481C6091491C7091DE
:101090004A1C01E010E0082E02C0000F111F0A9444
:1010A000E2F7222717FD2095322F68017901C4222B
:1010B000D522E622F722CD28CE28CF2829F4402BAE
:1010C000512B622B732B04C04027512762277327B3
:1010D0004093471C5093481C6093491C70934A1CD2
:1010E000A4DF1F910F91FF90EF90DF90CF900895B4
:1010F0000E949C4984E49FE00E94CA4980EE90E0EF
:101100000E943EDE9C0140E050E061E081E00E94F0
:101110009E4B81E08ADF81EE90E00E943EDE9C01E2
:1011200040E050E061E082E00E949E4B82E07DDF83
:1011300082EE90E00E943EDE9C0140E050E061E0E3
:1011400083E00E949E4B83E070DF83EE90E00E947C
:101150003EDE9C0140E050E061E084E00E949E4B56
:1011600084E063DF84EE90E00E943EDE9C0140E07C
:1011700050E061E085E00E949E4B85E056DF85EE01
:1011800090E00E943EDE9C0140E050E061E086E09D
:101190000E949E4B86E049DF86EE90E00E943EDE94
:1011A0009C0140E050E061E087E00E949E4B87E0B8
:1011B0003CDF87EE90E00E943EDE9C0140E050E084
:1011C00061E088E00E949E4B88E02FDF88EE90E08F
:1011D0000E943EDE9C0140E050E061E089E00E9418
:1011E0009E4B89E022DF80E00E943E4E0E94754ABD
:1011F000853021F00E94884A3EDFF5CF0C94BD492E
:10120000EF92FF920F931F930E949C4983E690E117
:101210000E94CA49E5E9EE2EE0E1FE2E04E810E165
:1012200023E730E140E050E061E081E00E94654B5F
:101230008091821B882309F44FC021EBE22E20E12C
:10124000F22E0CEA10E127EA30E140E050E061E0E4
:1012500082E00E94654B3AEBE32E30E1F32E8701EA
:1012600026EB30E140E050E061E083E00E94654B16
:1012700048EDE42E40E1F42E0DEC10E12EEB30E1D0
:1012800040E050E061E084E00E94654B56EEE52EC0
:1012900050E1F52E8701970140E050E061E085E0E4
:1012A0000E94654B64EFE62E60E1F62E8701970100
:1012B00040E050E061E086E00E94654B79E1E72E76
:1012C00071E1F72E09E011E12AEF30E142EF53ED31
:1012D00061E087E00E94654B1F910F91FF90EF90B6
:1012E0000895ABE0B0E0E7E7F9E80C94FAF088DFA6
:1012F000F4EFCF2EDD24D39480E00E943E4E0E9476
:10130000754A853009F407C10E94884A182F109247
:101310003708813009F5F090821BEE24E39407E052
:1013200022E641E050E060E070E08F2D90E00E9406
:10133000957E8093821BF816F9F2882349F00E946B
:10134000C2CD892B19F01093841B02C01092841B0C
:101350000E94BD4955DFD0CF823019F50E94A9C641
:101360004BE050E06BE87BE1CE0101960E94C9554D
:1013700028E231E141E06AE0CE0101965BD880913C
:101380003708813009F0B8CF85E694E10E94E15535
:101390004BE050E065E674E18BE89BE10E9423F4AA
:1013A000ABCF833051F58091861B89838091871B59
:1013B0008A838091881B8B838091891B8C831D82FB
:1013C0002EE331E142E064E0CE01019633D8809112
:1013D0003708813009F090CF809165148093861B87
:1013E000809166148093871B809167148093881B7B
:1013F000809168148093891B7FCF843059F50E94B7
:1014000058B58091E61B8093940A0E94C2CD20E0DB
:10141000019749F444E551E163E080E00E9414B98A
:101420000E9459C40FC04FE551E163E080E00E9483
:1014300014B91092841B40E060E470E088EE93E001
:101440000E94DD7288EA91E6F6013197F1F7019783
:10145000D9F752CF853089F50E9458B522E04DE684
:1014600051E160E080E00E9414B920E043E851E1DE
:1014700064E080E00E9414B90BE91BE1F12CE12C3F
:10148000F80141918F0120E065E08F2D0E9448B95D
:10149000E0FE0BC0FAE0FE1540F0F39420E048E8CF
:1014A00051E165E08F2D0E9414B9F394E3948DE02F
:1014B000E812E6CF0E94C87A1FCF863009F01CCF11
:1014C0008091961B89838091971B8A838091981BBA
:1014D0008B838091991B8C831D822AE831E142E045
:1014E00064E0CE0101960E941A8280913708813013
:1014F00009F002CF809165148093961B8091661449
:101500008093971B809167148093981B8091681437
:101510008093991BF1CE0E94BD492B96E8E00C9474
:1015200016F1EF92FF920F931F930E949C4980EA5D
:1015300091E10E94CA498FE290E00E943EDE9C0148
:1015400040E050E061E081E00E949E4B8091811B71
:10155000882309F466C0A9EBEA2EA1E1FA2E8701DF
:101560002DEA31E140E050E061E082E00E94654B0D
:10157000B4EDEB2EB1E1FB2E870127EC31E140E029
:1015800050E061E083E00E94654B10EEE12E11E136
:10159000F12E8701970140E050E061E084E00E9475
:1015A000654B0BEEE02E01E1F02E8701970140E044
:1015B00050E061E085E00E94654B86EFE82E81E116
:1015C000F82E8701970140E050E061E086E00E943C
:1015D000654B9DEFE92E91E1F92E8701970140E0DF
:1015E00050E061E087E00E94654B28EDE22E20E1AB
:1015F000F22E0DEC10E12EEB30E140E050E061E026
:1016000088E00E94654B39E1E32E31E1F32E09E0D9
:1016100011E12AEF30E14FE055ED61E089E00E94F1
:10162000654B1F910F91FF90EF900895EF920F93EC
:10163000CF9377DF80E00E943E4E0E94754A85304E
:1016400009F4B7C00E94884A10923708823081F4AA
:10165000EE24E39400E025E545E050E060E070E032
:101660008091751B90E00E94957E8093751BE2CF60
:10167000833081F4EE24E39400E026E54FE750E068
:1016800060E070E08091761B90E00E94957E8093F0
:10169000761BD0CF843081F4EE24E39405E027E577
:1016A00041E050E060E070E08091771B90E00E94A4
:1016B000957E8093771BBECF853081F4EE24E39432
:1016C00000E028E54FE750E060E070E08091781B93
:1016D00090E00E94957E8093781BACCF863081F499
:1016E000EE24E39400E029E54FE750E060E070E08D
:1016F0008091791B90E00E94957E8093791B9ACF10
:10170000883029F48091E61B0E94504593CF8130A8
:10171000E1F4C091811BEE24E39407E02AE541E067
:1017200050E060E070E08C2F90E00E94957E809306
:10173000811BC81709F47ECF882321F08091E61B16
:101740000E9450450E94BD4974CF873009F072CF86
:101750008091E61B8093940AEE24E3940BE02CEA3C
:1017600046E050E061E070E090E00E94957E80935A
:10177000E61B8093590380936B0880913708813072
:1017800009F058CF8091821B813031F40E9408D13A
:101790000E94C2CD0E9420D18091811B813021F412
:1017A000809159030E9450458091E61B8093940AD2
:1017B00041CF0E94BD49CF910F91EF900895EF92D4
:1017C000FF920F931F930E949C4982E793E10E942E
:1017D000CA49B8E9EB2EB3E1FB2E0AE813E12CE786
:1017E00033E140E050E061E081E00E94654B10ECA5
:1017F000E12E13E1F12E05EB13E127EA33E143EB90
:1018000054E862E082E00E94654B0DECE02E03E1BB
:10181000F02E8701970146E15BE862E083E00E94D9
:10182000654B84EDE82E83E1F82E8701970141E7AF
:1018300059E862E084E00E94654B80912B26882362
:1018400061F0AEEDEA2EA3E1FA2E870197014FE891
:1018500052E462E08FE00E94654B4AEFE42E43E1E0
:10186000F42E0FEE13E123EE33E14FED56E862E084
:1018700086E00E94654B25E034E148E758E862E0E5
:1018800080E10E949E4B5AE1E52E54E1F52E87013E
:1018900021E134E140E15FE762E088E00E94654BCE
:1018A00064E3E62E64E1F62E870124E234E14AEA9D
:1018B00056E662E085E00E94654B74E4E72E74E131
:1018C000F72E8701970147ED59E762E08AE00E9411
:1018D000654BEDE4EE2EE4E1FE2E8701970145E72E
:1018E0005DE861E08CE00E94654BF8E5EF2EF4E1E5
:1018F000FF2E8701970145E95AE761E08EE00E94DB
:10190000654B80E00E943E4E0E94754A8530E9F0AA
:101910000E94884A813039F480917F1B0E941A808E
:1019200080937F1BEECF8D3061F7EE24E39400E0CF
:1019300024E541E050E060E070E08091801B90E0A1
:101940000E94957E8093801BDCCF0E94BD491F9131
:101950000F91FF90EF9008950E9458B58CE190E0B0
:101960000E943EDE20E0AC0162E080E00E9414B9FB
:101970008EE190E00E943EDE20E0AC0167E08CE06A
:101980000E9414B980E10E949972882319F00E9484
:1019900079C4299880E20E94A372882399F380EF8A
:1019A0000E9499720E9458B522E045E654E160E039
:1019B00080E00E9414B922E042E754E160E08CE04C
:1019C0000E9414B981E090E00E943EDE20E0AC016C
:1019D00067E080E00E9414B98AE190E00E943EDE58
:1019E00020E0AC0167E08CE00C9414B9A8E0B0E012
:1019F000ECEFFCE80C94FDF00E94D857892B09F419
:101A00006EC080E00E947DB622E048E754E160E0CD
:101A100080E00E9414B984E690E0909333148093A0
:101A20003214F12C00E010E040E023C048870E940F
:101A300072579C012227488521153140D1F0413051
:101A400041F018F04230A9F408C04B9789F441E006
:101A500010C04B9769F442E00CC08537910531F016
:101A60008637910529F4FF24F39403C011E001C0E7
:101A700001E02091321430913314232B39F01111ED
:101A800005C0011105C0FF2089F20AC0002319F02A
:101A900085E40E94A457112319F085E50E94A457FC
:101AA0002091321430913314232B19F484E50E94D1
:101AB000A457FF2081F086E50E94A4574AE050E039
:101AC000BE016F5F7F4F86E890E00E9473F4CE0105
:101AD00001960E94C05780E00E949EB601C010E0AF
:101AE000812F2896E5E00C9419F10E9458B522E068
:101AF0004EE854E160E080E00E9414B980E290E09A
:101B00000E943EDE20E0AC0162E080E00E9414B959
:101B100081E290E00E943EDE20E0AC0164E080E0E3
:101B20000E9414B920E044EA54E165E080E00E949C
:101B300014B982E290E00E943EDE20E0AC0167E052
:101B400080E00E9414B980E20E949972882319F003
:101B500080EF0C94997280E10E949972882399F326
:101B600083E50E94A4572CE088E190E00FB6F8943A
:101B7000A895809360000FBE20936000FFCF36DFF2
:101B8000882329F00E9479C4B0DF81E0089580E0C5
:101B900008951F93CF93DF9380912E26813019F003
:101BA000C5EED2E002C0CAEED2E080912E2682308D
:101BB00011F4CFEED2E00E9458B587E30E94655140
:101BC000882309F4B2C1DF93CF9380EC94E19F9313
:101BD0008F9383EB94E19F938F9312E01F930E9466
:101BE000ED5188E090E00E943EDE9F938F931F931B
:101BF0000E94ED5186EC94E19F938F931F920E9477
:101C0000ED5187EC94E19F938F931F920E94ED51C9
